:1000000000400020D59300001594000017940000D4
:1000100000000000000000000000000000000000E0
:100020000000000000000000000000001994000023
:1000300000000000000000001B9400001D94000060
:100040001F940000816B0000819700001F94000046
:100050001F940000000000001F9400001F94000087
:10006000C9460000559B00001F9400001F9400002B
:100070001F9400001F9400001F9400001F940000B4
:100080001F940000059800001F9400001F940000BA
:100090001F9400001F9400001F9400001F94000094
:1000A0001F9400001F9400000000000000000000EA
:1000B0000000000000000000000000000000000040
:1000C00010B5064C2378002B07D1054B002B02D02E
:1000D000044800E000BF0123237010BD840200200B
:1000E00000000000341E0100044B10B5002B03D0AB
:1000F0000349044800E000BF10BDC04600000000F6
:1001000088020020341E0100164B002B00D1144B36
:100110009D46402292029A1A924600218B460F4633
:100120001348144A121A0EF0BBFB0F4B002B00D0E1
:1001300098470E4B002B00D0984700200021040068
:100140000D000D48002802D00C4800E000BF0EF062
:1001500067FB2000290009F065FB0EF03BFBC04661
:100160000000080000400020000000000000000027
:1001700084020020C42F00200000000000000000C6
:100180000020704700207047002070470020704713
:1001900010B5034A0421034806F0E4FD10BDC04633
:1001A000CCFE0000ECFE000002000120104011D146
:1001B000042A0ED91368180980B2002809D0013822
:1001C0008000031D11180979002902D001309842DE
:1001D000F8D170470020FCE70378002B03D05AB217
:1001E000002A01DB013070473F229343C03B594254
:1001F0004B41C01803789343802BF4D10130F9E7C9
:1002000010B500240378002B01D1200010BDFFF7AA
:10021000E3FF0134F6E7020000787F2809DDDF28DC
:1002200008DCF8238001DB00184053783F2213409C
:1002300018437047EF280BDCFC21537809019B0120
:100240000007000C0B40034390783F221040EFE77B
:10025000F72812DCFC21537889021B030B40E021B4
:100260008004490308403F210343D07808400343FA
:100270009078FC2280011201E8E701204042D8E793
:1002800070B5002204000D00411C092004F046FD59
:10029000002806D001236200134343600023A342D9
:1002A00000DB70BD9A00A958821891600133F6E70F
:1002B00070B5012803DC1C2001F0E4FC70BD0123B3
:1002C0000C6811201C42F7D04868184206D1042857
:1002D00004D90F2302681340042B01D00E20EBE752
:1002E00004F07AFB64100500002C03DDFFF788FFA3
:1002F000A04205DA1220DFE7FFF76EFF0500013CA0
:100300002800012CF8D1FFF786FF40002043D5E7F5
:10031000F8B54D680F00EB0706D4042D04D90F2360
:100320002E683340092B03D00B2001F0ABFCF8BD45
:100330006B683609B6B25C10731EA3420FD8032156
:1003400020000CF045F86421642803DC0100032838
:1003500000DA03212800891904F012FD05002B683A
:1003600000201B099BB2013B9C42E0D23A68A31CCF
:100370009B005A510123013464001C436C60D6E792
:10038000F0B585B0012803DC1C2001F07BFC12E0F5
:1003900001274B683A000093022806D08B683B4245
:1003A00003D05F10002F00DC17000125009B2B42BB
:1003B00003D00120404205B0F0BD009B042BF8D9CA
:1003C0001B680C680F261900314004292DD12C42DE
:1003D00005D1042C03D923681E40042E01D00E2021
:1003E000D3E70098FFF7E0FEB842E2DB009804F0A4
:1003F000F3FA0600200004F0EFFA03780100002B66
:10040000D7D0781E30180EF001FE041ED1D03378FC
:10041000002B01D0A64202D36800012521E0300064
:10042000FFF7DAFE01350600F1E709293ED1009B0E
:100430005B685B1001939F42BBDC2C422ED1042CE5
:100440002CD923683340042B28D1200004F0C4FAAF
:10045000039602907E1C009AB300D058844202D1C9
:1004600078002843A7E728420ED104280CD9036856
:10047000039A1340042B07D104F0AEFA010002984E
:100480000EF08EFD0028EBD0019B37009E42E1DD8F
:100490008FE71F00019B9F4200DD8AE77B1C0099CC
:1004A0009A008A58A242F4D17800B6E7032900D016
:1004B0007FE71A0992B25B0F92000B40D31A0193A7
:1004C0009F4200DD75E72C4229D1042C27D92268F0
:1004D0001640032E19D1100980B2520F800032400D
:1004E000251D801A019B2E181B1A0193009B781E54
:1004F0000433019A904200DD5BE72A001918B242EA
:100500000FD316D10130400087E7042E07D1200019
:1005100004F062FA05002000FFF746FEE2E70F2034
:1005200033E70C78A4461478A44502D10131013296
:10053000E5E70130DDE70000F0B50D0085B00128EA
:1005400004DC1C2001F09EFB05B0F0BD012708680B
:10055000384206D1042804D90F2102680A40042A2F
:1005600001D00E20EEE76A681740FAD1042AF8D9C4
:1005700013680B40042BF4D104F02EFA04006868D1
:1005800004F02AFA02900EF015FD039000280FD116
:100590002000FFF735FE0190019B0122591C092024
:1005A00004F0BCFB364E3060002815D10020CBE7AC
:1005B000029920000EF02AFD001B43424341200017
:1005C0000193019B5E1C0028E6D0039B0299C01892
:1005D0000EF01CFD0196F4E70122019B5B00134322
:1005E0004360039B002B18D12000FFF7F5FD019B12
:1005F0000500BB4201DC3068A6E7291B200004F09F
:100600000BFC0028D2D0BB1C32689B0098502800FD
:10061000FFF7E2FD01372C00E9E7019B012B02D136
:100620002B68836090E7029920000EF0EFFC012513
:100630000700019B002F13D0AB42DCDB391B2000ED
:1006400004F0EAFB0028B1D032680135AB009850C5
:10065000039B0299FC1820000EF0D8FC0700E8E785
:10066000AB42C8DB20000EF0A5FC0100200004F026
:10067000D3FB00289AD001353368AD00E850BAE7C3
:10068000B40F002010B504F08BF94300012018438B
:1006900010BD0000C30711D404280FD90F2302682E
:1006A0001340032B0AD119400133591AC0234907BB
:1006B000DB051940024B1A40114301607047C046E8
:1006C000FFFFFF9F70B5002805DC1C2001F0DAFA5F
:1006D0000500280070BD01220C68144201D10D20D4
:1006E000F4E701281CD04B681342F8D05B101320AC
:1006F000FF2BEBD81A0619040A431A431B021343B3
:100700006410E243D2171440E11C89101A00032040
:1007100004F004FB051EDCD02100FFF7BBFFD8E787
:100720000023EDE7F7B507000E001C20012F06DDC2
:100730004C68012322001A40009203D10D2001F0E1
:10074000A1FA53E0022F02D08A681A42F6D00123A0
:1007500035681D4200D0A9E0042D00D8A6E01C4158
:10076000002C00DC1C000F2029680840092828D133
:100770006B685B100093022F05D0B368009A5B1082
:100780009A4200DD0093009B01221D1B0135EB43C3
:10079000DB171D40691C092004F0C0FA071E09D0B0
:1007A00001236D001D430300326808334560009942
:1007B000A14201DA3800FEBD0134A100515802C344
:1007C000F5E7042845D1280004F006F9FFF718FDE5
:1007D0000190022F04D0B3685B10984200DD0193B2
:1007E000019BA34204DA002004F00AFB0700E1E7C2
:1007F000280004F0F1F80700009BA34221DB280049
:10080000009704F0E9F805003800FFF7E5FC019BCC
:1008100001340700A342F7DA009BC41A200004F059
:10082000EFFA071EC6D004F0D7F80190306804F044
:10083000D3F82200009B591B411801980EF014F8C0
:10084000B8E73800FFF7C8FC009B070001330093AE
:10085000D2E703282AD10B099BB2490F9B00014024
:10086000591A022F04D0B2685210914200DD1100D3
:10087000A14205DA00220320110004F04FFAB5E787
:1008800003200E1B331DD9170140C91889100022FF
:1008900004F044FA071E00D18CE70136310003341E
:1008A000FFF7F8FE381D29193200C7E7212046E777
:1008B000F7B5002804DC1C2001F0E4F9040014E082
:1008C0000D6801272E003E4011D03D41FF2D01D97A
:1008D0001320F1E700223900032004F01FFA041E60
:1008E00003D03900FFF7D6FE25712000FEBD042D90
:1008F000EED90F232A681340042B1BD12800FFF7E1
:1009000053FCC31C07000320D9170140C9188910E4
:10091000320004F003FA041EE7D03900FFF7BAFEF4
:10092000280004F059F8231D01003A0018000DF0CA
:100930009BFFDAE7092B1FD103206B6832005B10A5
:1009400001930333D9170140C918891004F0E6F95F
:10095000041ECAD00199FFF79DFE019B9E42C4DA96
:10096000B300EB189B683B4204D05B10FF2BAFD861
:10097000A21913710136F0E7032BA9D12C00B4E7BB
:1009800010B57F2902DC0170013010BD1A4B99426D
:100990000CDC40238A115B42134303703F230B405E
:1009A00080214942194341700230EEE7134B9942CE
:1009B00010DC20230A135B4213433F248022037080
:1009C0008B1152422340214013430A4343708270EB
:1009D0000330DAE70A4B9942D7DCF0230370603B1F
:1009E0004370113B8A11FF3B1A4382703F22114032
:1009F0001943C1700430C8E7FF070000FFFF000083
:100A0000FF0F010010B5094C0022206002210920CF
:100A100004F084F92368002803D10A3001F032F988
:100A200010BD032283604260FAE7C046B40F002085
:100A300070B5C30710D544101320FF2C07D800222F
:100A40000121032004F06AF9051E09D10A2001F0F2
:100A500019F90500280070BD0400601E8441EEE70E
:100A60000121FFF717FE2C71F4E710B501240440B3
:100A700002D04410200010BD042810D90F230268B2
:100A80001340042B07D103F0A7FF21000A220EF028
:100A900059FB0400EEE7032B01D10430F5E70D20EC
:100AA00001F0F0F8E6E70000F0B50E0085B0002890
:100AB00003DC1C2001F0E6F817E00F6801243D007C
:100AC000254006D1042F1ED90F233A681340042B6A
:100AD0000DD13800FFF7C9FF02AC01002000FFF77D
:100AE0004FFF011B200004F097F9040032E0092BAE
:100AF00009D17B685B100193019B9C4205DD01F0ED
:100B0000C7F8002819D02A20D4E70134A300F858E8
:100B1000FFF7ABFF01237F280DDD154ADB1890425C
:100B200009DD144A0133904205DD0021124AC30F4A
:100B300082424B419B00ED18DEE7280004F060F98B
:100B4000041E07D0376803F047FF01250600019B0C
:100B50009D4202DD200005B0F0BD0135AB00F85824
:100B6000FFF783FF01003000FFF70AFF0600EEE702
:100B7000FF070000FFFF0000FF0F0100F7B50300B3
:100B800001900E001C20012B11DD0868FFF76DFF9E
:100B900007007068FFF769FF019B05000124022B25
:100BA00008D0B068FFF761FF041E03DC292001F0C4
:100BB00069F8FEBDAF421CDCE81B21000BF008FC0D
:100BC000451C691C0022092004F0A8F80028F0D078
:100BD00001226B00134343609440002379009D423F
:100BE000E7DD17009E000F438619B760013309192E
:100BF000F5E7781B21000BF0EBFB6442451CE0E7B6
:100C000010B504000120084010D104290DD90F238C
:100C10000A681340042B08D1080003F0DDFE010030
:100C200020000EF0BDF94342584110BD0020FCE702
:100C3000F7B50E00012803DC1C2001F023F8FEBDEF
:100C40004D68EB0706D4042D04D90F222B681A40F7
:100C5000092A01D00B20F0E76A681B099BB25410E7
:100C6000A34200D85C1E012731680F404810002FB6
:100C700035D12648FFF7C4FF01230190002813D186
:100C800031682348FFF7BCFF002811D0002C0DD09D
:100C90000122631C013C94409B005A5114436C6038
:100CA00004E00137BA00AB50BC42FADA0020C6E7D4
:100CB00001233068184223D1042821D902680E3359
:100CC0001340042B1CD1FFF7D0FE002807D1316858
:100CD0001048FFF795FF002812D01220ADE700283A
:100CE000FBDD8442F9DB8300EB180433844209DC2A
:100CF0000123621C013C9C40920053511C43CEE7EF
:100D000011209AE75A6801301A60EEE7C5FF00002B
:100D1000C9FF0000B9140100002310B50C000B70CE
:100D2000C30705D50D49421020000EF0FDF808E07C
:100D30000B49002802D0042804D10A4920000EF0F3
:100D400013F910BD0428FCD90F2302681340042BAB
:100D5000F7D103F041FE04490200E5E7930E0100DC
:100D6000B9140100CEFF0000D0FF0000F0B593B031
:100D7000060002911C20012E1DDD029B01251B682F
:100D80001C002C4000D0ADE0042B00D8E6E01A682F
:100D90000F231A40092A4AD10394039A0299920018
:100DA0008A5817002F4005D1042A03D9106818402B
:100DB000092806D0222000F065FF0190019813B0A9
:100DC000F0BD52685210A418039A01320392964261
:100DD000E3D1611C012203F0A1FF0190002802D1A0
:100DE00000230193EAE7019B6400190025435D603D
:100DF0000831029ABB00D05802684368120992B2C7
:100E00005B109A4200D8531E0022934209DCDA4359
:100E1000D21713409B00C918039B01379F42E8DBA0
:100E2000CCE794000519AD6801320D51EDE72700BC
:100E3000032A59D10193029ABB00D3582B42B9D14E
:100E4000042BB7D9186801990140032939D1020947
:100E500092B2430F92000B40D31A1C190137BE42C5
:100E6000E9D10320E31CD9170140C91889100022D9
:100E700003F054FF01900028B2D000252100FFF7B5
:100E800009FC019B1E1D029AAB00D45801231C4291
:100E90001FD1042C1DD90F2123681940032918D113
:100EA000180980B25B0F80000B40C01A00238342F8
:100EB00013DBC343DB17184001353618BD42E2DBB4
:100EC0007CE7042900D075E71800FFF76DF92418B6
:100ED000C4E72000FFF768F9E8E7E2181279F25456
:100EE0000133E4E700273C000F25029ABB00D358EA
:100EF0000122134234D1042B32D918680100294051
:100F0000042935D11800FFF74FF924180137BE42E4
:100F1000EBD1200003F074FF0190002800D15FE7BF
:100F2000029FB600BB19041D029301233D681D42B8
:100F300029D1042D27D90F262B681E40042E37D126
:100F40002800FFF731F90600280003F045FD0100F5
:100F5000200032000DF088FCA41922E02700C3E72E
:100F6000180005A9FFF7D8FE05A80EF023F8CCE776
:100F7000032900D01EE7020992B2430F92000B40F2
:100F8000D31A1C19C2E705A92800FFF7C5FE05A85A
:100F90000EF010F805A90500020020000DF064FC19
:100FA0006419029B0437BB42BFD10023237005E7BD
:100FB000032EF6D11A0992B25B0F92001E40961BC7
:100FC000291DC5E7F0B50D0097B0002806DC1C20F0
:100FD00000F058FE0700380017B0F0BD0C68012182
:100FE00023000B40009306D1042C04D922680F3350
:100FF0001A40092A01D00B20EAE7626852100392D6
:10100000002A03DC009803F0FBFEE3E7504A01925C
:1010100001280BD06868084208D1042806D9026864
:101020001340042B02D103F0D7FC019001980DF07E
:10103000C1FF06000F27039B0834013B05935E4365
:10104000039B02909B00E31804930123206818423D
:1010500073D1042871D901680B003B409C46042BD6
:1010600003D1FFF7A1F8861909E0032B6CD1624682
:101070000B099BB2490F9B0011405A1A9619049B09
:101080000434A342E1D1300003F0BAFE071EA2D01F
:101090002B680793029B002B03D0686803F09CFC2D
:1010A0000190380003F098FC0400009B079A9B0015
:1010B000D3189E68300003F08FFC012333400500F5
:1010C0000693002B01D1042E04D809A93000FFF7A4
:1010D00023FE09AD28000DF06DFF069B0490002B48
:1010E0000ED1042E0CD90F2133681940032907D1E2
:1010F0001A0992B25B0F92000B40D31A351D04936C
:101100002000049A29000DF0AFFB049BE418029B19
:10111000002B0AD0059B009A934206DD2000029A1C
:1011200001990DF0A1FB029BE418009B0133009391
:10113000009A039B9342B8D14DE709A9FFF7ECFD54
:1011400009A80DF037FF8EE703F046FCF9E7C0462B
:10115000CF050100F0B58BB0012806DC1C2000F0A3
:1011600091FD040020000BB0F0BD01230C680226A5
:101170001C4205D11E00042C02D923680E361E40E5
:10118000486803F029FCB34907000DF009FF012569
:1011900000281FD1B04938000DF002FF002800D10F
:1011A0000225AE4938000DF0FBFE002800D10425D1
:1011B000AB4938000DF0F4FE002800D10925A949FB
:1011C00038000DF0EDFE002800D1B5E16B1C03D115
:1011D0003020C4E76D42DDE7701E0828C2D80BF04E
:1011E00059F809001F0054014000C1FFC1FFC1FFB1
:1011F000C1FFAF00A81E0728B4D80BF037F8042EA3
:1012000009B3B3B3B32A042C00D193E10124A9E7B5
:101210009548042C00D09548012103F0FDFDA0E77E
:10122000681E08289ED80BF021F8059D18099D9D81
:101230009D9D140064102BD0042493E78C49621008
:1012400002A80DF071FE02A80DF0B4FE010002A884
:10125000E3E72000FFF7D6FB83E72000FFF7E8FB7A
:101260007FE7681E082800D97CE70BF013F8090017
:10127000130048007BFF7BFF7BFF7BFF7BFF1A0097
:10128000200003F0A9FB79490DF08AFE0028D3D194
:10129000002467E72000FFF7E8FB01244000044337
:1012A00060E7200003F098FBFEF7AAFF714D411C98
:1012B0000600002209202C6003F030FD041E01D13D
:1012C0000A204CE70122730013432868636003F08F
:1012D00083FB0123070000250193AE4200DC41E7B8
:1012E0003800FEF798FF019AAB0040001043E31866
:1012F00098603800FEF770FF01350700EDE7200029
:1013000003F06AFB0DF056FE5A4EC11C0500891011
:1013100000220320346003F001FD041ED0D03668A3
:101320002900FFF7B7F9300003F056FB00239D4278
:1013300000DC17E7C15CE21811710133F7E7032500
:101340006368681E5F10032800D90BE70AF098FF56
:1013500002125D3A012F0BD1A4683C4208D1042C43
:1013600000D8FFE60F2322681340012B00D1F9E6D5
:101370002D20F4E6012F03D1A4683C4200D0F1E611
:101380002C20ECE60136B300E058FFF76EFB01239A
:101390007F280CDD384ADB18904208DD374A0133DC
:1013A000904204DD364A2B00904200DD0023019A72
:1013B000D3180193B742E5DA00F06AFC002804D0A4
:1013C0002A20CCE601260023F3E72A4D01982C6061
:1013D00003F016FD041E00D15AE72E6803F0FCFA54
:1013E0000125AF4200DABDE60135AB00F15801231B
:1013F000194201D12720B2E6224B4910994201D966
:101400003120ACE6FFF7BCFAEBE70320FB1CD91751
:101410000140184DC918891000222C6003F07EFC91
:10142000041E00D14CE739002D68FFF733F9002383
:1014300001219F4200DC95E69A00AA1892680A42B0
:10144000D8D05210FF2A01D9132088E6E018027183
:101450000133EEE79FFF0000A7FF0000AEFF000092
:10146000B5FF0000BAFF0000CEFF0000B914010074
:10147000930E0100B40F0020FF070000FFFF0000E3
:10148000FF0F0100FFFF100035002368681E1E09D2
:10149000B6B25B00B6009B0FF61A082800D961E6C9
:1014A0000AF0F8FE0900120060FE190060FE60FEFE
:1014B00060FE60FE2C00012E00D059E72379042441
:1014C000002B00D04EE6E3E6012E00D058E7247949
:1014D0006400344346E6204D30002C6003F090FC5D
:1014E000296804000423002800D1E9E61A1F964267
:1014F00000DC37E6CA5CE2540133F7E7164D711C95
:10150000002209202C6003F009FC041E286800D189
:10151000D6E6012573002B43636000239E4200DC66
:1015200020E6C21812799900520061182A438A6095
:101530000133F3E7032415E6701E082800D911E6ED
:101540000AF0A8FE8BFE8BFEA2FFDDFE10FE10FE51
:1015500010FE10FEFDFEC046B40F002010B50122A3
:10156000002400280BDD0B681A40141E03D05C1009
:10157000E343DB171C400122904200D04A68611C03
:10158000092003F0CBFB002803D0012364001C4397
:10159000446010BD0A6870B510000125284034D1A0
:1015A000042A32D90F24136849681C40092C17D12A
:1015B00054681B099BB22C41A34200D85C1E844294
:1015C00005DC02200133984206DB00200FE0850095
:1015D0005519A9600130F2E7840011510130F2E79A
:1015E000032C12D1294203D1132000F04BFB70BD14
:1015F0004910FF29F8D81B099BB204329B00D3186D
:101600009342E2D911700132FAE70B2000F03AFB65
:10161000DBE700000123F7B500254E680C003340DE
:101620000193AB420ED11D00042E0BD90F2233685B
:101630001A40092A14D172681B099BB25510AB429B
:1016400000D85D1E27687C10FB074CD439003E484B
:10165000FFF7D6FA002829D0002D12D112203EE043
:10166000042A04D13000FEF79FFD0500EAE7019D42
:10167000032AE7D11D09ADB25B0FAD001340ED1A8F
:10168000E0E70DF0EDFB29000AF088FF4C1C019B00
:10169000002B56D1042E54D932680F331340092B36
:1016A00028D10134A400A4592000FEBD39002748E8
:1016B000FFF7A6FA00281BD1042F0FD90F233A6891
:1016C0001340042B0AD13800FFF7CFF9041E0AD1CA
:1016D00039001F48FFF794FA0028BFD1112000F00D
:1016E000D1FA0400E0E7002CB8DDA542CFDAB5E777
:1016F0002C00CCE7042B1CD1300003F06DF9050061
:10170000012C0EDCFEF768FD461B300003F078FB71
:10171000041EC9D003F060F9320029000DF0A4F8CE
:10172000C2E72B78013C002B98D02800FEF754FD2F
:10173000E5E7032B05D13419E37801245B001C4352
:10174000B2E70B20CBE7C04698FF0000C9FF0000BE
:10175000B9140100F7B54D680E002A0001210A40B6
:101760002FD1042D2DD90F242B68B7681C40092CCC
:1017700014D169681B099BB24C100192A34200D896
:101780005C1E31683448FFF73BFA00282DD00F2348
:101790002A681340092B1DD1012317E0032C10D117
:1017A0000F4203D1132000F06DFAFEBD7A100192B2
:1017B000FF2AF7D81A0992B25B0F92001C40141B43
:1017C000DFE70B20EFE701339A00AF509C42FADAD3
:1017D0000020EAE7032BFBD12B0001335A1BA24266
:1017E000F6DC6A461279DA70F7E736687010F307AC
:1017F00019D431001948FFF703FA002822D1042E2A
:101800001ED90F2332681340042B19D13000FFF783
:101810002CF9002807D131001148FFF7F1F9002811
:101820000ED01220BFE70028FBDD8442F9DB0F2336
:101830002A681340092B07D1013080004751C7E7C0
:101840001120B0E72000F2E7032BC1D16B461B79D2
:101850002D18EB70BCE7C046C5FF0000C9FF0000B3
:10186000B914010070B501240868204207D104288A
:1018700005D90F2501680D40092D02D144682000CB
:1018800070BD032D08D10A0992B24B0F92002B4074
:10189000D31A5B001C43F2E7042DF0D103F09CF84F
:1018A000FEF7AEFC40000443E9E7000010B5034A30
:1018B0000F21034805F056FA10BDC04620FF000076
:1018C0001BFF000000207047042070470120704774
:1018D00010B5002003F094FA10BD002070470020DE
:1018E000704700207047002070470020704700209C
:1018F000704700207047002070470020704700208C
:10190000704701207047000010B5034A0F210348BB
:1019100005F028FA10BDC04668000100E000010093
:10192000704700207047002070470020704700205B
:10193000704700207047002070470020704700204B
:101940007047000010B5034A0821034805F00AFA61
:1019500010BDC04674010100B40101000378002BE2
:1019600003D05AB2002A01DB013070473F22934373
:10197000C03B59424B41C01803789343802BF4D1AC
:101980000130F9E7F8B501270600140008003942D4
:1019900027D104293FD90F230A681A40042A3AD1D3
:1019A0003C4213D1042C11D922681340042B0DD1D1
:1019B00003F012F80500200003F00EF801002800E3
:1019C0000DF0EEFA00282EDB1FD127E0E30722D529
:1019D00003F002F80A2200210DF0B4FB05006010AC
:1019E00010E0174015D1042A15D90F2312681340AF
:1019F000042B10D120004D1002F0EEFF0A22390016
:101A00000DF0A0FB85420EDB08DD002E09DC002076
:101A10000CE04D10E3E70F22054B1A700136022E41
:101A2000F5D8042002E0042076173040F8BDC04607
:101A3000C4020020F8B5060000252C4BEC00E41889
:101A40002379032B09D00135FF2DF6D1300005F0A5
:101A50009DF9002848D1013846E030000DF0AAFA7F
:101A6000EBB202003100180005F016FA002839D157
:101A7000226851688842E6D08300D3189B68013001
:101A8000F02BF7D101238000083012181A42DAD166
:101A9000042AD8D90F21136819400429D3D11B096E
:101AA00098B201230130800010181842CBD10428CD
:101AB000C9D90F2203681340042BC4D102F08CFF54
:101AC00003270400092120000DF05CFA0028BAD099
:101AD000013F441C002FF5D1310020000DF096FA93
:101AE0008442B0D102482843F8BDC0467425002086
:101AF00000FFFFFF10B50124044002D04410200075
:101B000010BD042810D90F2302681340042B07D1FD
:101B100002F062FF21000A220DF014FB0400EEE740
:101B2000032B01D10430F5E70D22014B1A70E6E7D3
:101B3000C4020020012210B5024018D1042802D9A5
:101B400003681A0992B201230B4012D1042902D969
:101B50000B681B099BB20024934206D104309B0002
:101B60000431C318984206D30124200010BD00227E
:101B7000E9E70023EFE704780A78002C01D1002A76
:101B8000F2D0013001319442ECD00024EDE70000A6
:101B9000F7B50700009101933049314B002A02D07C
:101BA00002220A70013A00261A601B68CE54BE4217
:101BB00000DBF7BD009AB300D058294B274D1C68B5
:101BC000C8239B0065191C1B0123184206D0254A17
:101BD0004310210028000DF075F909E0224A002881
:101BE00002D004281BD1214A210028000DF06AF9F7
:101BF0001A4C20000DF0DEF9194A019B1060002BF1
:101C00000BD07B1EB34208DD194B984205D8431C0C
:101C10001360202222540022E2540136C7E7042830
:101C200019D90F2301680B40042B04D102F0D4FE14
:101C3000104A0300CDE7092B03D143680E4A5B101D
:101C4000C7E7032B08D10A0992B2490F92000B4053
:101C5000D31A0A4ABDE70123094ABAE7C5020020A0
:101C6000E8050020930E0100100401001604010095
:101C70001F030000BF1401001B0401002A0401001F
:101C800035040100014B187000207047C402002089
:101C9000024B1878431E98417047C046C40200208A
:101CA000FF22024B1860024B1A707047F0050020AB
:101CB000C4020020002310B51A00FFF769FF034B90
:101CC0000348196805F000FE002010BDE80500205B
:101CD000C502002070B502F009FC094C0100251D69
:101CE0001F2228000DF07EF928000DF063F904236F
:101CF00004308008000118432060200070BDC046F9
:101D0000A0020020C368F0B59F00836889B0DF1986
:101D1000030018330193036901999A00019B009015
:101D20009C18436902939B00CB180393C94B1B7803
:101D3000002B51D192103B6802617F221D12C649CF
:101D400013409B005B58043702929F46009B9B68A0
:101D50000293FA1A009B92109B7812021A43009B7E
:101D6000587805F09DFA0023009A2B701370009BA1
:101D7000009A9B680293FB1A9B10D360019BE41AA4
:101D8000A4101461039B019A9B1A009A9B10536143
:101D900009B0F0BD009B587805F07AFA0023009A4C
:101DA0001370E4E7AB4B1B78002B15D1019A009917
:101DB000A21A92103B680A61029A1D121340A64AA9
:101DC0009B009B580437C0E7019B211DCA1AA14BF9
:101DD000D82A18DD1A221A709E4D2978FF29B5D10C
:101DE00000232B709D4D2B68002BC0DD0123009A32
:101DF000137002F063FBFA232A689B005343181800
:101E0000009B5860B3E720001B780C000560002B96
:101E1000E2D1009992103B680A61029A1D121340A8
:101E20008D4A9B009B5804378FE7019A231D9A1A0D
:101E3000D82A03DD1A22874B1A70CDE720001C0038
:101E40003B68391D0360834B1B78002B01D00F00CA
:101E5000C2E7009992107B680A61029A1D12134032
:101E60007D4A9B009B5808376FE7019B201DC21AD3
:101E7000784BD82A02DD1A221A70ADE72100AD0096
:101E80001B787D1904000D60002BA5D100999210DC
:101E90003B680A61029A1D1213406F4A9B009B58CF
:101EA000043752E7019A231D9A1AD82A03DD1A2211
:101EB000684B1A7090E721001C00694BAD00EB588D
:101EC0000B60644B1B78002B86D1009992103B6805
:101ED0000A61029A1D1213405F4A9B009B58043707
:101EE00033E7043C5E4B2268AD00EA50594B1B7847
:101EF000002B00D070E7019A0099A21A92103B685B
:101F00000A61029A1D121340534A9B009B580437E2
:101F10001BE7534BAE00F058FFF7ECFD4D4B0500AF
:101F20001B78002B09D1043C2068FFF7E3FD45191D
:101F300001206D004A4B0543F550464B1B78002BA2
:101F400000D049E7019A0099A21A92103B680A61F1
:101F5000029A1D121340404A9B009B580437F4E636
:101F6000019B211DCA1A3B4BD82A02DD1A221A7086
:101F700032E70198039D0122A84202D22A000C3ABE
:101F8000126820001B780C000260002B00D023E7B1
:101F9000019A3B688A1A009992100A61029A1D12EE
:101FA00013402D4A9B009B580437CEE6019A231D0F
:101FB0009A1A2849D82A02DD1A230B700CE70198D7
:101FC000039EB0421BD231000C39096825484910E4
:101FD0002D186D1AAD00A95921601C001D4B1B78EE
:101FE000002B00D0F8E6009992103B680A61029A33
:101FF0001D121340184A9B009B580437A5E6182071
:1020000008700021E8E7019B039A93421ED2130057
:102010000C3B1B68134A5B10AD18043CED1A226898
:10202000039BAD00EA500B4B1B78002B00D0D3E68E
:10203000019A0099A21A92103B680A61029A1D1235
:102040001340054A9B009B5804377EE61822014B3B
:102050001A70E8E7C402002010020100F005002019
:102060006C2D0020FDFFFF3F019B039A93422DD270
:10207000D34B043CEE1815000C3D2B685B10F31A93
:102080009B009858FFF736FD04902068FFF732FD5B
:102090002D68049B6D10751B1E1801207600039B94
:1020A000AD000643EE50C74B1B78002B00D093E6E3
:1020B000019A0099A21A92103B680A61029A1D12B5
:1020C0001340C14A9B009B5804373EE61822BD4B83
:1020D0001A70E8E7019B211DCA1ABA4BD82A02DD03
:1020E0001A221A7078E620000C000399AD00695896
:1020F0001B780160002B00D06EE6009992103B68BF
:102100000A61029A1D121340AF4A9B009B58043784
:102110001BE6043C039B2268AD00EA50A94B1B78E8
:10212000002B00D058E6019A0099A21A92103B6841
:102130000A61029A1D121340A34A9B009B58043760
:1021400003E6039BAD005D192B68043C20685E101C
:10215000FFF7D0FC361801209A4B76001B78064317
:102160002E60002B00D037E6019A0099A21A921037
:102170003B680A61029A1D121340934A9B009B58C8
:102180000437E2E5AD00019B641BE61A8D4DA342C6
:102190000FD82B78002B00D01EE6009AB6103B68B3
:1021A0001661029A1D121340874A9B009B58043700
:1021B000CBE5864802F000FC2B78002B00D00BE624
:1021C000009AB6103B681661029A1D1213407E4AAF
:1021D0009B009B580437B8E5AB00FF18002D00DAD0
:1021E000C5E5784B1B78002B00D0F5E5019A0099E6
:1021F000A21A92103B680A61029A1D121340724A99
:102200009B009B580437A0E5043C2368042B04D1B1
:10221000AB00FF18002D00DAA9E56A4B1B78002BF4
:1022200000D0D9E5019A0099A21A92103B680A6180
:10223000029A1D121340644A9B009B58043784E5A0
:10224000043C2368042B04D0AB00FF18002D00DAF7
:102250008DE55C4B1B78002B00D0BDE5019A009901
:10226000A21A92103B680A61029A1D121340564A44
:102270009B009B58043768E5261F3068C3070AD5C2
:1022800040100138002809DB01234000AD0018434D
:102290007F1930606BE5FFF72DFCF2E7494B1B78A7
:1022A000002B01D0340097E5019A0099B21A9210E0
:1022B0003B680A61029A1D121340434A9B009B58D7
:1022C0003400043741E52600019A039B0C369B1A23
:1022D0009B100793B21AD82A02DD1A230B707BE5F4
:1022E00020006C00FF2501236D0025401D43009C4C
:1022F0000560A468009D03943C1BAD78A4102402E3
:102300002C43079D9C409D401C432B4383604460AD
:102310006846009B007E09789870634604983400F4
:10232000C358009892108360002903D008331F001F
:10233000039651E51F0000999B680A61029A1D12DD
:102340001340214A9B000C379B580396FDE4231F42
:102350001D68039A019B93423AD10A20EB0711D4DE
:10236000042D18D90F232A681340042B16D12800F6
:1023700002F032FB0CF01EFEC8239B00984200D9ED
:1023800018000630643004F0BBFD00280FD1043F74
:10239000019B0393EBE40720042DF3D02800431E98
:1023A0009841FA234042FF3318400730EAE7009B88
:1023B0002900587804F086FF0023009A1370E7E79D
:1023C000FDFFFF3FC402002010020100470401008E
:1023D000039B039A0C3B1B6800995B109B00D31A6C
:1023E0000C3B1D601C1D1300083B1B685A108A70B3
:1023F000FF210A40CE49D2005B0057589B0A009A41
:102400009B009760FF18039B019A043B1B685B10BD
:102410009B00D3180393C74BA21A1B789210002B72
:1024200000D0D9E400993B680A61029A1D1213405A
:10243000C14A9B009B58043787E4231F1868FFF7A5
:1024400059FBAD000600641B1E2831DC002812DC9D
:10245000B84B1B78002B00D0BEE4019A0099A21A59
:1024600092103B680A61029A1D121340B24A9B0007
:102470009B58043769E402F021F8033E361802F055
:102480001DF8AE4B801B9842F9D8AA4B1B78002B45
:1024900000D0A1E4019A0099A21A92103B680A6147
:1024A000029A1D121340A44A9B009B5804374CE427
:1024B0000123009A137002F001F8009B0A38861974
:1024C0005E6054E4231F1868FFF714FBAD0006009C
:1024D000641B002812DC974B1B78002B00D07BE498
:1024E000019A0099A21A92103B680A61029A1D1281
:1024F0001340914A9B009B58043726E4904B984226
:1025000003DD1D228B4B1A7066E40123009A1370C1
:1025100001F0D4FFFA239B005E430A3E30186FE4BB
:10252000AB00E41A002328001A002100FFF730FB5B
:10253000844E854D3168280002F06EFC834B316873
:102540001860280005F08AF83168280005F0BCF909
:10255000784B1B78002B00D03EE4019A0099A21A18
:1025600092103B680A61029A1D121340724A9B0046
:102570009B580437FFF7E9FB6E4BAD001B78641BDB
:10258000002B00D028E4019A0099A21A92103B680F
:102590000A61029A1D121340674A9B009B58043738
:1025A000FFF7D3FB009804F00FFD624B1B78002B64
:1025B00000D011E4019A0099A21A92103B680A61B6
:1025C000029A1D1213405C4A9B009B580437FFF788
:1025D000BCFB231F1E68002E47D1083B186801363C
:1025E00006401FD04610220001237100083A0B4319
:1025F0001360002E00DC99E0012372001A43211FB2
:102600000A602200083A12681A41921B04922200C2
:102610000C3A106818422BD0049AAD00D2189A4098
:10262000134331E004281BD90F2203681A40092AFA
:1026300002D146687610D6E7042A08D102F0CCF918
:102640000378002BCFD0FFF789F90136F8E7032A8A
:1026500006D1180980B25E0F80001640861BC2E7C3
:102660001922344B1A70FFF7B7FB7610013EC0E712
:10267000042856D90F2201680A40092A1BD1049B5D
:10268000AD0002339B001B58039AAB50294B1B78BB
:10269000002B01D0FFF7A0FB019A0099A21A92101B
:1026A0003B680A61029A1D121340234A9B009B5803
:1026B0000437FFF74AFB042A2BD1039BAD005B19BB
:1026C000069302F089F90600049D0135012D10DC06
:1026D0003000FFF743F9831B1800049302F090FBCE
:1026E000051E0ED002F078F9049A31000CF0BCF807
:1026F00007E03178013D002906D112220D000D4B73
:102700001A70069B1D60C1E73000FFF727F906002D
:10271000DCE7032A05D1049AAD0082181279520031
:102720007EE71922034B1A70FFF756FB0437ADE71B
:1027300074250020C4020020100201007F9698003A
:1027400080EE3600E8050020C502002008000020C9
:10275000AB00019AE3189B1AD82B18DC01226B1EE0
:10276000002D19DCCF4B1B78002B01D0FFF734FB79
:10277000019A0099A21A92103B680A61029A1D12EE
:102780001340C94A9B009B580437FFF7DEFA1A2210
:10279000C44B1A70FFF720FB22601D000434DEE7F3
:1027A000019A231D9B1ABF4ED82B03DD1A233370C9
:1027B000FFF712FB019B039AAD0093422FD2231F18
:1027C0001868FFF797F9011E26DD039B0C3B1A687A
:1027D0005210824220DB9007801AB44B4018C01878
:1027E000039B8000C258631B1A60AE4B641B1B78AE
:1027F0000434002B01D0FFF7EFFA019A0099A21AD6
:1028000092103B680A61029A1D121340A64A9B006F
:102810009B580437FFF799FA20233370E5E7182314
:10282000FBE7A34BAD001A68631B1C001A609D4BAD
:1028300004341B78002B01D0FFF7CEFA019A0099DF
:10284000A21A92103B680A61029A1D121340964A1E
:102850009B009B580437FFF778FA221F1368042B5C
:1028600002D12200AD007F198E4B1B78002B02D0C5
:102870001400FFF7B1FA01990098511A89103B68CA
:10288000016102991D120B4087499B005B5814009F
:102890000437FFF75AFA043C2368042B04D00023C2
:1028A000AD0023607F1904347E4B1B78002B01D0D0
:1028B000FFF792FA019A0099A21A92103B680A61F6
:1028C000029A1D121340784A9B009B580437FFF769
:1028D0003CFAAB009C46E61A002D1CDC1C22714B16
:1028E0001A70002333606346E41A6E4B04341B787D
:1028F000002B01D0FFF770FA019A0099A21A9210EA
:102900003B680A61029A1D121340674A9B009B585C
:102910000437FFF71AFA002033685A108300F15881
:1029200001230B4003D10D215E4A1170DAE74910F3
:102930008A4200DD0A0001308542EFDC01235200AB
:102940001343CFE7AB009C46E61A002D1CDC1C228B
:10295000544B1A70002333606346E41A514B04341D
:102960001B78002B01D0FFF737FA019A0099A21AC1
:1029700092103B680A61029A1D1213404A4A9B005A
:102980009B580437FFF7E1F9002033685A108300A1
:10299000F15801230B4003D10D21424A1170DAE7AF
:1029A00049108A4200DA0A0001308542EFDC012337
:1029B00052001343CFE723000122083B1968AD0002
:1029C000114222D0231F1B6813421ED01141134114
:1029D0000022994200DA0432631B1A60314B641BF7
:1029E0001B780434002B01D0FFF7F6F9019A009907
:1029F000A21A92103B680A61029A1D1213402A4AD9
:102A00009B009B580437FFF7A0F90220231F1A6888
:102A10004042FEF7B7FF661B3060DFE72300083B4C
:102A200019680123AE00194223D0221F12681A42EE
:102A30001FD019415010CB0FD21788425341A21B0F
:102A40009B001360174BA41B1B780434002B01D090
:102A5000FFF7C2F9019A0099A21A92103B680A6125
:102A6000029A1D121340104A9B009B580437FFF72F
:102A70006CF90120231F1A684042FEF783FFA51B53
:102A80002860DFE72300083B1868231F1968AE00A1
:102A9000A61B0423814202D004280BD800233360F4
:102AA0001FE0C046C402002010020100FCFFFF3FEF
:102AB0000800002001231842F0D10F2302681A40B9
:102AC000042AEBD1033A1142E8D10429E6D90A6875
:102AD0001340042BE2D1FFF72DF8431E98418000EC
:102AE0003060DC4BAD001B78641B0434002B01D03C
:102AF000FFF772F9019A0099A21A92103B680A61D5
:102B0000029A1D121340D44A9B009B580437FFF7CA
:102B10001CF92300083B1868231F1968AE00A61B88
:102B20000023814202D0042802D80423336016E037
:102B300001231842F9D10F2302681A40042AF4D164
:102B4000033A1142F1D10429EFD90A681340042B4A
:102B5000EBD1FEF7EFFF4342584180003060BD4BA0
:102B6000AD001B78641B0434002B01D0FFF734F94F
:102B7000019A0099A21A92103B680A61029A1D12EA
:102B80001340B54A9B009B580437FFF7DEF823003B
:102B90000122083B1968AE00114223D0231F1B6895
:102BA00013421FD05B104A10D80FC9179A424141F7
:102BB000A31B89001960A74BA41B1B780434002BAE
:102BC00001D0FFF709F9019A0099A21A92103B6807
:102BD0000A61029A1D1213409F4A9B009B580437BA
:102BE000FFF7B3F8231F1A680120FEF7CBFEA51BE1
:102BF0002860E0E723000122083B1968AD0011427C
:102C000022D0231F1B6813421ED011411341002202
:102C1000994200DD0432631B1A608E4B641B1B78E3
:102C20000434002B01D0FFF7D7F8019A0099A21ABB
:102C300092103B680A61029A1D121340864A9B005B
:102C40009B580437FFF781F8231F1A680220FEF70C
:102C500099FE661B3060E0E7231F1B68AD00043B54
:102C60005A1E9341621B14009B001360794B04347D
:102C70001B78002B01D0FFF7AFF8019A0099A21A38
:102C800092103B680A61029A1D121340724A9B001F
:102C90009B580437FFF759F82300083B1868FEF7E4
:102CA00029FF231F06001868FEF724FF36180120AD
:102CB000AD00631B1C00760006431E60654B0434A8
:102CC0001B78002B01D0FFF787F8019A0099A21A10
:102CD00092103B680A61029A1D1213405E4A9B00E3
:102CE0009B580437FFF731F82300083B1868FEF7BC
:102CF00001FF231F06001868FEF7FCFE361A0120AC
:102D0000AD00631B1C00760006431E60514B04346B
:102D10001B78002B01D0FFF75FF8019A0099A21AE7
:102D200092103B680A61029A1D1213404A4A9B00A6
:102D30009B580437FFF709F82300083B1868FEF793
:102D4000D9FE231F06001868FEF7D4FE4643012073
:102D5000AD00631B1C00760006431E603D4B04342F
:102D60001B78002B01D0FFF737F8019A0099A21ABF
:102D700092103B680A61029A1D121340364A9B006A
:102D80009B580437FEF7E1FF231F1868FEF7B2FED9
:102D9000061E1CD11F232F4A1370AD00631B1C009D
:102DA0001E602C4B04341B78002B01D0FFF714F865
:102DB000019A0099A21A92103B680A61029A1D12A8
:102DC0001340254A9B009B580437FEF7BEFF2300A3
:102DD000083B1868FEF78EFE310009F0F9FA01266B
:102DE00040000643D9E7AE00A51B2868FEF782FE27
:102DF00006906868FEF77EFE00281AD11F22154B48
:102E00001A70144BA41B1B7828600434002B01D0CB
:102E1000FEF7E2FF019A0099A21A92103B680A613C
:102E2000029A1D1213400C4A9B009B580437FEF770
:102E30008CFFC2178318534019000698049309F0B9
:102E4000ADFB002901DA049BC918012049000843A1
:102E5000D7E7C046C402002010020100231F1868F3
:102E6000FEF748FEC217801850400122AD00631BD8
:102E70001C00400010431860EE4B04341B78002BFC
:102E800001D0FEF7A9FF019A0099A21A92103B689F
:102E90000A61029A1D121340E74A9B009B580437AF
:102EA000FEF753FFAB000793E31A0693012D32D1CF
:102EB0001868FEF71FFEC617AE4304900136049B48
:102EC0009E4201DC04961E00049B0136F61A0BF0AC
:102ED000C7FF310009F062FB049B069ACB18012161
:102EE0005B000B431360079BE41AD24B04341B783E
:102EF000002B01D0FEF770FF019A0099A21A9210E0
:102F00003B680A61029A1D121340CB4A9B009B58F2
:102F10000437FEF71AFF022D0AD1069B1868FEF748
:102F2000E9FD069B06005868FEF7E4FD0490C6E73D
:102F3000012364260493C7E7AB00E61A310028009A
:102F4000049302F0BFF8049B3060E41AB94B0434D8
:102F50001B78002B01D0FEF73FFF019A0099A21ABF
:102F600092103B680A61029A1D121340B24A9B00FC
:102F70009B580437FEF7E9FE2300083B1868FEF76C
:102F8000B9FD231F06001868FEF7B4FD06400120B6
:102F9000AD00631B1C00760006431E60A54B043485
:102FA0001B78002B01D0FEF717FF019A0099A21A97
:102FB00092103B680A61029A1D1213409E4A9B00C0
:102FC0009B580437FEF7C1FE2300083B1868FEF744
:102FD00091FD231F06001868FEF78CFD06430120B3
:102FE000AD00631B1C00760006431E60914B043449
:102FF0001B78002B01D0FEF7EFFE019A0099A21A70
:1030000092103B680A61029A1D1213408A4A9B0083
:103010009B580437FEF799FE2300083B1868FEF71B
:1030200069FD231F06001868FEF764FD4640012075
:10303000AD00631B1C00760006431E607D4B04340C
:103040001B78002B01D0FEF7C7FE019A0099A21A47
:1030500092103B680A61029A1D121340764A9B0047
:103060009B580437FEF771FE231F1868FEF742FDD8
:10307000C0430122AD00631B1C00400010431860D8
:103080006C4B04341B78002B01D0FEF7A5FE019A8F
:103090000099A21A92103B680A61029A1D1213400D
:1030A000654A9B009B580437FEF74FFE2300083B00
:1030B0001868FEF71FFD231F06001868FEF71AFDAB
:1030C00086400122AD00631B1C00760016431E6083
:1030D000584B04341B78002B01D0FEF77DFE019A7B
:1030E0000099A21A92103B680A61029A1D121340BD
:1030F000514A9B009B580437FEF727FE2300083BEC
:103100001868FEF7F7FC231F06001868FEF7F2FCAC
:1031100006410122AD00631B1C00760016431E60B1
:10312000444B04341B78002B01D0FEF755FE019A66
:103130000099A21A92103B680A61029A1D1213406C
:103140003D4A9B009B580437FEF7FFFD23000C3BD4
:103150001868FEF7CFFC2300083B06001868FEF74E
:10316000C9FCF1170200C317300009F08DFA231FC4
:10317000049005911868FEF7BDFC020004980599BB
:1031800009F012FA43000120AD00661B3400184319
:10319000284B30601B780434002B01D0FEF71CFE56
:1031A000019A0099A21A92103B680A61029A1D12B4
:1031B0001340214A9B009B580437FEF7C6FDAB0025
:1031C000E61A310028000493FEF7C8F9049B30602A
:1031D000E41A184B04341B78002B01D0FEF7FCFDD9
:1031E000019A0099A21A92103B680A61029A1D1274
:1031F0001340114A9B009B580437FEF7A6FDAB0015
:10320000E41A21002800FEF7C5F90A4B1B78002BB1
:1032100001D0FEF7E1FD019A0099A21A92103B68D5
:103220000A61029A1D121340034A9B009B580437FF
:10323000FEF78BFDC402002010020100AB00E61A6D
:10324000310028000493FEF7E5F9049B3060E41A8E
:10325000E44B04341B78002B01D0FEF7BDFD019A2E
:103260000099A21A92103B680A61029A1D1213403B
:10327000DD4A9B009B580437FEF767FDAB00E41A5C
:1032800021002800FEF766FAD64B1B78002B01D0F0
:10329000FEF7A2FD019A0099A21A92103B680A61FA
:1032A000029A1D121340D04A9B009B580437FEF728
:1032B0004CFDAB00E61A310028000493FEF7D2FA69
:1032C000049B3060E41AC74B04341B78002B01D0F8
:1032D000FEF782FD019A0099A21A92103B680A61DA
:1032E000029A1D121340C04A9B009B580437FEF7F8
:1032F0002CFD231F186801F06FFB2200083A1268AA
:103300000300AD00D1072ED4042A0CD910680F2277
:103310001040013808280FD808F0B2FF05252B27E8
:103320000E0E0E0E2900B14918000BF039FE434273
:103330005841631B80001860AA4B641B1B7804343F
:10334000002B01D0FEF748FD019A0099A21A9210B5
:103350003B680A61029A1D121340A34A9B009B58C6
:103360000437FEF7F2FCA249DEE7A249DCE7A249F6
:10337000DAE7A249D8E7019B251DEE1AD82E04DD15
:103380001A22984B1A70FEF727FD01F0A1F84300AE
:10339000012022001843934B2C001B781060002B57
:1033A00001D0FEF719FD009AB6103B681661029A2B
:1033B0001D1213408C4A9B009B580437FEF7C5FC36
:1033C000019B251DEE1AD82E04DD1A22854B1A709A
:1033D000FEF702FD01F072F8894A40001040012218
:1033E0002300104318607F4B2C001B78002B01D06A
:1033F000FEF7F2FC009AB6103B681661029A1D12A5
:103400001340794A9B009B580437FEF79EFC019AB3
:10341000231D9B1A734DD82B03DD1A232B70FEF747
:10342000DBFC01F055F8774B1A68831A904201D201
:10343000754A9B18012022005B00034313602B7820
:103440000434002B01D0FEF7C7FC019A0099A21AA0
:1034500092103B680A61029A1D121340624A9B0057
:103460009B580437FEF771FC01F032F8654BAD0054
:1034700018605C4B641B1B78002B01D0FEF7ACFC82
:10348000019A0099A21A92103B680A61029A1D12D1
:103490001340554A9B009B580437FEF756FC03F037
:1034A000C9FFAE00002815D14E4BA41B1B78002B82
:1034B00001D0FEF791FC019A0099A21A92103B6884
:1034C0000A61029A1D121340474A9B009B58043719
:1034D000FEF73BFC0123A61B28001A003100FEF773
:1034E00057FB4A4D2868643003F00AFD002802D1DA
:1034F000043FFEF73CFC009B29685A78444803F0DF
:10350000E8FE0123009A3400137000F0D7FF414B0E
:103510002A681B68063253431818009B5860FEF750
:1035200026FC03F087FFAE00002815D12D4BA41B0D
:103530001B78002B01D0FEF74FFC019A0099A21ACC
:1035400092103B680A61029A1D121340264A9B00A2
:103550009B580437FEF7F9FBA61B28000123002225
:103560003100FEF715FB294D2868643003F0C8FCD4
:103570000028BDD0264803F06FFEC2E7AD00661BF1
:10358000FEF7A8FB3400174B30601B780434002B87
:1035900001D0FEF721FC019A0099A21A92103B6813
:1035A0000A61029A1D1213400F4A9B009B58043770
:1035B000FEF7CBFB0B4BAD001B78641B002B01D03F
:1035C000FEF70AFC019A0099A21A92103B680A6160
:1035D000029A1D121340044A9B009B580437FEF7C1
:1035E000B4FBC046C4020020100201009FFF00008F
:1035F000A7FF0000AEFF0000B5FF0000BAFF00000B
:10360000FEFFFF7FF405002037894100E805002018
:10361000C502002004000020EF48AA00012D1ADC9A
:103620001C2300210370A31A19600378A41A043420
:10363000002B01D0FEF7D0FB019A0099A21A92103C
:103640003B680A61029A1D121340E44A9B009B5892
:103650000437FEF77AFB019B039EA51A211FB34294
:1036600002D30B682B60E0E72300083B1B680E6861
:103670005B10002B0BDD03990C39096849108B4254
:1036800005DC5B1AD6495B1803999B005E582E60D7
:10369000CBE7AD00661B300000F053FF3400CE4B8B
:1036A00030601B780434002B01D0FEF795FB019AA3
:1036B0000099A21A92103B680A61029A1D121340E7
:1036C000C64A9B009B580437FEF73FFBAD00661BC4
:1036D000300000F038FF3400BF4B30601B780434FA
:1036E000002B01D0FEF778FB019A0099A21A9210E4
:1036F0003B680A61029A1D121340B84A9B009B580E
:103700000437FEF722FBAB00E61A310028000493D1
:1037100000F064FD049B3060E41AAF4B04341B7866
:10372000002B01D0FEF758FB019A0099A21A9210C3
:103730003B680A61029A1D121340A84A9B009B58DD
:103740000437FEF702FBAD00641B200000F0FEFE14
:10375000A14B1B78002B01D0FEF73EFB019A00998C
:10376000A21A92103B680A61029A1D1213409B4AEA
:103770009B009B580437FEF7E8FAAB00E61A3100CD
:103780002800049300F08EFC049B3060E41A924BF6
:1037900004341B78002B01D0FEF71EFB019A009920
:1037A000A21A92103B680A61029A1D1213408B4ABA
:1037B0009B009B580437FEF7C8FAAD00641B20003D
:1037C00000F01EFF844B1B78002B01D0FEF704FB9A
:1037D000019A0099A21A92103B680A61029A1D127E
:1037E00013407E4A9B009B580437FEF7AEFA012136
:1037F000280000F0DFFE784B1B78002B01D0FEF78D
:10380000EBFA019A0099A21A92103B680A61029A97
:103810001D121340714A9B009B580437FEF795FA1E
:103820000021280000F0C6FE6B4B1B78002B01D056
:10383000FEF7D2FA019A0099A21A92103B680A6127
:10384000029A1D121340654A9B009B580437FEF7ED
:103850007CFAAD00661B300000F000FF34005E4BC8
:1038600030601B780434002B01D0FEF7B5FA019AC2
:103870000099A21A92103B680A61029A1D12134025
:10388000564A9B009B580437FEF75FFAAD00661B53
:10389000300000F0F7FE34004F4B30601B780434EA
:1038A000002B01D0FEF798FA019A0099A21A921003
:1038B0003B680A61029A1D121340484A9B009B58BC
:1038C0000437FEF742FAAD00641B200000F0AEFEA4
:1038D000414B1B78002B01D0FEF77EFA019A00992C
:1038E000A21A92103B680A61029A1D1213403B4AC9
:1038F0009B009B580437FEF728FAAD00641B20009C
:1039000004F00EFC344B1B78002B01D0FEF764FA58
:10391000019A0099A21A92103B680A61029A1D123C
:1039200013402E4A9B009B580437FEF70EFAAD0059
:10393000661B300004F0F6FC3400274B30601B7827
:103940000434002B01D0FEF747FA019A0099A21A1D
:1039500092103B680A61029A1D1213401F4A9B0095
:103960009B580437FEF7F1F9AD00641B200004F00A
:1039700051FB194B1B78002B01D0FEF72DFA019A51
:103980000099A21A92103B680A61029A1D12134014
:10399000124A9B009B580437FEF7D7F9AD00661B0F
:1039A000300004F051FB34000B4B30601B780434C2
:1039B000002B01D0FEF710FA019A0099A21A92107A
:1039C0003B680A61029A1D121340044A9B009B58EF
:1039D0000437FEF7BAF9C046C40200201002010005
:1039E000FCFFFF3FAB00E41A2100280002F07AF848
:1039F000E34B1B78002B01D0FEF7EEF9019A0099FA
:103A0000A21A92103B680A61029A1D121340DD4A05
:103A10009B009B580437FEF798F9AB00E41A21008D
:103A2000280001F065FED64B1B78002B01D0FEF775
:103A3000D3F9019A0099A21A92103B680A61029A7E
:103A40001D121340CF4A9B009B580437FEF77DF9A7
:103A5000AB00E41A2100280001F0FCFEC84B1B78E3
:103A6000002B01D0FEF7B8F9019A0099A21A921022
:103A70003B680A61029A1D121340C24A9B009B5880
:103A80000437FEF762F9AB00E41A2100280001F0C8
:103A900009FFBB4B1B78002B01D0FEF79DF9019A63
:103AA0000099A21A92103B680A61029A1D121340F3
:103AB000B44A9B009B580437FEF747F9AB00E61A5F
:103AC00031002800049304F09DFC049B3060E41A4C
:103AD000AB4B04341B78002B01D0FEF77DF9019A23
:103AE0000099A21A92103B680A61029A1D121340B3
:103AF000A44A9B009B580437FEF727F9AB00E61A4F
:103B000031002800049304F085FC049B3060E41A23
:103B10009B4B04341B78002B01D0FEF75DF9019A12
:103B20000099A21A92103B680A61029A1D12134072
:103B3000944A9B009B580437FEF707F9AB00E61A3E
:103B400031002800049304F06DFC049B3060E41AFB
:103B50008B4B04341B78002B01D0FEF73DF9019A02
:103B60000099A21A92103B680A61029A1D12134032
:103B7000844A9B009B580437FEF7E7F8AB00E61A2F
:103B800031002800049304F055FC049B3060E41AD3
:103B90007B4B04341B78002B01D0FEF71DF9019AF2
:103BA0000099A21A92103B680A61029A1D121340F2
:103BB000744A9B009B580437FEF7C7F8AB00E41A21
:103BC0002100280001F00EFF6D4B1B78002B01D067
:103BD000FEF702F9019A0099A21A92103B680A6155
:103BE000029A1D121340674A9B009B580437FEF748
:103BF000ACF8AB00E41A2100280001F07BFE604B1A
:103C00001B78002B01D0FEF7E7F8019A0099A21A61
:103C100092103B680A61029A1D121340594A9B0098
:103C20009B580437FEF791F8AB00E61A31002800E4
:103C3000049301F0DBFD049B3060E41A504B043424
:103C40001B78002B01D0FEF7C7F8019A0099A21A41
:103C500092103B680A61029A1D121340494A9B0068
:103C60009B580437FEF771F8AB00E41A21002800D6
:103C700001F06AFD424B1B78002B01D0FEF7ACF837
:103C8000019A0099A21A92103B680A61029A1D12C9
:103C900013403C4A9B009B580437FEF756F8002D12
:103CA00000DC93E0231F1E68012D0CD12E4207D1AA
:103CB000042E05D90F23326830001340042B10D096
:103CC00001235B4212E0022DFAD12300083B186861
:103CD000C307F5D40428F3D90F2302681340042B3B
:103CE000EED100F079FEFDF7A5FE0300AA00A41AAC
:103CF0005A1C6BD00020022D12D101223240824288
:103D000035D1042E33D90F213068014009292ED135
:103D100071684810FF2108408100914222D1641847
:103D2000019A0099A21A92100A61FF251A001649F9
:103D3000AA438A422CD11D062D0C05432B12069353
:103D4000FF232A121340114ADB0094460493634474
:103D50001B790B49032B01D1FEF7B5FA02230B7037
:103D6000FEF73AF8B518AD68A5500432D5E70B2236
:103D7000034B1A70002323600434FEF72DF8C0466D
:103D8000C40200201002010000FFFFFF7425002084
:103D90008600A61B310098470022374B341D1A605D
:103DA000364B30601B78934201D0FEF715F8019A2C
:103DB0000099A21A92103B680A61029A1D121340E0
:103DC0002F4A9B009B580437FDF7BFFF0023236059
:103DD0002A4B221D1B78002B02D01400FDF7FCFF9C
:103DE00001990098511A89103B68016102991D12CE
:103DF0000B4023499B005B5814000437FDF7A5FFD7
:103E0000AB00E41A2100280003F050FB1B4B1B7889
:103E1000002B01D0FDF7E0FF019A0099A21A921041
:103E20003B680A61029A1D121340154A9B009B5879
:103E30000437FDF78AFFAB00E61A3100280004932F
:103E400003F034FB049B3060E41A0C4B04341B7801
:103E5000002B01D0FDF7C0FF019A0099A21A921021
:103E60003B680A61029A1D121340054A9B009B5849
:103E70000437FDF76AFFC046B40F0020C4020020DB
:103E8000100201000023F7B55A1E0192002B07DA39
:103E900001F03EFE03F022FC03F02EFD19230193F6
:103EA00000263000194B1968B14212DD184B1A6810
:103EB00001328A420FDAF0241A601D68154F6C43F4
:103EC000E35D002B1FD0E419022B06D12000FDF783
:103ED00019FF019BD8E70022EDE7012B0DD1002847
:103EE00001D100F0EBFAF0226A43BB185B680A4983
:103EF000C31A8B4201D80223BB54F0235D43054B08
:103F0000EB5C022BE2D00136CCE7C046EC0500208A
:103F100000000020141C00207F96980080220B4B8C
:103F200052001A600121A822A920094BD20019646D
:103F30009A58C00005321A5006481A50C122C020B3
:103F4000920000039850044B1970704700E100E0A4
:103F5000008000404C05000035060020042070471A
:103F6000F8B550C9012322001A40101E2DD033404D
:103F7000181E2AD0641000201A2C26D81D4B76104B
:103F800035009E4200DD1D001B4F3B5D012B05D01F
:103F90000121200005F02AFE01233B55174B1B7819
:103FA000002B01D1FFF7BAFF0023154A9E420DDC1A
:103FB000FF2514491448D65CB44202D15E00705209
:103FC000D5540133082BF6D10420F8BDD15C8C42C6
:103FD00003D10C4A5B009D52F6E70133082BF5D163
:103FE0000023D15CFF2901D1D454F2E70133082B1F
:103FF000F7D1E9E7881300001806002035060020F5
:10400000240000200E000020DC05000070B530C93F
:10401000012322001A40101E1FD02B40181E1CD056
:1040200064101A2C00D91924174E335D012B05D0CA
:104030000121200005F0DAFD012333556910080045
:10404000124A1038124B904208D9012200215242E4
:1040500020001A6005F0E8FD042070BD1C600D48CA
:1040600008F0B6F90C4B040018800C4B1B78002BA1
:1040700001D1FFF753FF0122094B9A64A922D20014
:10408000995864189C50E7E71806002090860100B4
:104090002000002020A107000C0000203506002091
:1040A0000080004070B501240D68254204D10D2028
:1040B000FDF7E8FD200070BD6D101A2D17D8002403
:1040C000012804DD4C68043C63425C416400094EF5
:1040D000735DA34204D02100280005F087FD7455CC
:1040E000280005F0B7FD03000420012BE3D00020D9
:1040F000E1E7C04618060020F8B501260D68340037
:10410000B04200DD4C682B003340181E0BD023005A
:104110003340181E07D06D10002D05DCA1230020B0
:104120001E4ADB00D650F8BD641000201A2CFAD8C5
:104130001B4F3B5D012B04D00121200005F056FDF3
:104140003E552900174808F043F90A21053008F0C8
:104150003FF9154BA400E258144B12021343A2225C
:104160001349D2008B50134C0C4B9C50124C1951DC
:10417000012412495C50124B196900219950114ACF
:10418000904200DD1000A8228021D2009850012228
:1041900089005A5004201A60C5E7C04600F001406B
:1041A0001806002000B4C404F41801000300030042
:1041B0000060004040A1004014050000040500001C
:1041C00000A00040FFFF0000030010B50120002BFD
:1041D00002DC1B30FDF756FD10BD0000F8B50124D0
:1041E0000B6806000D00234204D10D20FDF74AFDA7
:1041F0002000F8BD5B1004D103F038FF40002043DD
:10420000F7E72000072BF4D80D4A9B009C580D4F70
:104210003B5D002B05D00021200005F0E7FC0023CA
:104220003B55012E06DD6B68042B03D102212000D3
:1042300005F0DCFC200005F087FB01244000DEE7F0
:10424000C80401001806002010B50124044002D063
:104250004410200010BD042810D90F230268134019
:10426000042B07D100F0B8FB21000A220AF06AFFF4
:104270000400EEE7032B01D10430F5E70D20FDF734
:1042800001FDE6E7F8B50C00022803DC1C20FDF771
:10429000F9FCF8BD0868FFF7D7FF06006068FFF774
:1042A000D3FF0500A068FFF7CFFF0100794808F0B1
:1042B0008FF8841E1A2D01D90020EAE7764F7B5D26
:1042C000012B05D00121280005F090FC01237B552E
:1042D0000021280005F0A8FC002C0ED02000013899
:1042E000C046C046C046C046C046C046C046C0469E
:1042F000C046C046C046C046F1D101273100280063
:10430000394005F091FC002C0ED020000138C04649
:10431000C046C046C046C046C046C046C046C0466D
:10432000C046C046C046F1D171103940280005F0A2
:104330007BFC002C0ED020000138C046C046C04691
:10434000C046C046C046C046C046C046C046C0463D
:10435000C046F1D10127B1103940280005F064FCB6
:10436000002C0ED020000138C046C046C046C046D2
:10437000C046C046C046C046C046C046C046C0460D
:10438000F1D1F1103940280005F04EFC002C0ED080
:1043900020000138C046C046C046C046C046C046A0
:1043A000C046C046C046C046C046C046F1D10127FF
:1043B00031113940280005F037FC002C0ED02000C8
:1043C0000138C046C046C046C046C046C046C0468A
:1043D000C046C046C046C046C046F1D17111394002
:1043E000280005F021FC002C0ED020000138C0462A
:1043F000C046C046C046C046C046C046C046C0468D
:10440000C046C046C046F1D10127B111394028004D
:1044100005F00AFC3900002C0ED020000138C046FF
:10442000C046C046C046C046C046C046C046C0465C
:10443000C046C046C046F1D1F6113140280005F013
:10444000F3FB002C0ED020000138C046C046C04609
:10445000C046C046C046C046C046C046C046C0462C
:10446000C046F1D10121280005F0DEFB002C00D16F
:1044700022E720000138C046C046C046C046C046BC
:10448000C046C046C046C046C046C046C046F1D140
:1044900012E7C04640420F00180600200420704773
:1044A00010B5002803DC1C20FDF7ECFB10BD0B68E9
:1044B0000020DB07FAD40D30F6E700000122034BA1
:1044C0001A64A822D20098587047C0460080004065
:1044D0000122054B10B51A64A822FA21D20098587F
:1044E000890007F0EBFE10BD0080004000487047D7
:1044F000E80401001B20704770B5054E0400335CD2
:104500000D008B4202D005F071FB355570BDC046E1
:104510001806002070B50024084D635D012B09D1F9
:104520000021200005F080FB0021200005F05EFB4B
:104530000023635501341B2CEED170BD18060020FA
:10454000704711207047372070470000F8B50127E9
:1045500004683C4202D045683D4203D10D20FDF77E
:1045600091FBF8BD64101A2CFBD80C4E335D012B67
:1045700004D03900200005F039FB375508496D108B
:104580008D4202DCE943C9172940200005F062FA98
:10459000335D012BE5D1034A1355E2E718060020ED
:1045A000FF030000F805002010B50800FFF7CEFF5C
:1045B000002010BD70B505000C001A2814D80E4E4E
:1045C000335C012B04D0012105F010FB012373554E
:1045D0000A4B5B5D002B08D0611E8C41614289054E
:1045E000890D280005F036FA70BD210028004C1E08
:1045F000A14105F019FBF7E718060020F805002097
:10460000036810B5DA0703D40D20FDF73BFB10BD9E
:104610004168581004394A425141FFF7CBFFF6E791
:1046200010B50800FFF7ECFF002010BD37B5694654
:104630000A00064B30CB30C203680220042B02D1A3
:1046400001F008F937BD01F02DF9FBE7580401002E
:1046500010B50800FFF7EAFF002010BD10B5084CA8
:10466000237D002B05D00021142005F0BFFA002384
:104670002375142005F0EEFA43425841800010BD26
:104680001806002010B5084CA37D002B05D0002192
:10469000162005F0ABFA0023A375162005F0DAFA10
:1046A00043425841800010BD18060020A02200237C
:1046B0000349D2008B50034910328B507047C046DB
:1046C00000F0014000600040F7B52F4D2F4EEB6C1D
:1046D000002B14D0A9240023E4003759EB642C4BA1
:1046E000186800280BDB2B4B19784A425141C9B29C
:1046F000197005F099FA284B1B88DF1937512B6D7B
:10470000002B38D00021254B254FF45829653A78E5
:104710000193244D8A4206D02B68072B03D8224AE6
:10472000D05C05F081FA2B68204A0133134004D590
:104730000822013B5242134301331B4900228C469D
:104740002B60082B18D06046C05C591CFF2802D192
:104750000B000122F5E7002A00D02B60012105F0B3
:1047600063FA01233B702B68114A5B009B5A0C349F
:10477000E418019BF450F7BD01235B422B6000233A
:104780003B700C4BF4E7C046FC80004000800040CA
:1047900020000020340600200C0000204C05000002
:1047A00033060020140600202400002007000080AB
:1047B0000E0000205C46000030B50023FF25074CAA
:1047C000074A084859001D5501338852082BF9D172
:1047D0000023054A1370054A136030BD24000020F1
:1047E0000E000020DC050000330600201406002027
:1047F0000122024B52421A607047C046200000203E
:1048000010B5034A0D21034802F0ACFA10BDC046B2
:1048100060040100C70F0100E12170B549021B4887
:1048200004F008FE002401220320194B19491A61E3
:104830005C50043158508018083158501A600630C6
:1048400005F07CF8FF21144AA15401341B2CFBD144
:1048500001220020114B01001A600423104A114D5F
:104860001468002CFCD02C680002013B204311602E
:10487000002BF5D101220C4B1A6004F097FF01F0D8
:104880008DFA04F0B9F804F0B8F870BD9C1B002054
:1048900000800040040500001806002000D0004001
:1048A00000D1004008D5004004D00040F8B50B4EC0
:1048B000070030000D0004F005FE0400A84200DDF2
:1048C0002C003D00EB1B9C4205DD300004F004FE93
:1048D00028700135F6E72000F8BDC0469C1B00207B
:1048E00010B50100014804F0ADFD10BD9C1B002077
:1048F00010B5054C200004F0B3FDE1212000490271
:1049000004F098FD10BDC0469C1B0020C3070CD4CA
:10491000064B1B68834208D8054B1B68984204D895
:10492000031F1B68002B00D01800704740060020B2
:104930003C0600200023012210B50A4899000133EB
:104940004250642BFAD1084B084C1A609722002180
:104950001201200009F0A4FF054B064A6360064BD4
:104960001A6010BD6C2D00200800002044060020B5
:10497000A0250000480600203806002010B5044B92
:10498000044A1A60044B054A1A60FFF7D3FF10BDB2
:1049900040060020440600203C060020B40F002002
:1049A000044B1B681868000980B20238C343DB1748
:1049B000184070473806002000B59BB0020005493A
:1049C00001A80AF0B1FA01A802F04AFD02F094FF32
:1049D000FCE7C046BF0501000B4BC20704D4042806
:1049E00004D80A4B00D00A4B180070470F22036806
:1049F0001A40031D042AF7D0064B092AF4D0064BAF
:104A0000032AF1D0054BEFE79905010016040100D8
:104A100010040100A3050100B3050100AA0501006F
:104A20000020064A0649131F186013681B099BB231
:104A300002339B00D2188A42F5D370474806002003
:104A4000B40F0020F7B50F240126314B314A196805
:104A5000314B324D186813681F002740072F26D8A6
:104A600013681B099BB202339B00D218AA42F2D3EF
:104A700000242B4EA500AD192868FFF747FF01342D
:104A80002860642CF6D1274C2068FFF73FFF206098
:104A9000254C2068002802D0FFF738FF2060002551
:104AA000224B1B680093009B9D4214DBF7BD1B0942
:104AB0009BB29B00D3189A42D2D01F68374208D1CC
:104AC000B94206D2B84204D3043F3F68002F00D059
:104AD0001F60043BEFE7F0236B43154A9B181A78DD
:104AE000002A01D10135DEE71F693C2300266B4314
:104AF000DB199B0001930136BB1BF3D4019BB4006F
:104B00001C1B0B4B1C19A069FFF700FFA061F2E70B
:104B100040060020480600203C060020B40F00207C
:104B20006C2D002008000020B40F0020EC050020B0
:104B3000141C0020F7B50124204246D1234B1B68EA
:104B40009C46984241D3224B1B68019398423CD823
:104B5000031F1B68002B38D10200036800941B0957
:104B60009BB2002B0FD10099131F196090422CD0DB
:104B700015682B1F1B68990069180C68013B1460AD
:104B80000A602A00EDE79D0055192968009C214222
:104B900019D18C4517D8019C8C4214D30E1F346850
:104BA000002C10D10F680F343C40072C08D92F601F
:104BB000151F2B600B680A601B099BB20A00D0E727
:104BC00000993160CDE7013BCBE7F7BD40060020FF
:104BD0003C0600200D4970B50A000D4D1368141FE6
:104BE0001B0926689BB2981C002E0BD000238A421A
:104BF00000D00B0023608300C91880001218AA425D
:104C0000ECD370BD1B011360F7E7C04648060020D7
:104C1000B40F0020F8B5124C27000F223B681D0985
:104C2000ADB213420DD06E1CB600A74204D03200C4
:104C30003900200009F021FE0022A3190436A4192E
:104C40001A600235AD00074B7F199F42E5D31B1B4D
:104C50009B10013B1B012360034B1C60F8BDC04649
:104C600048060020B40F002038060020F0B59BB0A5
:104C7000FFF724FC00240700214AA300D058013488
:104C8000FFF758FF642CF7D11E4B1868FFF752FF4F
:104C90001D4B1868002801D0FFF74CFF00261B4B66
:104CA0001B689E4217DBFFF795FFFFF7CBFEFFF770
:104CB000B1FFFFF703FC164BC21B1B6815491B68AD
:104CC00001A81B099BB2023B0AF02EF901A802F0D1
:104CD000C7FB1BB0F0BDF02575430F4BED182B78CB
:104CE000002B01D10136DAE72B695C1E002CF9DBC1
:104CF000A300EB189869FFF71DFF013CF6E7C046DB
:104D00006C2D002008000020B40F0020EC050020CE
:104D10003806002079050100141C0020F7B5174D56
:104D20004F1C2B6806001B680C001B099BB20192EC
:104D30009F420BDBFFF79AFF2B681B681B099BB296
:104D40009F4203DB0A20FCF79DFFFEBD2868A71CDD
:104D5000BA00DB1B81181B010B6029600021031FB7
:104D600019600F231E4003002401264340C3083A64
:104D70009A189A42E9D9019902C3FAE73806002045
:104D8000F7B503000122134004000D000193002B2E
:104D90002BD1174B1B68834227D8164B1B688342C5
:104DA00023D90F23144F386000681840FFF7B6FF6F
:104DB000019B3C68061E3B6017D0236804301B092A
:104DC0009BB29D4200DD1D00AA00211D251F09F098
:104DD0004BFDFFF725FE2E60FFF734FE00232B600E
:104DE0002268064B1340236034002000FEBDC046FD
:104DF000400600203C060020B40F0020F0FF0F000A
:104E00000323043010B5C117194009188910002276
:104E10000420FFF783FF10BD70B5050008000C00EB
:104E2000FFF7EEFF0023002804D170BDE95CC21833
:104E300011710133A342F9DBE343DB171C4000236C
:104E400004192371F1E7F0B50C009BB0022804DCD3
:104E50001C20FCF717FF1BB0F0BD012308681842A7
:104E600006D1042804D90F2601683140042901D055
:104E70000E20EEE761680D001D40F9D10429F7D935
:104E80000A683240042AF3D1A2681A4201D10D20E7
:104E9000DFE7FFF7A1FD06006068FFF79DFDA7684B
:104EA000010001AC7F103000257003F0EDFE3900E9
:104EB0006423220003F04DFF20000AF07BF801007C
:104EC0002000FFF7A9FFC6E710B51C4CA544041E3F
:104ED00002D1FFF795FF0BE003F0EEFD0138062845
:104EE00028D807F0CDF90909111829042400002059
:104EF0008023DB009D4410BD200003F059FE011B00
:104F00002000FFF789FFF3E7200003F0FFFD4300D7
:104F100001201843ECE780226946D200200003F00C
:104F20000CFE68460AF046F801006846E9E70421ED
:104F30000348E6E70020CCE70420D9E700FCFFFFA8
:104F4000B806010070B50C00022803DC1C20FCF739
:104F500099FE70BD01230868184206D1042804D9BF
:104F60000F2501682940042901D00E20EFE7616870
:104F70001942FAD10429F8D90A682A40042AF4D13E
:104F8000A2681A4201D10D20E1E7FFF725FD0500D7
:104F90006068FFF721FDA46801006410280003F099
:104FA00073FE210003F0B0FEFFF78EFFD1E770B56E
:104FB0000D00012803DC1C20FCF764FE70BD0124F9
:104FC0000868204206D1042804D90F2102680A404B
:104FD000042A01D00E20EFE76A682242FAD1042A9F
:104FE000F8D913680B40042BF4D1FFF7F5FC060049
:104FF0006868FFF7F1FC0100300003F045FE03F0A4
:10500000C7FE40002043D9E7F8B507000C001C207C
:10501000012F0BDD01250868284206D1042804D998
:105020000F2102680A40042A03D00E20FCF72AFE52
:10503000F8BD62682A42F8D1042AF6D913680B40F9
:10504000042BF2D1FFF7C8FC06006068FFF7C4FC30
:105050000100022F14D0A4682C4211D0641030003B
:1050600003F012FE050003F027FD012811D1002CEA
:1050700002DD0135012C06D12800FFF725FFD7E717
:1050800001246442EBE7280003F09FFD013C05008A
:10509000F0E70228F0D1002CEEDD0135012CEBD039
:1050A00000222800110003F0C2FD03F08EFD013C38
:1050B0000500F3E710B502F0BDF9431E98418000EA
:1050C00010BD0000086870B501240500254006D118
:1050D000042804D90F2302681340042B03D00E20A8
:1050E000FCF7D0FD70BDFFF777FC03782900233B68
:1050F0005A4253411022C0180AF024F880239B051D
:10510000C218044B9A4201D91420E9E74000204319
:10511000E8E7C046FFFFFF3F10B50124044002D07E
:105120004410200010BD042810D90F23026813403A
:10513000042B07D1FFF750FC21000A220AF002F8E5
:105140000400EEE7032B01D10430F5E70D20FCF756
:1051500099FDE6E710B50868FFF7DEFF09F088F96A
:1051600005F088F8054B002208F076FB04F028FED5
:1051700009F048F943000120184310BD00408F405A
:1051800010B50868FFF7C8FF07F0F6FB094907F0FC
:10519000C1FA09F0A7F904F06BFE074B002208F0F2
:1051A0005BFB04F00DFE09F02DF9430001201843CC
:1051B00010BDC046D30237390000D040F7B50C000F
:1051C000042803DC1C20FCF75DFDFEBD0868FFF72A
:1051D000A3FF01906068FFF79FFF0600A068FFF73C
:1051E0009BFF0500E068FFF797FF07002069FFF7C6
:1051F00093FFAE4201D11F20E5E7019BC01B9B1B23
:105200005843A91B07F0E4F8C71901207F00384371
:10521000DBE70000F0B50D00A1B0022804DC1C2083
:10522000FCF730FD21B0F0BD0868FFF775FF040002
:105230006868FFF771FF0600A868FFF76DFF0F258C
:1052400007000F2E02DCF543ED173540224E4022B9
:105250003100684609F008FB31004022403110A8B7
:1052600009F002FBF91705220023380007F00CFAB9
:1052700000231A4AAE00801859416B46F2580023A9
:1052800007F002FAE7170D04020C2A430B14650C11
:10529000F9032943E0030125FF246D422406241865
:1052A0004D4140206946091888590021A4185D41E4
:1052B00007F0EAF9CE05420A32436008EE074B12C6
:1052C00030436910801859412B00220007F0B8F9CB
:1052D000430001201843A5E7D00501003C0500006C
:1052E00070B50E00012803DC1C20FCF7CBFC70BD60
:1052F0004B68581009F0BCF8040030680D004010ED
:1053000009F0B6F802000B002000290007F09AFE11
:105310000B4A0C4B04F0F4FD02000B0000200A497C
:1053200008F00CFD0022094B08F096FA084B002209
:1053300008F092FA09F066F8430001201843D6E716
:105340006C45D9CC955BC83F0000F03F40A5E540D7
:1053500000408F4010B5034A0C21034801F002FDC4
:1053600010BDC046580601005006010000207047DD
:1053700010B51E20FCF786FC10BD10B51E20FCF7F2
:1053800081FC10BD10B51E20FCF77CFC10BD10B5D3
:105390001E20FCF777FC10BD10B51E20FCF772FC38
:1053A00010BD10B51E20FCF76DFC10BD10B51E2001
:1053B000FCF768FC10BD10B51E20FCF763FC10BDA7
:1053C00010B51E20FCF75EFC10BD10B51E20FCF7CA
:1053D00059FC10BD10B51E20FCF754FC10BD10B5D3
:1053E0001E20FCF74FFC10BD10B51E20FCF74AFC38
:1053F00010BD10B51E20FCF745FC10BD10B51E20D9
:10540000FCF740FC10BD10B51E20FCF73BFC10BDA6
:1054100010B51E20FCF736FC10BD10B51E20FCF7A1
:1054200031FC10BD10B51E20FCF72CFC10BD10B5D2
:105430001E20FCF727FC10BD10B51E20FCF722FC37
:1054400010BD10B51E20FCF71DFC10BD10B51E20B0
:10545000FCF718FC10BD10B51E20FCF713FC10BDA6
:1054600010B51E20FCF70EFC10BD10B51E20FCF779
:1054700009FC10BD10B51E20FCF704FC10BD10B5D2
:105480001E20FCF7FFFB10BD10B51E20FCF7FAFB39
:1054900010BD10B51E20FCF7F5FB10BD10B5034A7A
:1054A0001F21034801F05EFC10BDC0464407010007
:1054B0003C08010000207047012070470120704720
:1054C000002070470120704700207047002070477F
:1054D000002070470020704710B5034A0921034897
:1054E00001F040FC10BDC046D8090100200A0100AF
:1054F0000120034B1860034B1B688340184370471F
:10550000D40F0020B80F0020F0B5EFF31081012375
:10551000194083F31088134AA1261268124D013AEC
:105520009340A022114FD205F600002B17D02C6813
:10553000945103420BD0C046C046C046C046C04648
:10554000C046C046C0462C68D4515B08EDE7D45134
:10555000C046C046C046C046C046C046F5E781F3D7
:105560001088F0BD2C000020C40F00200C050000A6
:1055700030B585B001AD0C220649280009F074F958
:105580000024285D01210134FEF7B6FF0C2CF8D170
:1055900005B030BD6D0A010030B585B001AD0C22FB
:1055A0000649280009F060F90024285D0021013433
:1055B000FEF7A2FF0C2CF8D105B030BD6D0A01003A
:1055C000F7B56A463B4B01AE1380062393703A4B06
:1055D00033800F23B370FEF771FF384B384DC0187E
:1055E0002B68984201D200232B602C68002C41D1FB
:1055F000375D01213800FEF77FFF013400213800BC
:1056000004F012FB032CF3D1002401276B461E5D2E
:1056100039003000FEF770FF01343900300004F02B
:1056200003FB032CF2D1C8200138C046C046C04657
:10563000C046C046C046C046C046C046C046C0463A
:10564000C046F1D16B4600211878FEF755FF6B4636
:1056500000215878FEF750FF6B4600219878FEF73E
:105660004BFFFEF72BFFFA2300241B01C018286014
:105670002000FEBDFEF722FF2B6800249842F7D3DE
:10568000042004F061F90600052004F05DF93618E5
:10569000062004F059F90B4B9B1B181A0A4BA04229
:1056A00006DB18600023094A2B6013600124DFE742
:1056B0001C60F7E7040500000D0E00001027000035
:1056C000CC0F002043030000B80F0020D40F0020AF
:1056D0000B6810B5044A5B101360044B186803F0A4
:1056E0008EF9002010BDC04630000020D00F0020F1
:1056F0000022054B10B51A60044B1B68934201D081
:1057000003F07BF9002010BDD00F0020C01A00204C
:1057100010B5041E0CDA1A24084BA400E2581F230B
:105720001A401E3B9340064A1360064A136010BDA0
:10573000FEF7E0FEA042EEDDEEE7C046F418010001
:10574000C40F0020180500500200086810B5C307F8
:105750000FD540101823012A03DD4A68042A00D11E
:105760000833054A1360FEF7EBFEFFF7D1FF002078
:1057700010BD01204042EDE72C00002010B50028AC
:105780000CDD0A68131F591E8B4107490B60042A60
:1057900006D0FFF701FF0022044B1A60002010BD65
:1057A000FFF7E6FEFAE7C046C80F0020B80F00205A
:1057B00010B50124044002D04410200010BD04287C
:1057C00010D90F2302681340042B07D1FFF704F907
:1057D00021000A2209F0B6FC0400EEE7032B01D1F8
:1057E0000430F5E70D20FCF74DFAE6E70868F8B558
:1057F000C3071AD5FFF7DCFF0300203B5E2B25D83B
:105800000520434301221D180020114E9D4219D04E
:1058100005211024F75C3C4200D080180139520069
:1058200064100029F7D10133F0E704280ED90F22C4
:1058300003681A40042A09D11B099BB2002B05D02A
:105840000379DAE7012340001843F8BD0120FCE7A3
:10585000790A010070B508680D00FFF7A9FF040080
:105860006868FFF7A5FF621E0100042A14D8451ED0
:10587000042D11D805236B439B18012215009D4070
:105880002B00064805682B430360054B1B68002B63
:1058900002D0200003F0B2F8002070BDD00F00202D
:1058A000C01A002070B508680D00FFF781FF0400E2
:1058B0006868FFF77DFF621E0100042A13D8451EA9
:1058C000042D10D805236B439B1801229A400748EA
:1058D000036893430360064B1B68002B03D0002230
:1058E000200003F08BF8002070BDC046D00F0020D0
:1058F000C01A0020F0B5050089B008680C00FFF759
:1059000057FF0690022D36DD6068FFF751FF0190CA
:10591000A068FFF74DFF04000127231D661E0793B3
:10592000731C0293079B9E4235D005237343059356
:10593000019B019D05330493049BAB421ED0042EB2
:1059400016D86B1E042B13D80122059B2349013B5B
:105950005B199A409446224A0B681068069A3A40AE
:1059600003920DD062461A430A60012200280DD12D
:105970007F000135E0E701240194CDE7029ECFE7E7
:10598000624693430B600028F2D0039A02992800E4
:1059900003F034F8ECE7019B1E1D042E1AD8012CED
:1059A00018D1002505273B0021006B439B19994026
:1059B0000B000A4A013511689943094B11601B68B5
:1059C000002B05D0019B0022581D290003F016F87A
:1059D000052DE8D1002009B0F0BDC046D00F002051
:1059E000C01A0020F0B53B4B85B01B680C00002BA3
:1059F00003D101204042FFF78BFE012627683E407D
:105A00003CD1042F3AD90F233A681340092B35D1E2
:105A10007B685B100293029B9E4258DAB300FB182E
:105A20009868FFF7C5FEFF23050004140012184014
:105A30001C4029492B404043019306F0C9FC030454
:105A4000200025496043039306F0C2FC039C00023A
:105A5000044301982049404306F0BAFC1F4B204301
:105A60001B68202B06D1AD00AD0E1D4BAD00EC58D0
:105A700000022043FFF748FD0136CCE73800FFF76E
:105A800097FEFF26050007140012304012494043DC
:105A900006F09EFC3740040438000F49784306F0B6
:105AA00097FC2E400002044330000B49704306F07F
:105AB0008FFC0A4B20431B68202B06D1AB009B0EAA
:105AC000074A9B009B5800021843FFF71DFD00206A
:105AD00005B0F0BDC40F0020590600002C000020C6
:105AE000540C0100086810B5C30703D5FFF760FE2A
:105AF000054B1860054B1B68002B03D0024B186840
:105B000002F07DFF002010BDD00F0020C01A002041
:105B10009D4B70B51B68002B0DD19C4C2368002B4E
:105B20000AD19B4A1268002A06D19A4B1B68002BA7
:105B300001D0FFF745FD70BD974D2A68002A1BD1A3
:105B4000944A1268002A10D0FFF73AFD0028F2D0DC
:105B5000FFF70EFD8E4B226819681A6000290BD0E2
:105B6000002A09D1FFF718FDE5E7894A1268002AE3
:105B7000F0D1002BEED0EBE700210D2004F054F81B
:105B800000210E2004F050F800210F2004F04CF802
:105B90002E68012E5DD0022E00D1A2E0002E51D140
:105BA000013631007A4C04202368994304F03CF814
:105BB00004212368052019404B42594104F034F870
:105BC00010212368062019404B42594104F02CF85B
:105BD00080212368090119404B4259410C2004F0EF
:105BE00023F880212368090219404B4259410B20B8
:105BF00004F01AF880212368490219404B425941A8
:105C00000A2004F011F880212368890219404B42D0
:105C10005941092004F008F880212368C90219407D
:105C20004B425941082003F0FFFF802321681B03EA
:105C300019404B425941072003F0F6FF31000D2077
:105C400003F0F2FF2B680321581C06F0A7FC296023
:105C500071E702214E4C0720236819404B425941FD
:105C600003F0E2FF0820216801404B42594103F054
:105C7000DBFF80212368C90019404B4259410520B0
:105C800003F0D2FF80212368490119404B4259415A
:105C9000062003F0C9FF80212368C90119404B4247
:105CA0005941042003F0C0FF802123688903194073
:105CB0004B4259410A2003F0B7FF802321681B049F
:105CC00019404B425941092003F0AEFF31000C202E
:105CD00003F0AAFF31000B2003F0A6FF31000E20D5
:105CE000AEE720212A4C0720236819404B42594136
:105CF00003F09AFF40212368082019404B42594184
:105D000003F092FF80212368092019404B4259413A
:105D100003F08AFF80212368490019404B42594112
:105D20000A2003F081FF80212368890019404B423B
:105D300059410B2003F078FF802123688901194025
:105D40004B4259410C2003F06FFF80212368490327
:105D500019404B425941062003F066FF8021236819
:105D6000C90319404B425941042003F05DFF8023D1
:105D700021685B0419404B425941052003F054FF50
:105D800001210F205CE7C046C80F0020D00F002083
:105D9000C00F0020D40F0020BC0F0020012010B540
:105DA0004042FFF7B5FC0020FFF7AEFB012003F0F7
:105DB0001BFD10BD10B5034A0B21034800F0D2FFB4
:105DC00010BDC046540D0100AC0D01008023F0B59C
:105DD00002255B051A690A4C0A4BA1261D510327AF
:105DE0008025F600ED00BA43884202D300221A5102
:105DF000F0BD5F59002FFCD098518018F4E7C046E1
:105E00000405000000E0014010B5002806D1C020C4
:105E1000B02140028902FFF7D9FF10BDB0208021D8
:105E20008002C902F7E7000043425841064B404256
:105E30001840B0239B02C018036800201A0E532A92
:105E400001D11B02180A704700C0FEFF30B50124C3
:105E50008025054B054AED009C505C59002CFCD078
:105E600001600021995030BD00E0014004050000B0
:105E700043425841074B40421840B0239B02C01890
:105E8000A62310B50902DB05090A1943FFF7DEFF57
:105E900010BDC04600C0FEFFF0B5012480260D4BAA
:105EA0000D4DF6005C51002902DC00225A51F0BD74
:105EB000577814783F022743947824042743D478F2
:105EC000043224063C439F59002FFCD010C00139F6
:105ED000E9E7C04600E001400405000070B5050098
:105EE0004B680A009C1C2100A400FFF7D5FF28196D
:105EF00070BD0000134B1B68002B0CD08022B02318
:105F0000D2029B0200280BD11A1D5B681B0E522B7C
:105F100000D110007047B022C02392025B02F1E76B
:105F200082420DD903681B0E522B09D143680233FC
:105F30009B00C018824203D903681B0E522BE9D084
:105F40000020E7E7D8100020F0B50020B7B000240B
:105F5000FFF7D0FF270005002600002D2ED1284D89
:105F60002868FFF761FF32003B000190009425494B
:105F700004A808F0D9FF04A801F072FA224B6420AB
:105F80001C682B68A0215A425341204A5B421340AF
:105F9000B02292029B18E41A6043490206F018FAF4
:105FA000A0225202030000921949220004A808F01E
:105FB000BBFF04A801F054FA37B0F0BDFF226B68B4
:105FC00029689C460233FF180B12013613409C428D
:105FD00000DA1C00FF200A140240039262460140CE
:105FE00001920091039A0B4904A808F09DFF04A8B0
:105FF00001F036FA2800FFF77DFF0500ADE7C04647
:10600000D8100020D10E0100DC10002000C0FEFFDF
:106010007B0E0100BD0E010070B50020FFF704FFEC
:1060200004000120FFF700FF844200DA04000A4B5D
:106030001D686A42554128001D60FFF7E5FEA02259
:106040006B4252021340054A28009B18044A611C07
:106050001360FFF70DFF70BDD81000200480010011
:10606000DC100020F8B50020FFF7DEFE070001205D
:10607000FFF7DAFE3E00204D0643204C0DD1802173
:10608000C020C9024002FFF7A1FE01213000FFF746
:10609000EFFE1B4B2E6023601DE0874209DD0023CD
:1060A000B0212B60164B8902236023680020012554
:1060B00017E0012380212B60124BC9022360F4E713
:1060C000120E522A08D0002800D023600E4801F09A
:1060D000C7F9FFF7A1FFF8BD28005A680232920005
:1060E0009B188B4205D21A68561CE9D10028F2D0C1
:1060F000D1E72160EFE7C046D8100020DC10002077
:106100000480010004C00200960E010070B500205A
:10611000FFF7F0FEFF260500002801D1280070BD22
:1061200003681C143440FFF7E5FEDA2CF4D10500B7
:10613000F2E70000FF2270B51F4CD20000212000C2
:1061400008F0AEFBFF25FFF7E1FF0026002818D17D
:10615000F0210A22194849420B00962553432D018C
:106160001B185D192D78002D07D0154D154E5D19A2
:106170009B191B78DB00E3582B60013A002AEBD116
:1061800070BD03681A142A400A2A0AD11A122A403A
:10619000FF2A03D0D200A1180B71A050FFF7AAFE6E
:1061A000D4E7132AFAD11B122B40FF2BF6D0DB00C9
:1061B000E2181671E650F1E774250020141C002047
:1061C000680900006109000010B59AB0FFF74AFFA6
:1061D000FFF7B0FF00231A000A48D90041580133E5
:1061E0004C1EA1415218FF2BF7D1074901A808F016
:1061F0009BFE01A801F034F9044801F031F91AB00E
:1062000010BDC04674250020060F01001A0F0100C2
:106210008022F0B55200A1B00021684808F040FB90
:10622000802200215200664808F03AFB654BFF27A8
:106230001B681A00049353425A4110000592FFF75D
:10624000E3FD049C0020631E9C415F4B64421C40A4
:106250005E4BE418FFF75AFF0600002E2FD104987A
:10626000FFF7E2FD411C0598FFF702FE059A554B2A
:10627000574D1A602C60FFF75DFFFEF739FB514B5D
:1062800064201B68A0215A4253414F4A5B4213408D
:10629000B0222C6892029B18E41A6043490206F06F
:1062A00097F8A0225202030000924A49220007A850
:1062B00008F03AFE07A801F0D3F821B0F0BD32682B
:1062C000131412123A403B4003921A000A3A092A68
:1062D00049D83A4B039A995C002931D110223E48A3
:1062E00008F0DEFA35002B6803991A123A40914201
:1062F00009D11A143A400B2A27D0132A2DD00A2A82
:1063000001D1354B1D602800FFF7F4FD051EEAD1D1
:10631000314B196800290FD02000FFF7DFFD040082
:106320002D4B5B195968002903D02000FFF7D6FDDB
:10633000040004350C2DF3D1204B0121039A99540C
:106340003000FFF7D7FD060087E73B40022BDADC81
:10635000214A9B00D3185D60D5E7102200211E481A
:1063600008F09EFACFE71A00153A082AE8D8144A2E
:106370000399525C002AE3D13500152B00D015009B
:10638000300003681A143A40152A0FD01D2A00D194
:106390000025FFF7AFFD0028F3D1002D04D0200029
:1063A0002900FFF79BFD0400054BC6E7039A1B126B
:1063B0003B409A42EDD10500EBE7C046D80F0020E4
:1063C000E0100020D810002000C0FEFF04C0020032
:1063D000DC100020600E0100FC2E002010B5FFF73D
:1063E00017FF10BDF0B585B0039203220333DC170D
:1063F000294D1440E4182B68284F5A4253418022FB
:106400005B42D202A4103B409B18A21C0291244E76
:10641000910000910190316800980A18934215D2BA
:10642000FFF7F6FE2B685A42534180225B421F4021
:10643000D202BF183368009A9B189F4206D21948AF
:1064400001F00EF80025280005B0F0BD029B35686C
:1064500019066B461A7BA423DB051343FF222F008A
:10646000090C1943019B12041B0413401943280013
:10647000FFF7ECFC0837281D21003760FFF7E6FC2A
:10648000002C04D00A9A21003800FFF705FD009B7C
:10649000083BFF183760D6E7D810002000C0FEFF89
:1064A000DC1000203A0E0100704770470021094BB4
:1064B000094A59600131516059680029FCD0002116
:1064C0001961012393600222044B8131FF315A503C
:1064D0001A607047FC1000400010004000E100E02E
:1064E0000222064B0121DA670022054B5A61054A58
:1064F00011615A69002AFCD07047C04604E100E0EF
:10650000FC1000400010004010B5044C2378002B14
:1065100001D0FFF7E5FF0020207010BDE111002041
:106520000120024B1B685B00184370476412002077
:106530000120024B1B685B001843704734000020A9
:106540001FB5064B06491A6801A808F0EDFC0821A2
:1065500001A8FEF761FC05B000BDC046681200202E
:10656000A80F01001FB580235B051A6E044901A81E
:1065700008F0DAFC082101A8FEF74EFC05B000BDCA
:10658000A80F010010B5044C200008F013FD010015
:106590002000FEF741FC10BD6D1200200E4B10B51F
:1065A0001B680E4C5A1C0FD00D4C002B0CD00D4C00
:1065B000012B09D00C4C022B06D0094C042B03D024
:1065C0000A4C052B00D1074C200008F0F3FC010019
:1065D0002000FEF721FC10BD38000020AD0F0100A7
:1065E000A7FF0000B80F0100AEFF0000B20F0100CE
:1065F00070B504000D001600FDF76AFF802301222C
:1066000000215B051B6E6270E270020AA271020C2F
:10661000E2711A0A60716372000EA2721A0C1B0EEC
:1066200026702571A1702072E272237370BD000084
:1066300070B5214C2278002A3DD1204B01215A60AF
:106640008022D20511605A68002AFCD0002207205F
:106650001B4B1C4901255A500439585008315A50D7
:1066600019481A4958501A491A485A501A495A5042
:10667000A622D2009D50082218495A500431585081
:1066800002201749585017491748585017480439DD
:106690005850182016495850C12189005A500539C0
:1066A000FF395858921802435A501249124A9950C9
:1066B000FFF7FCFE257070BDE1110020FC000040DA
:1066C000001000400C050000746962751C05000094
:1066D00024050000200004022C0500001405000021
:1066E000340500003C050000FFFF00002110010000
:1066F00054050000E21100200405000013B5094B09
:1067000004000093084B019307280AD8074B1B7815
:10671000002B01D1FFF78CFF6B46054A1957054B3B
:10672000D15013BDE2ECF0F4F8FC0004E1110020BC
:10673000001000400C05000070B50E4B06001B78E1
:10674000002B01D1FFF774FF00200B4D2C78844201
:106750000ED00A4B202219780323091B1940084B3D
:106760004901C918300008F07FF80120013C2C7065
:1067700070BDC046E11100206C120020E011002025
:10678000E2110020002370B588B0984235DD0D6815
:1067900001262C0034409C422FD12300042D2CD9FB
:1067A0000F222B681A402300092A26D16A683F2A43
:1067B00023DD6846FFF7C0FF230000281DD06B468D
:1067C00019783300A14203DB6B461B5D5B0033434A
:1067D000A200AA1801349360202CF2D10921694447
:1067E0004A780B7812021A438B781B041A43CB7831
:1067F0001B061343024A13600423180008B070BD3F
:106800006812002070B5454B8AB01B78002B01D16F
:10681000FFF70EFF02AC2000FFF78EFF002802D129
:1068200000200AB070BD23780B2BF9D96378012BB7
:10683000F6D1E378012BF3D100231120384E394DE6
:1068400033602B7068442379374A417813600278AB
:1068500009021143827812041143C27812060A43D6
:1068600032490A60002B0ED1152169444A780B7811
:1068700012021A438B781B041A43CB781B0613436E
:106880003360002318E0012B1AD1152169444A789E
:106890000B7812021A438B781B041A43CB781A2107
:1068A0001B06134333600E23627C6944934200DD70
:1068B000130000229A422CD100220420EA54B0E7AF
:1068C000022B03D1627B10331621EEE7042B0DD18E
:1068D000152108226944684607F0C6FF009801990F
:1068E00003F0DEF907F08EFD3060CAE7052BC8D152
:1068F000152108226944684607F0B6FF00980199FF
:1069000003F0CEF907F07EFD3060627D0A231E2180
:10691000CBE7885CA8540132CCE7C046E1110020E7
:10692000641200206D120020380000206812002040
:1069300010B5134B04001B78002B01D1FFF778FE34
:10694000FFF7CEFD00200F4A0F49104B54505860FE
:106950000130106058680028FCD000201861013018
:10696000906018690028FCD0094B0A481B785B012D
:106970001B185350FFF7B4FDFFF798FD10BDC0463C
:10698000E11100200010004004050000FC10004050
:10699000E0110020E211002010B588B000281DDDB4
:1069A0000A68012113000B4018D1042A16D90F20C0
:1069B00014682040092811D150683F280EDD980046
:1069C000101880680024084201D04010C4B2684604
:1069D000C4540133202BF2D1FFF7AAFF002008B0E6
:1069E00010BD000010B5002813DD0C68E30710D5BA
:1069F0006410532C0DD8084B1B78002B01D1FFF7E6
:106A000017FEFFF76DFDA123044ADB00D450FFF70A
:106A10004DFD002010BDC046E111002000100040D7
:106A200010B500280EDD0C68E3070BD56410FF2CB1
:106A300008D8054B1B78002B01D1FFF7F9FD034A5D
:106A4000034BD450002010BDE11100200010004085
:106A50002405000010B5002805DD0868C30702D52D
:106A60004010FFF74BFE002010BD70B588B0002825
:106A700020DD0124086804401CD104281AD90F2302
:106A800002681340042B15D1FDF7A6FF060008F09D
:106A900091FA0500122800D912252A0002210D3290
:106AA0006846FFF7A5FD6B465D73A54205DC6846A9
:106AB000FFF73EFF002008B070BD2300325D6B443D
:106AC0009A730134F1E7F0B50D008BB0012832DD87
:106AD00008680122040014402DD104282BD90F236B
:106AE00001680B40042B26D16B68134223D0FDF7BD
:106AF00073FF6E6807007310019308F05BFA0500DE
:106B00000E2800D90E252A000121113202A8FFF714
:106B10006FFD6A46127902AB5A7302AA731293731D
:106B2000019B76141B0ED67313745574A54205DCB5
:106B300002A8FFF7FDFE00200BB0F0BD3A5D02A9F0
:106B400063189A740134F1E730B589B0002814DD78
:106B50000C68E30711D5102268460021FFF748FDB5
:106B60006B466A4665105D73684663122D0E6414A9
:106B70009373D4731574FFF7DBFE002009B030BDAA
:106B8000174B184A5968002903D000215960013178
:106B90009160196900291FD0002018618023DB0053
:106BA000D3581149012B18D1A923DB00D3585B42DC
:106BB0000B600E490B78032B01D801330B700320B7
:106BC0000B490B78013303400B700A495B015B18DA
:106BD000094953500123936070470860FAE7C046A3
:106BE000FC10004000100040340000206C12002017
:106BF000E0110020E21100200405000010B50A4B4E
:106C00001B78002B0ED0FFF76BFCA1230722074C4B
:106C1000DB00E250FFF74AFC0022054B0620E25061
:106C2000FFF76CFD10BDC046E111002000100040D0
:106C30002405000010B5034A1021034800F092F823
:106C400010BDC046280F0100220F0100044A05496B
:106C50001368C85401339B059B0D13607047C046F1
:106C60009C1600209C12002070B5124C124A23681A
:106C7000834202DC0023236018E0115C451C0E00F7
:106C8000FA3E012E07D8AB4211DD515D002902D03A
:106C900028399F2901D82800EAE70100151A565C17
:106CA0006E5401318B42FADC181A206070BD1170ED
:106CB000FAE7C046A81A0020A816002010B5FDF774
:106CC000FDFB064B1A68824201D900221A601B683C
:106CD000C31A034898428041404210BD98120020D8
:106CE000204E000010B5094C094A236812689342EF
:106CF00000D110BD074AD05CFDF7F2FD0028F8D0A6
:106D0000236801339B059B0D2360ECE7A016002050
:106D10009C1600209C12002010B50400064B074A68
:106D20001B6812689B1ADB439B059B0DA34200DB8B
:106D300010BDFFF7D7FFF1E79C160020A01600203A
:106D400070B5FFF7E3F9FF250400002801D120000A
:106D500070BD03681B142B401D2B00D10400FFF7EE
:106D6000C9F8F2E770B5074E33680E2B08DC0C2526
:106D70005D43054C0133285164196160A2603360A2
:106D800070BDC046A41600200C2F0020F0B5B7B08F
:106D9000040008F00FF9012802D8002037B0F0BD38
:106DA00023785B2BF9D1013825182B785D2BF4D192
:106DB00001343A21200008F0E5F8061EEDD0071B4B
:106DC000002FEADD210000243A0004A808F00AF9A7
:106DD00004AB711CDC556F1AA742DEDD1DAD3A0015
:106DE000280008F0FFF8134BEC551B68039501933E
:106DF000019BA342D1DD0C2666430F4B04A9F61874
:106E0000306808F0CDF8051E05D17368B6680293A6
:106E1000029B9D4201DB0134EAE73068039908F0E8
:106E2000BFF837000836002801D17868B6E7013589
:106E3000EEE7C046A41600200C2F002010B5FAF78C
:106E400035FDFEF7B7FFFAF75FFDFDF7D9FCFEF75A
:106E500081FAFEF723FBFFF7EDFE01F033F901F0B5
:106E60009BFD01F0CDFD02F017F8FAF76BFDFEF780
:106E700033FBF9F78DF910BD962210B512010021F0
:106E8000034807F00DFD0022024B1A6010BDC046FA
:106E9000141C0020EC05002070B514007F22174B55
:106EA000C000C0580D00836813401C2B01D0002087
:106EB00070BDC368190011400429F8D101690A4066
:106EC000192AF4D11B0A01339B000C30C018FDF7BE
:106ED00083FD037806000120002BE9D0300008F084
:106EE00069F80023A042E2D1A34201DB0120DFE7E1
:106EF000F15CEA5C9142DAD10133F5E774250020B8
:106F0000064B074A1B6812689B1ADB439B059B0DC7
:106F10000122834200DC0022100070479C160020F2
:106F2000A0160020F8B505000C0016001F1E0ED19B
:106F30000320FFF7E5FF002808D0FA20FFF786FEC0
:106F4000E8B2FFF783FEE0B2FFF780FEF8BD501D08
:106F5000FFF7D6FF0028F9D0FB20FFF777FEE8B255
:106F6000FFF774FEE0B2FFF771FEF0B2FFF76EFEBE
:106F70003012C0B2FFF76AFE3C00E31B9E42E5DD23
:106F80002078FFF763FE0134F7E7000070B50024B6
:106F9000F0250B4B1B68A34202DCFFF76DFF70BDB1
:106FA0002B006343074A9B181A78002A05D05978AA
:106FB000002311201A00FFF7B5FF0134E9E7C046AE
:106FC000EC050020141C0020F8B507000024F02573
:106FD0002B0063430C4A01349E18B74211D031781C
:106FE00000290BD00133D15C002311201A00FFF7D8
:106FF00099FF2A000021300007F052FC0A2CE7D14B
:10700000F8BD024B1C60F9E7141C0020EC050020C1
:10701000F0B5150001222F007A4C1740A5440190CD
:107020000291002F11D005AB1A706A105A70120E1F
:107030001A710522691299706D140299DD70FFF7BB
:1070400071FFCF239B009D44F0BD042D2AD90F244E
:1070500028680440042C32D1022304AA28001371AA
:10706000FDF7BAFC050007F0A5FFC82302009B004E
:10707000984200DD1A007C1C97420DD1984206D937
:10708000614804AB03226149C01807F0EDFB220000
:1070900005AB02990198D2E72700611E695C05AC37
:1070A000E155E8E7042D00D0A7E0032304AA043D3E
:1070B00013716B425D4105AB55710222E9E7092C62
:1070C0007ED1042205AB1A706A685110009169469E
:1070D000521209789A70009A59701F2A01DD2022F5
:1070E00000926A46127806ACDA70009BBB4202DC62
:1070F00005ABE21ACDE70126BB00EB189868064005
:1071000006D1042837D90F210368194002290CD170
:10711000012323704310637042121B0E4014A270AF
:10712000E070237105340137DFE7042921D1022300
:107130002370FDF751FC039007F03CFFA31C1428BB
:1071400009D86070864201D19C19ECE7039A925DE0
:107150009A550136F6E714226270039A925D9A55A9
:107160000136112EF9D12E23E3742375637516347D
:10717000D9E7012907D1032304382370434258413A
:1071800060700234CFE7092909D1042323704368D2
:107190005A1062705B12A370E6700434C3E70329CF
:1071A0000BD1052323700068020992B2430F9200AD
:1071B0000B40D31A63701B12EDE726700134B2E75F
:1071C000032C00D03DE7052205AB01091A7089B2F6
:1071D000420F890022408A1A11125A709970642A4B
:1071E00000DD64220421DA70081F824201DC0432CF
:1071F0004FE7685C58540131F6E7002D00D020E7D6
:1072000053E7C046C4FCFFFF22030000D5FF000087
:1072100070B502000024F0210D4E08006043801973
:107220004578954203D001340A2CF6D170BDF02286
:10723000002107F035FB074A1368013BA34200D148
:107240001460002329001A001120FFF76BFEEDE700
:10725000141C0020EC05002010B5B2B002236A46D1
:107260000400137007F0A6FEC72800D9C72000232A
:10727000984207DC421C6B46FE211420FFF752FEA9
:1072800032B010BD694601335A1EA25CCA54EFE702
:10729000002310B501001A001120FFF743FE10BDB6
:1072A00007B56B46197069465A7013128B70131428
:1072B000120ECB700A716B46010005221320FFF7F6
:1072C00031FE07BD10B50A0001001220FFF7A0FE35
:1072D00010BD10B50C000300110014202200FFF7B0
:1072E00021FE10BD012370B5FF24084A41185B42FE
:1072F000884201D3D84370BD06781D0A23407340ED
:107300009B009B5801306B40F2E7C046A41001007F
:1073100013B50400FE2813D80A4BC200D058002829
:107320000ED0436808309900FFF7DCFF0190092078
:10733000FFF7F2FC01AB042221001720FFF7F2FD5A
:1073400013BDC04674250020F8B500231800254D54
:10735000DA00AA580133511E8A418018FF2BF7D159
:10736000052444430A20FFF7D7FCFB20FFF76EFCFF
:107370002720FFF76BFC0020FFF768FCE0B2241227
:10738000FFF764FCE0B2FFF761FC174BFA211868C5
:1073900005F01EF800260700F300E85800281CD06E
:1073A000436808309900FFF79DFF04000520FFF7B0
:1073B000B3FCF0B2FFF74AFCE0B2FFF747FC200451
:1073C000000EFFF743FC2002000EFFF73FFC200EEB
:1073D000FFF73CFC380002F007FA0136FF2EDBD144
:1073E000F8BDC0467425002004000020F7B50190C8
:1073F000FFF7A6FC01250400FF276D42002C01D1F8
:107400002800FEBD266833143B40152B0DD121000A
:107410000198083107F0C4FD002801D135123D4024
:107420002000FEF767FD0400E8E71D2BF8D10125D9
:107430006D42F5E7002010B5074C236883420AD05F
:10744000FDF73CF822680300904200D3831A002025
:10745000024A9A42404110BD98120020BFC62D003A
:1074600030B5B3B00500FFF7E5FF002816D00223C2
:107470006A462800137007F09DFD0400C72800D954
:10748000C7240023A3420BDB20003230FFF744FC6B
:10749000621C6B46FF211420FFF744FD33B030BD62
:1074A000694601335A1EAA5CCA54EBE7F0B5BDB079
:1074B00005900C00012803DC1B20FAF7E3FB55E0E4
:1074C0002C4B08680393C30709D4042807D90F235A
:1074D00002681340042B02D1FDF77EFA0390254B7E
:1074E00060680493C30709D4042807D90F230268EE
:1074F0001340042B02D1FDF76FFA049000261E4BB7
:107500001B680893089BB3420BDC049B1B4A009347
:10751000C821039B0AA807F0D5FC0AA8FFF7A0FF23
:10752000CAE70C257543164B0399ED18286807F038
:1075300037FD071E05D16B68AD680993099B9F4213
:1075400001DB0136DEE728680499079507F028FD7E
:107550000835069000280BD121000598079B0831BB
:107560005B6802389847074B069A1A603DB0F0BD39
:107570000137E3E7CF050100A416002089100100C0
:107580000C2F0020B40F0020F7B5234B06001B681A
:10759000F02100930023009A9A4211DC0024F0238A
:1075A0001A006243019201991C4A55182F78002F46
:1075B00012D001340A2CF3D11948FFF751FF29E00A
:1075C0000A005A43154882185078B04202D1127806
:1075D000002A1FD10133DEE7F0223900280007F02E
:1075E0005FF902230D4A0199EB6053540D4AF100F3
:1075F0008A58009B6E70AE70AA602F616F61A342C3
:1076000002DC054B01341C60002331001A001020FD
:10761000FFF788FCF7BDC046EC050020141C0020D5
:10762000D11401007425002010B5FFF7AFFCFF2432
:10763000084AE3005B429B18074AD35C043B012BDA
:1076400003D8E043C0B2FFF79FFF013C002CEFD10D
:1076500010BDC046FC07000074250020F8B50500E9
:107660000E00FDF7D9FBFF240D4B18600D4AE30017
:107670005B429B180C4AD35C062B01D0032B0BD129
:10768000E743FFB2320029003800FFF705FC00286D
:1076900002D03800FFF778FF013C002CE6D1F8BD9E
:1076A00008000020FC0700007425002070B50500CC
:1076B000FF24084AE3005B429B18074AD35CAB42B5
:1076C00003D1E043C0B2FFF75FFF013C002CF0D1D3
:1076D00070BDC046FC07000074250020F7B5FCF71C
:1076E000EDFE574B1A68824201D900221A601A68CF
:1076F0005449821A8A420DD9FF2253491860D30097
:107700005248CB1A1B181B78073B022B0CD9013AA5
:10771000002AF4D1F7BD0720FFF7C8FF4C4B27E044
:107720000820FFF7C3FF38E0FCF7D2FE071E00D1A8
:1077300001270020FCF792FF01900020FCF7A2FF38
:10774000019B0090434C444D002B12D02368002B2A
:107750006ED12B682760002B6ED0404B01261B7822
:10776000002BD8D10920FFF7A1FF394B1E703B4BEE
:107770001E70009B002B12D02B68002B0FD12368AA
:107780002F60002B1ED0324B01261B78002BC7D157
:107790000920FFF78BFF2E4B1E70304B1E702368A5
:1077A000002B0FD02A4E3278002A0BD19F4200D2F4
:1077B00027602368FB1A312B04D90720FFF776FFD7
:1077C000012333702B68002B0FD0244E3278002A0F
:1077D0000BD1BB4200D92F602B68FF1A312F04D97F
:1077E0000820FFF763FF012333702368002B0CD0C0
:1077F000019B002B09D1164E3378002B02D10720B4
:10780000FFF754FF0023236033702B68002B00D157
:1078100080E7009B002B00D07CE7104C2378002BE6
:1078200002D10820FFF742FF00232B60237071E78D
:10783000009A002AA0D1B5E7009B002B9FD1AEE7AC
:10784000941200200F27000074250020FC07000080
:1078500088120020841200208C1200209012002038
:1078600013B50400FFF792FBFEF71FFE0023009301
:10787000134B1B68002B02D16846FCF7D7FE04238C
:1078800001A901200193FDF779FF00210800FDF710
:107890002FFFFEF73DF9FFF7B1F9FCF707FFFCF703
:1078A0008BFFFCF7A5FFFEF779FAFCF733FE002CFF
:1078B00004D0FDF73FF80348FFF7D2FD13BDC046E3
:1078C000C01A0020C214010070B50D003235060048
:1078D00028000C00FFF714FB002806D1FFF7AAFDD3
:1078E000002808D02800FFF717FA330022000021F3
:1078F0001B20FFF717FB70BDF0B5A1B0FFF7F2F941
:107900008021A94CA94F2068C900091AC019FCF7A9
:10791000CDFF2368C0182060002811D0FCF7CEFDF1
:10792000A34B18603B78FA2B00D04FE12368022B61
:1079300008DCFFF7C3F9002802D00120FFF794F913
:1079400021B0F0BD7B78BC78981E242800D91FE1B7
:1079500004F0AAFC250038003C00400043004C0025
:107960001E015600880092009900AF00EE0005014C
:107970001E011E011E011E011E011E011E011E010F
:107980001E011E0119011E011E011E011E011E0104
:107990001E011E011E011E011E011E019600FF2C6C
:1079A0000ED02000FFF734FC0022824BE100CA50C9
:1079B0005B181A712100009213001320FEF712FDCC
:1079C0000320BBE72000FFF7DFFDF9E72000FFF70A
:1079D0001FFCF5E7FFF728FEF2E7FFF7D7FA0020D4
:1079E000FFF73EFF7448FFF73BFDE9E7632CE7D85C
:1079F000724BA200D25821001520FFF709FBDFE7E8
:107A0000FFF79EF9FF270400002CD9D025682B141E
:107A10003B40152B04D02000FEF76CFA0400F3E77E
:107A20002000083007F0C6FA06000530FFF774F9A9
:107A3000FB20FFF70BF92D121D20FFF707F9E8B225
:107A4000FFF704F9F0B2FFF701F93012C0B2FFF707
:107A5000FDF825002B1B9E42DDDD287AFFF7F6F8A6
:107A60000135F7E700211D2000910B000A00FEF709
:107A7000B9FCFCF75FFFA3E72000FFF749FC9FE795
:107A8000FFF762FC9CE7FCF731FD07AC4C4A642130
:107A900000904C4B200007F015FA022320002370C1
:107AA00007F088FA2300020000211620FFF73AFAB7
:107AB00086E7454BFA21186804F08AFC00260490FA
:107AC0003C4AF3009B181C68002C28D01B790593B6
:107AD000636808349F00B81D0393FFF71DF9FB206E
:107AE000FFF7B4F801207D1CFFF7B0F8F0B2FFF704
:107AF000ADF8E8B22D12FFF7A9F8E8B2FFF7A6F843
:107B00000598FFF7A3F8E719A7420CD8FFF7EAF8A2
:107B1000049B0398584301F067FEFFF7E3F8013632
:107B2000FF2ECDD14CE72078FFF790F80134EBE73A
:107B30000024FFF72BFA2300220021000094DA2012
:107B4000FEF750FCFF222100D2001A4806F0A8FEE2
:107B5000FCF7F0FE21002000FDF7CAFD30E7012C04
:107B600002D1FEF7F1F92BE7022C02D1FEF736FC29
:107B700026E7032C03D100210800FDF7B9FD012001
:107B8000FFF76EFE1CE7002321001A001A208DE784
:107B90001A00C83A052A00D912E70022180011007D
:107BA000F9F7BEFE0CE7C046A81A0020A816002070
:107BB0009812002074250020A41401006C2D0020D0
:107BC000BB140100B614010004000020FB2B00D000
:107BD000B3E62268042A00DCABE63E79F878614B14
:107BE000360206439E4200DDA7E6331D9A4200DCC2
:107BF0009FE6FB5CFE2B00D09FE67878BC78751E74
:107C00001B2869D01AD807284FD0082824D001286B
:107C100019D1FF2C10D02000FFF7FAFA7D79524AD3
:107C2000B31E009221002A000A20FEF7DBFB4F4B17
:107C3000E400E0501B191D71701D7FE61D285DD00A
:107C40004FD31E2871D00300C83B052BF4D8484AF7
:107C50002900F9F765FEEFE7632CEDD87A79022A5F
:107C600013D0032A1BD0012AE6D1F979BB79090286
:107C700019433B7AA4001B0419437B7A1B060B4370
:107C80005B0013433B4AA350D6E7002DD4DDB11E61
:107C90003548FDF7C1F8374BA400E050CCE7BB797D
:107CA000A4005A1E93419B00ECE7632DC4DC07AF90
:107CB0002A002F49380006F0D7FD002338007B55F5
:107CC000FFF794FB0028B7DB2A4B8000C258210045
:107CD0001520FFF79DF9AFE729002548FFF7BEFC07
:107CE000AAE7FF2CA8D07A79022AA5D81E490B2032
:107CF00000912100B31EFEF775FB9DE7632D00DDAB
:107D00006325002307A99D420ADCEB430022DB1711
:107D10002B40CB181A70152000916B1C2100EAE74C
:107D2000FA185279CA540133EDE7022C13D0032C10
:107D300014D0012C00D07FE7002D00DC7CE77B799C
:107D4000002B03D01C00322B00DD322464235C4363
:107D5000094B1C6070E7FEF7A7FB6DE7FEF7A5FB7C
:107D60006AE7C046F6030000AE1600207425002026
:107D7000AD1600206C2D002004000020012070476B
:107D800010B5064C200001F09BF90549200001F0D8
:107D9000CBF90122034B1A6010BDC046E41A002043
:107DA000801A0600AC1A00201FB500211020FCF735
:107DB000A3FB01211620FCF79FFB01211120FCF7FA
:107DC0009BFB1E4C200001F0D9F81D4B1D491A6881
:107DD00009681D4B1D481B78C9B282420DD880220C
:107DE0009204019201AA1171013B581E834101992D
:107DF000029A200001F0DEF81FBD1548824202D829
:107E00008022D204EDE71348824202D88022120574
:107E1000E7E71148824202D880225205E1E70F4885
:107E2000824202D880229205DBE70D48824202D8C6
:107E30008022D205D5E780221206D2E7C41A00209C
:107E400044000020400000203C00002048E80100E1
:107E500090D0030020A1070040420F0080841E0044
:107E600000093D0070B5002812DD0C68E3070FD54E
:107E70006410012C0CDD074D2B68002B01D1FFF79E
:107E80007FFF2B68002B03D02100034801F04CF941
:107E9000002070BDAC1A0020E41A002070B5002844
:107EA0002CDD01240B68234228D02341174A13609C
:107EB000174AA04209D04B68234206D02341022B27
:107EC00020D0032B20D0A3421AD002231360012418
:107ED000104D2C70032811DDC86804400ED1042811
:107EE0000CD90F2302681340042B07D1FCF774FD53
:107EF000094907F055F8002800D02C70002070BD0B
:107F00000023E3E70323E1E71460E0E744000020F7
:107F1000400000203C000020E6140100F8B50125D7
:107F20000868284203D10D20F9F7ACFEF8BD4010D7
:107F3000FCF706FB041E14DBFCF7DCFAA04210DBA6
:107F400002212000FCF7D8FAFA222900D2002000F2
:107F500001F07CFC0025A84205D101002000FCF7BF
:107F6000CBFA0020E2E700270726FA22012192003F
:107F7000200001F06BFC0028F3D0282802DD01234B
:107F8000B3401F43013EF0D20E4EAF550135052DD3
:107F9000E9D100212000FCF7AFFA012206210920D7
:107FA000FCF7BCFE0028DCD00B2301244360002337
:107FB000F25C990052004118224301338A60052B7C
:107FC000F6D1B3E7B01A002070B500281EDD0D68A9
:107FD000EB071BD4042D19D90F242B681C40032C4C
:107FE00014D11A0992B25B0F92001C40141B2E0090
:107FF000FFF7DAFE731B06489C4205DD317900F07D
:10800000DFFF0136F070F5E700F0D9FF002070BD0A
:10801000C41A002010B504680D20E30703D56410CE
:10802000FF2C03D91720F9F72DFE10BDFFF7BCFE7A
:10803000E1B2044C200000F0C3FF200000F0BFFFBD
:108040000020F2E7C41A002070B5FFF7ADFE064D20
:108050000021280000F0B4FF0400280000F0AFFF6A
:1080600001206400204370BDC41A0020A021012219
:108070000B4BC9005A500B480B4958500B491A601A
:108080004A68002AFCD000224A60A121C900585841
:1080900001215960A021C9005A50054BC0187047F2
:1080A000007000406A10000004050000FC700040F1
:1080B000FBFDFFFF10B5FFF7D9FF43000120184378
:1080C00010BD000010B5034A0F210348FEF74AFE19
:1080D00010BDC046EC14010064150100F8B50E4F48
:1080E00004003B680E001500002B01D1FFF748FE8D
:1080F0003B68002B0FD0E1B2084C200001F0ABF838
:10810000F1B2200000F0A8FFE9B2200000F0A4FFC7
:10811000200001F00BF9F8BDAC1A0020E41A002091
:1081200010B501240368234205D04168214202D0E2
:108130008268224203D10D20F9F7A4FD10BD58102A
:10814000802801D91520F7E74910FF2901D9162009
:10815000F2E75210FF2A01D91720EDE7FFF7BEFF23
:108160000020EBE710B5002803DC1C20F9F78AFD9E
:1081700010BD0B68DA0701D40D20F7E75B1003226E
:10818000012B06DD0522022B03D00C22042B00DC80
:1081900008220F211820FFF7A1FF0220F9F780FD28
:1081A0000020E5E70123F0B5020085B018009A42EF
:1081B0001ADD0D682B4217D01D414C680193022A2D
:1081C00005D08B68043B5A425341DBB20193394ED0
:1081D0003368002B01D1FFF7D3FD3368002B05D1A5
:1081E0002320F9F74FFD002005B0F0BD324EE9B273
:1081F000300001F030F827000122174010D0144160
:10820000FF2C02D91720F9F73DFDE1B2300000F054
:1082100023FF0199300001F029F80028E4D0DFE7BE
:10822000042CF6D90F2523681D40092D1CD1636845
:1082300003925B100293029BBB42EADDBB00E31892
:108240009D68039B1D420BD06D10FF2D02D9172096
:10825000F9F718FDE9B2300000F0FEFE0137EAE759
:108260001720F9F70FFDF9E7032D0FD127001A09A1
:1082700092B25B0F92001D40551B3B1B9D42C8DD17
:108280003979300000F0E8FE0137F6E7042DC0D15F
:108290002000FCF7A1FB0500200006F08BFE2C005F
:1082A0000700631B9F42B4DD2178300000F0D4FE4C
:1082B0000134F6E7AC1A0020E41A002070B5174C20
:1082C000050023680E00002B01D1FFF759FD23683C
:1082D000002B21D0124CEDB22900200000F0BBFF92
:1082E000F1B2200000F0B8FE0021200000F0BEFF37
:1082F000002801D040420EE072B601222900200081
:1083000000F0A4FF62B6200000F097FE002802D023
:10831000200000F097FE70BD6420EBE7AC1A00204F
:10832000E41A002010B501240368234202D04168FA
:10833000214203D10D20F9F7A5FC10BD581080286B
:1083400001D91520F7E74910FF2901D91620F2E7D6
:10835000FFF7B4FF40002043EFE7000070B5284D61
:1083600004002B68002B08D105211820FFF7A6FF79
:10837000022001F039FA01232B60012C14D10521D0
:108380001820FFF79BFF7F282BDC03007F3301DAE7
:108390007F204042C8235B4258437F2104F018F8F5
:1083A000052C00D1404270BD032C11D121001820B2
:1083B000FFF784FF7F2814DC03007F3301DA7F207E
:1083C0004042C8235B4258437F2104F001F8EAE7AA
:1083D0000020052CF5D107211830FFF76FFF7F280B
:1083E00002DD0138FF38D0E703007F3301DA7F2058
:1083F0004042C8235B4258437F2103F0E9FFD1E7A5
:10840000B81A002010B50120FFF7A8FF4300012093
:10841000184310BD10B50320FFF7A0FF4300012053
:10842000184310BD10B50520FFF798FF4300012049
:10843000184310BD10B508211820FFF73FFF0300B7
:10844000C00FC0180123401015304000184310BD64
:10845000F8B5514B05001B68002B01D1FFF790FCCC
:108460004E4C23787F2B00D892E007210E20FFF797
:1084700025FFC42833D101220E26494B10211A7042
:10848000484B30001A702670FFF728FE8022112119
:108490003000FFF723FE0021615600291EDB424E0B
:1084A000C9B2300000F0D7FE3D4B3000197800F023
:1084B000D3FD300000F03AFF21780622300000F0B2
:1084C000C5FEAC1D300000F0B8FD002806D030001D
:1084D00000F0B8FD28700135A542F3D1F8BD0F2199
:1084E0001920FFF7EBFE33280FD168222C4B1E26F4
:1084F0001A7000222B4B60211A7030000C3226704B
:10850000FFF7ECFD02226121C2E700211820FFF7EE
:10851000D5FEFA281CD14222214B10261A700022C7
:10852000204B4B211A70300001322670FFF7D6FD28
:10853000042001F059F938224C213000FFF7CEFD1C
:108540000F2251213000FFF7C9FD1B2252219FE766
:108550000F211C20FFF7B2FE3D289CD128221C26AB
:1085600000270F4B20211A700E4B263A30001F7047
:108570002670FFF7B3FD3A0022213000FFF7AEFD71
:108580003A0023213000FFF7A9FD402224217FE794
:108590000021615683E7C046AC1A00204800002045
:1085A0004A00002049000020E41A002073B500268C
:1085B00006220021684606F073F96846FFF748FF77
:1085C000FFF79AF91A4B6A469E576C466B469178AC
:1085D0001878D5785B7812796479002E1FD0000264
:1085E0000902034329431BB209B212021148224374
:1085F000007812B240B2102802D15210DB10C9101C
:10860000D8171B184340C8170918414001205918B2
:10861000D317D2185A408A185200104376BD1B0255
:108620002D02034329431BB209B22402DEE7C046F0
:108630004900002048000020F7B5012801DC012096
:10864000FEBD01250B6801932B42F8D04E683540E2
:10865000F5D1042EF3D90F2332681340092BEED144
:1086600073685C10002CEADD174F3B68002B01D1CA
:10867000FFF786FB3B68002BE1D0202C00DD202497
:1086800072B6019B114F5910C9B22200380000F098
:10869000DDFD62B6380000F0D0FC002803D16D008B
:1086A00001302843CCE7380000F0CCFC0122AB00BD
:1086B0004000F3181043AD189860A542EADB9440DF
:1086C00010002043BCE7C046AC1A0020E41A00208A
:1086D00070B52B4B86B01B68002B02D10120FFF731
:1086E0003DFE01AD14220021280006F0D9F8254EE8
:1086F0001821300000F0AFFD0321300000F0ACFC89
:108700000021300000F0B2FD041E13D172B6052224
:108710001821300000F09AFD62B6300000F08DFCA8
:10872000002802D0300000F08DFCA3000134E85096
:10873000052CF2D1019B7F2B01DD013BFF3BAA6899
:108740007F2A01DD013AFF3A29697F2901DD0139DC
:10875000FF39C820434342434843DB11D2115243FF
:10876000C0115B4340439B18181805F081FE01F0CF
:1087700081FD05F047FE43000120184306B070BD9F
:10878000B81A0020E41A00200020704710B5054CEC
:108790002368002B02D01B20F9F774FA0020206018
:1087A00010BDC046BC1A002010B5002803DC1C20F8
:1087B000F9F768FA10BD0B68DA0706D4042B04D960
:1087C0000F221B681340032B01D02420F0E7034B3A
:1087D00025201B68002BEBD01B20E9E7BC1A0020EA
:1087E00010B5002803DC1C20F9F74CFA10BD0B680B
:1087F000DB0701D40D20F7E71B20F9F743FA00202F
:10880000F4E710B50400002C0ADD1B20F9F73AFA52
:10881000FEF764FFFFF770F8012000F0E5FFF2E7D4
:1088200010BD00002D4BF7B51B68002B03D1252090
:10883000F9F728FAFEBD012801DC1C20F8E748689A
:1088400047103B00013B019301D51220F0E70E6871
:10885000F30709D4042E07D90F2332681340D91E19
:10886000012903D9092B01D02420E1E7012420426A
:1088700001D11120DCE7092B1AD173685D10019B2F
:10888000AB42E2DABD420DDB0137BB00F3582342B5
:10889000F8D05B10FF2B01DD2820C9E72000FFF78F
:1088A000B0FFEFE7019BE81A013040002043C1E729
:1088B000042B0CD13000FCF78FF806F07BFB019BFA
:1088C0008342C2DA1B20F9F7DDF90120B2E7100973
:1088D00080B252008000920F801AF0E7BC1A00208C
:1088E00000207047044B10B51B682520002B00D0DA
:1088F0001B20F9F7C7F910BDBC1A0020F8B50028F5
:1089000003DC1C20F9F7BEF9F8BD224B25201B68BB
:10891000002BF7D00D6801202C00044004D0054145
:10892000FF2D1EDD2730EDE7042D0ED90F212A681B
:10893000114004290BD12800FCF74EF806F03AFB51
:1089400080280ED92620F9F79DF90020DCE70329BD
:108950000AD1100980B2520F80000A40801A802884
:10896000F0DCFFF74EFFF0E70929EED10400070025
:108970006B685E10A642E8DB0134A300EB583B4273
:10898000F8D05B10FF2B01DD2820BBE73800FFF794
:1089900038FFEFE7BC1A002010B5034A082103484E
:1089A000FEF7E0F910BDC046101601005016010098
:1089B000002070470120704700207047002070475A
:1089C000012070470020704700207047002070474A
:1089D000002070470020704700207047002070473B
:1089E000002070470020704700207047002070472B
:1089F00000207047002070477047704770477047ED
:108A000010B5034A12210348FEF7ACF910BDC04669
:108A100080160100101701000378013B1F2B00D9BD
:108A200070470130F8E710B5FFF7F6FF0378002B29
:108A30000BD00130222B11D10378002B03D0421C24
:108A4000222B03D11000FFF7E7FF10BD5C2B03D1F1
:108A50004378002B00D0821C1000EDE73A2BF2D0B7
:108A60002C2BF0D07B2B0BD1FFF7D6FF0378002BFC
:108A7000E9D07D2B01D10130E5E7FFF7D4FFF5E721
:108A800020225B2B14D1FFF7C7FF0378002BDAD02D
:108A90005D2BF0D0FFF7C7FFF7E7202BD3DD2C2BA2
:108AA000D3D0190091435D29CFD0222BCDD00130F6
:108AB0000378002BF1D1C6E7002210B5904216D002
:108AC000FFF7AAFF03780422222B10D0023A7B2B57
:108AD0000DD0013A5B2B0AD0190030390232092936
:108AE00005D92D2B05D14178303909290AD8100034
:108AF00010BD0522742BFAD00132662BF7D001325B
:108B00006E2BF4D0581E83415A42F0E770B5FFF740
:108B100083FF037801222D2B01D18018023A002314
:108B20000A2502E06B430130CB1801783039CCB212
:108B3000092CF7D95A43100070BDF8B50C00150088
:108B4000FFF76AFF0378222B02D000232370F8BDC1
:108B50000D236A1E210008250C260A279C46013099
:108B60000378222B02D100230B70F0E7002BFAD000
:108B7000441C5C2B0BD14378841C622B0ED0662BDB
:108B80000ED06E2B0ED0722B0ED0742B0ED0002A6E
:108B9000E9DD0B70013A01312000E1E72B00F6E737
:108BA0003300F4E73B00F2E76346F0E70923EEE722
:108BB00010B50400FFF737FFA04203D90378013B4B
:108BC0001F2B00D910BD0138F6E710B5002815D0CD
:108BD0000378002B13D0FFF71FFF2021037802003A
:108BE0008B4300205D2B09D01000FFF71CFF03789A
:108BF0002C3B5A425341C018FFF70EFF10BD18001E
:108C0000FCE70300002070B50C0081420EDD1A78ED
:108C10005B2A0BD1581CFFF7FFFE0125AC4205D0A3
:108C2000FFF7D3FF002801D00135F7E770BD70B51D
:108C30000C001500002901D000230B70002820D063
:108C40000378002B1ED0FFF7E7FE037806002C2BDD
:108C500003D10130FFF7E0FE0600337800207D2BC2
:108C60000FD0844204D02A0021003000FFF765FFB6
:108C70003000FFF7D8FE03783A2B02D10130FFF71E
:108C8000CBFE70BD1800FCE7F0B50D0004009DB0F0
:108C90002E78002E35D02E21280006F073F9071EFD
:108CA00014D0431B0193303E092E14D82800FFF73F
:108CB0002DFF01002000FFF7A4FF0400002C20D0AE
:108CC000002F1ED0019B0133ED18E1E7280006F0CC
:108CD00071F90190E7E723787B2B11D1601C6422A6
:108CE00003A9FFF7A4FF041E0BD0019A290003A8D3
:108CF00006F067F90028E1D02000FFF794FEEEE7C8
:108D0000002420001DB0F0BD70B5050000200C004F
:108D100081421DDD2800FFF7CFFE0300681C012BF8
:108D200014D00020022B13D10022681C1100FFF781
:108D30007EFF012C0CD0FFF748FF00221100FFF747
:108D400076FF013CF5E7FFF740FF013C012CFAD12B
:108D500070BDF8B5050000200C0016001F00814210
:108D60000DDD2800FFF7A8FE03000020022B06D12E
:108D7000681C3A003100FFF75AFF012C00D1F8BD02
:108D8000FFF723FF3A003100FFF751FF013CF4E702
:108D900010B50024A04218D0FFF73EFE03787B2BCD
:108DA0000AD1013000221100FFF741FF00280CD04A
:108DB000FFF739FE0134F5E75B2B06D10130FFF7F1
:108DC00004FF002801D00134F9E7200010BDF8B5F8
:108DD000002816DD0D68EB0713D56D10013D012449
:108DE000FDF794F90026FF27644200280CD1002EDD
:108DF00021D0300006F0DEF801003000FCF70CF85E
:108E0000F8BD01256D42EAE703681A143A40152AB5
:108E10000BD11B123B409C4200DA1C009D4201D149
:108E200006000836FDF766F8DFE71D2AFAD10124AF
:108E300000266442F6E70120013464002043DFE7A6
:108E400010B508680C00FBF7C7FDFEF7CFFA002845
:108E500003DB6268024B8000C250002010BDC04698
:108E60006C2D002010B50868FBF7B6FDFEF7BEFAC2
:108E70000123002802DB024B8000C358180010BDFC
:108E80006C2D002010B50868FBF7A6FDFEF7AEFAC2
:108E9000C043C00F800010BD10B5034A0421034831
:108EA000FDF760FF10BDC046D0170100CA170100D2
:108EB00010B5FBF7B1FCFBF761FDFDF7BFFF044800
:108EC000FEF7CEFAFDF780F9FEF7AEFB10BDC04607
:108ED0001F18010010B5FAF7D5FF10BD70B50025B9
:108EE00004AC24780573A94205D10A4B0A4A25210E
:108EF0000A4805F04BFC01600949920052589B005A
:108F000002715B58A400837163588560437102232A
:108F1000C37170BD37180100961801004518010093
:108F2000F4180100037B002B04D1437383730361A6
:108F300001330373704700001FB50191A021002485
:108F40000068C900D2B24450012A10D0A24209D010
:108F5000032A0AD0074A8350074B019AC2500123C3
:108F600043501FBD02221343F4E70422FBE706220D
:108F7000F9E7C046540500002405000010B50400C0
:108F8000FFF7D0FFA1222368A179D200995061791F
:108F9000064A20009950217904329950044B1968EF
:108FA0005A689B68FFF7C8FF10BDC0460C0500005B
:108FB000D81A00201FB5FFF7BFFF05B000BD7047EE
:108FC0000368074A99501A00FC32D1680029FCD086
:108FD000A321C90058580023C0B2D3607047C046CF
:108FE0001C05000007B58022074BD2051A6000223D
:108FF0009A6002321A7111230E320093034905332D
:109000000348FFF76BFF07BDD81A0020003000406F
:10901000C41A0020F8B505000E0017000024BC4259
:1090200008D02B68315D1B6828009847002801D0C4
:109030000134F4E72000F8BD704710B51C3000F093
:10904000AFF910BD10B51C3000F09CF910BD10B583
:109050001C3000F0ABF910BD70B5437E0D00002B45
:1090600001D1002070BD6430040000F0A8F9002890
:10907000F7D12000290000F076F90120F2E7000086
:10908000F7B50193FA23002504009B0083600B4B86
:109090004560083303601C300F00160000F058F9DB
:1090A0002000643000F054F96B461B792761667527
:1090B0006576A5762000A375FEBDC046D4180100D4
:1090C000012330B5A024C375837D13499B005A58F2
:1090D000437DC132114DFF32E40592009B005B5885
:1090E0001551CC22C133FF339B001D5104690C4B39
:1090F0005204E25005220469243BE250837D046956
:109100009B005A58A123DB00E250437D02699B007B
:109110005958044BD15030BDF41801000C06000022
:10912000240500000C050000A022002310B50469EE
:10913000D200A3500A4CA1420FD90A4C8C425B4189
:1091400009495B420B40CD21C9045B1804690749FA
:10915000635005210369995010BDCC235B04F5E7EA
:10916000A086010090D00300000098FD24050000B7
:10917000F7B5040000200D000193824265D016006F
:10918000402A00D9402627001C37380000F0F6F8A6
:10919000B1232269DB00D55080220123216992008E
:1091A0008B50A27E002A03D12269136222691360C8
:1091B0000025731EAB4207D1019B002B04D08022F7
:1091C0000221236992009950012223691A622369BE
:1091D000FC33DA68002A02D19A6A002AF9D09A6A26
:1091E000002A0BD1DA60A3232269DB00D1583800B2
:1091F000C9B2013500F0B7F8B542DAD3019B226954
:10920000002B0FD11300FC339B6A002B0AD10133D2
:10921000A376D3612369FC33DA6C002AFCD00022E8
:10922000DA640AE000230121A37651611A00236960
:10923000FC3399680029FCD09A602369FC339A6A50
:10924000002A01D000229A62E8B2FEBD10B50123C7
:10925000FFF78EFF10BD0300AC3310B5040019708A
:10926000643000F08BF80123637610BD0023020008
:1092700070B5AC3243760D001178B122040000695C
:10928000D20081508022216992008B5022690133E3
:1092900013622269936026006436300000F080F883
:1092A000002812D0300000F06DF81E4B2269D0501B
:1092B0002369FC331A6A002A02D19A6A002AF9D07B
:1092C0009A6A002A01D11A62E5E723690122002D7A
:1092D0000DD11900FC31896A002908D1DA612369AE
:1092E000FC33DA6C002AFCD00022DA6407E05A6111
:1092F0002369FC339A68002AFCD000229A6000207F
:109300002369FC339A6A82420BD098622169064A2B
:109310008B588B501800022B03D0181F431E984106
:10932000033070BD1C050000C404000010B501210D
:10933000FFF79CFF10BD000010B513231222024955
:109340000248FFF79DFE10BD00400040E41A0020D7
:1093500010B540220021040005F0A2FA00232000ED
:109360002364636410BD10B53F24026C531C23407A
:10937000446C9C4201D08154036410BD00230364FB
:1093800043647047436C026C934206D03F21C25C39
:1093900001330B4043641000704701204042FBE75B
:1093A000036C406C181A00D540307047436C026C57
:1093B000934201D0C05C704701204042FBE73F224E
:1093C000036C406C01331340181A43425841C0B239
:1093D0007047000003210A4802680A4302600948F6
:1093E00002680A4302600849084A094B9B1A03DDD8
:1093F000043BC858D050FBDC00F012F8F6F784FEAE
:109400002405004054050040401E010000000020DB
:1094100084020020FEE7FEE7FEE7FEE7FEE7FEE748
:10942000014B024A1A6070474C0000200024F400EF
:109430000120704710B503681322DB69984710BDFF
:1094400070470000054B0269D1500369FC331A6A6A
:10945000002AFCD0002201201A6270471C0500007F
:10946000030010B55C331A781F231A401E3B190005
:109470009140114AD167C222042104699200A1508F
:10948000026953600269D360A02300220169DB00F6
:10949000CA5001230169094A5B428B500169084A9D
:1094A0008B5001690C3A8B50016908328B50143093
:1094B000FFF764FF10BDC04604E100E00C050000AA
:1094C0001405000010B51430FFF76AFF10BD10B589
:1094D0001430FFF76BFF10BD10B51430FFF752FFCB
:1094E00010BD0000030070B55E331A780469724B3A
:1094F000E25003005D331A780469704BE2500300B8
:1095000061331C7802696E4B012C00D09EE005008F
:109510005F352E78A225ED00565102006032157895
:10952000A1220669D200B5500269D4509623DB000F
:10953000994200D88CE096231B01994200D88AE01A
:1095400096235B01994200D888E096239B019942BB
:1095500000D885E0E1239B01994200D882E0962360
:10956000DB01994200D880E0E123DB01994200D879
:109570007DE096231B02994200D87AE0E1231B028A
:10958000994200D877E096235B02994200D874E0B4
:10959000E1235B02994200D871E0E1239B029942EA
:1095A00000D86EE0474B994200D86CE0E123DB0223
:1095B000994200D86AE0E122002312038A425B410B
:1095C000414A5B421340802252059B1801693F4A81
:1095D0008B50A02304220169DB00CA5000210369DB
:1095E000FC33D9600369FC331962012301690B6004
:1095F00001698B60C1210469890062501F215C30C0
:1096000002780A4093406231314AFF3153500021C1
:10961000415600293CDA0F230B40083B2D4C9B0898
:109620009B001B1903242140A140FC348C40DD69C0
:10963000A5432C00C0258D4029002143D9611F235B
:10964000017819401E3B8B40136070BD00246CE70D
:109650009E23DB02BAE79D231B03B7E71E4BB5E74A
:109660001E4BB3E7EC239B03B0E71D4BAEE71D4B4E
:10967000ACE71D4BAAE71D4BA8E71D4BA6E71D4B0A
:10968000A4E71D4BA2E78023DB049FE71B4B9DE76C
:109690008C080F4BA400E41803230B40FF21C025C6
:1096A000DB009940AD0066598E433100C0269E40D4
:1096B00033000B436351C2E70C05000014050000A2
:1096C0006C05000090D0030000D0BEFE2405000011
:1096D00000E100E000ED00E000B0130000502700C2
:1096E00000A04E0000F0750000509D0000F0EB005F
:1096F00000903A0100E0D70100B0AF0300705F07AF
:10970000F7B5009308AB1B7800250193FA230400FA
:109710009B0083600E4B45600833036014300F00DC
:109720001600FFF715FE23005C3327611E70009BB7
:10973000084A9B00995823005D331970019B200053
:109740009B009A5823005E33DD701A70FEBDC04640
:1097500070190100F4180100036910B51A00FC32F9
:10976000D2680400002A0AD0A322D20099581430EB
:10977000C9B2FFF7F8FD00222369FC33DA6010BD9F
:1097800010B50248FFF7E8FF10BDC0469C1B002043
:109790001D2307B502220093024901330248FFF757
:1097A000AFFF07BD002000409C1B002010B5002823
:1097B00001D005F031FB10BD0849094A094B10B52D
:1097C0001B688858FA22190A1B06184392000023C6
:1097D00002F05AFF4904C00B084310BD00100140BD
:1097E00004050000001C002070B5041E09D0FFF71E
:1097F000E3FF050000F014F8FFF7DEFF401BA04276
:10980000F8D370BD0022044B9A60044A13680133F8
:10981000DBB213607047C046FC100140001C002002
:109820007047704710B500F05FF8FFF7FAFF0120AE
:10983000FFF7DAFFFFF73CFBFFF74CFB024B002B77
:10984000FAD000E000BFF7E700000000F8B54C1EBA
:10985000A1410125104B114F8000C3584C4238687C
:109860000F499D40160002F029FD0A21704302F0C5
:1098700025FD2C400300220029000A4800F016F8BC
:10988000FA21094C89004443386802F017FD0100B1
:10989000200002F013FDF8BDF41801004C00002078
:1098A00040420F00100500501027000030B504683A
:1098B0000C40944206D1013B002BF8D112E0013B51
:1098C000002B0FD004680C409442F8D100240568A6
:1098D0000D40954204D101349C42F8D1002002E0B1
:1098E000201C00E0181C30BDC420114B80001A5809
:1098F00010491140C02212020A431A50C02180228E
:10990000490092025A501A608023A3220021DB05ED
:10991000D20099500122F9309A60074BFF3019505C
:10992000C120023180001950403019501A60704730
:1099300000E100E0FF00FFFF00100140014B186054
:109940007047C04698000020F7B500231E285AD85B
:10995000384B8000C258042A5BD007D8022A54D062
:1099600055D80423012A09D000234CE0062A54D0FC
:1099700051D31A2A53D002231B2AF5D12E4A11683B
:1099800008294ED909294FD00A240226A0200125F2
:109990002A4AC00015502A482A4D07681C20BF00DB
:1099A00007402948019700685759009027481B0233
:1099B00007401F43C02300989B020340FF205751DC
:1099C0005759000207401F43019B1F43009B58014A
:1099D0006023184007433E43565101251C4B156038
:1099E00058680028FCD000205860A1230125DB0026
:1099F000D3585560A025ED0050511BB2A14202D0B2
:109A000015D2611ACB401800FEBD0823B6E710231B
:109A1000B4E72023B2E74023B0E78023AEE7012379
:109A2000ACE708240026B1E70C000126AEE7091BCD
:109A30008B40E8E7F418010094000020007000401B
:109A4000500000200405000054000020FF00FFFF2C
:109A5000FC700040F0B51E285BD8364B8000C25821
:109A6000354B1E68002E30D1C227344BBF00D85969
:109A7000334C03250440C02000022043D851C024A9
:109A800080206400800018512E4F18602E4B803CBF
:109A9000D859FF3CA043D8510437D859A843204394
:109AA000D8510837D8590C35A84384460720654655
:109AB0002843D851A820C0001E50C1208026800015
:109AC00076021E501C601C4B1C60142500202B00CD
:109AD0001E4C2E0046433659771C1BD14343E2509F
:109AE000A0230325C132FF329200DB05D550184B6D
:109AF0001A68082A14D114234343E3189A681248B9
:109B00005132FF32920059601150DA68C1239B0034
:109B1000C250F0BD9642E1D001300328D9D1F8E718
:109B2000082A02D9083AD140E5E708239A1A914059
:109B3000E1E7C046F4180100041C002000E100E049
:109B4000FF00FFFF040500000090004058000020C7
:109B5000980000202149F0B54A6C2148002A14D011
:109B6000A025A12600230124ED05F600C258571CAC
:109B700006D0C7187F68002F02D027009740AF514A
:109B800014333C2BF2D100234B64A0230121DB05CD
:109B900000260F009C4614234B43C3181A1F12685B
:109BA000104C0E4D920014195219526C002A10D00C
:109BB0001A00143A1268551C09D0103B1B68FF2B81
:109BC00005D03B00934065461A00074BEA50FC3431
:109BD000666401310429DED1F0BDC046FC9000402E
:109BE00058000020009000400C05000000B51E2821
:109BF00010D80C4A8000835803290BD8A0220800F3
:109C0000C133FF33D2059B0002F03AFB020905077E
:109C10000021D15000BD0C21FBE70421F9E703210D
:109C2000F7E7C046F41801001E280AD8074B800049
:109C3000C25801239340A022D205002902D1044931
:109C400053507047A121C900FAE7C046F41801003B
:109C50000C050000030000201E2B0AD8A021A22220
:109C6000C905D2008858034A9B009B58D84001235D
:109C700018407047F4180100F7B506000D000C00FD
:109C80008B180193019B671B9C4207D03368217896
:109C90001B683000984701340028F3D13800FEBD1E
:109CA000F0B5C64600B5CB0F9846404A4B005B0D59
:109CB0009A1882B00D000400132A2FDC002A49DB19
:109CC0003B4F17413E000E40064323D07F0839002A
:109CD00029400C430AD03749BD438C4663445C425B
:109CE0005C418023DB021341E4071D434146CE0063
:109CF00031492B008E192200346875682000290034
:109D000002F084FE009001910098019922002B003E
:109D100004F014F802B004BC9046F0BD332A08DD0C
:109D20008023DB009A42F5D102000B0002F06EFEA8
:109D3000F0E7224A9446012263445242DA4002424A
:109D4000E8D052080242D1D094438022D2051A4171
:109D50001443CBE74B005B080343DBD00B031B0B27
:109D60001C436342234380244D0C24031B0B2340DC
:109D70006D042B4319004346DA000F4B9B181C68F7
:109D80005D6802000B002000290002F03FFE0090F9
:109D900001910098019922002B0003F0CFFF424669
:109DA0004B005B08D60733431900B3E701FCFFFF04
:109DB000FFFF0F00EEFBFFFFA0190100EDFBFFFF0F
:109DC000F8B5274A4B005B0D9A180C000700132AC0
:109DD00010DC002A36DB234B13410B423AD080249F
:109DE00024031441002064189C4306002500300021
:109DF0002900F8BD332A0EDD80230600DB000D00AC
:109E00009A42F4D102000B003800210002F0FEFD5E
:109E100006000D00EBE7144D0600AC460125634437
:109E20006D42DD40AC4663460D000342DFD0332374
:109E30009A1A323B93401818874200D94C1C63464B
:109E40009843D2E7C90FCC070020531CCDD1074B54
:109E50001C43CAE706000D000028C0D1C7E7C04672
:109E600001FCFFFFFFFF0F00EDFBFFFF0000F03FD5
:109E700030B5214A4B0087B05B0893421EDD1F4A74
:109E8000934205DD02000B0003F058FF07B030BD20
:109E900002AA00F0B5FF03231840049A059B01288D
:109EA00013D002281DD0002814D00298039901F085
:109EB0008FFA80231B069C466144E7E700230022BB
:109EC0000093002301F0FEFFE0E70298039901F000
:109ED0007FFADBE7012402980399009401F0F2FF76
:109EE000D4E7012402980399009401F0EBFF80234A
:109EF0001B069C466144C9E7FB21E93FFFFFEF7F5A
:109F0000F0B557464E46DE464546E0B58FB01D00DB
:109F100006000F00140000F00DFACE4B00900191E6
:109F20009A461B785BB2994601333ED022002B0043
:109F30002000290004F04AFA8346002835D1320077
:109F40003B003000390004F041FA00220390002861
:109F500000D06FE000233000390002F043FB0028FE
:109F60002CD0002200232000290002F03BFB834676
:109F7000002800D192E004AB9846012342460493A6
:109F8000B54B53604346039A1C615D611A629E6043
:109F9000DF604246002300249361D4614B46002BCE
:109FA00067D00023AD4C00930194009801990FB045
:109FB0003CBC90469946A246AB46F0BD009801993C
:109FC00002F036F88146002800D19AE00098019905
:109FD0000022002302F006FB0028E6D03000390002
:109FE00002F026F80028E0D02000290002F020F836
:109FF0000028DAD004AB9846042342460493964BDB
:10A00000146155615360002300241362002393619F
:10A01000D46153461B789660D7605BB2022B04D0A4
:10A02000404602F0ABF8002829D104F0CDFB2223F2
:10A03000036024E000232000290002F0D3FA002866
:10A04000B3D004AB9846012342460493824B414669
:10A05000536043465A461A6200229E60DF601C61CC
:10A060005D617E4B8A61CB61009201934B46022B6E
:10A070009BD0404602F082F8002800D18AE0434697
:10A080001B6A002B04D004F09FFB43461B6A03604D
:10A090004346DC699B690093019486E72000290010
:10A0A00001F0C6FF002800D17FE700220023200036
:10A0B000290002F09DFA002800D176E704AB98460B
:10A0C000012342460493644B536043465A469E60C4
:10A0D000DF601A621C615D6153461B785BB2002B26
:10A0E0005DD0002042465E499061D161022B5BD178
:10A0F00004F06AFB2123036043461B6A002BC7D090
:10A10000C1E73000390001F093FF002800D15DE77E
:10A110002000290001F08CFF002800D156E70098AC
:10A12000019953461B7802005BB29B460B0004F07A
:10A130004DF904AB9846002862D1032342460493AC
:10A14000454B14615561536010629660D760454B72
:10A1500020002900002203F07FFB5B4604000D0075
:10A16000002B27D1E02241463F4B12068A61CB618A
:10A17000300000220023390002F03AFA00282AD1E8
:10A18000404601F0FBFF0028B6D104F01DFB22235E
:10A190000360B1E704F018FB212303606FE7424638
:10A1A000002300249361D461404601F0E7FF0028BA
:10A1B000A2D19DE7002241462C4B30008A61CB6141
:10A1C00000220023390002F013FA002835D15B4643
:10A1D000022BDAD0D4E720002900FFF761FD22002E
:10A1E0002B0002F0FFF9002805D1E022204B1206D7
:10A1F00041468A61CB6153461B785BB29B46E6E7DA
:10A20000012342460493144B536043464A469E60E2
:10A21000DF601A621C615D615B46002BBFD00023CA
:10A2200000221900100002F00DFF43469861D96129
:10A230005B46022B00D15BE7B6E720002900FFF761
:10A240002FFD22002B0002F0CDF90028D3D10022EF
:10A25000034BCDE79C000020B01901000000F03F47
:10A260000000F0FF0000E03FFFFFEF470000F07F3D
:10A27000FFFFEFC7F0B54746CE4680B58DB004006E
:10A280000D0000F0CDFF294B06001B780F005BB2DC
:10A290009846013310D022002B002000290004F042
:10A2A00095F88146002807D10022002320002900CC
:10A2B00002F09EF9002806D1300039000DB00CBC28
:10A2C00090469946F0BD01230293194B06940795D9
:10A2D00003934B460A93434604940595002B15D0EF
:10A2E000002300221900100002F0ACFE4346089043
:10A2F0000991022B0ED104F067FA212303600A9B17
:10A300000193002B0CD1089E099FD5E70023002460
:10A310000893099402A801F031FF0028EFD1EAE781
:10A3200004F052FA0A9B01930360ECE79C000020C2
:10A33000B4190100F0B55746DE464E4645465C006E
:10A340006408E0B598461F00230093B083468A4610
:10A35000160013430CD07D4B4D00029181466D08D1
:10A360009D4212DD7A4B9C465B4665441D4361D19C
:10A370000023784C009301940098019913B03CBCE1
:10A3800090469946A246AB46F0BD9D4250D09C42B5
:10A39000E8DC6E4B9C426BD0002304935346002BA9
:10A3A00069DB002A10D1694B9C424CD0694B9C421E
:10A3B00000D1A3E08023DB05984500D1BCE0664BCB
:10A3C000984501D100F0D6FB5846514601F02CFECD
:10A3D0004B4600900191002B07D1002D67D05346CA
:10A3E0005C4A9B009B08934261D05346DB0F013BC4
:10A3F00099464A46049B134300D190E0574B9C4238
:10A4000000DCBBE0564B9C4201DC00F010FC554BDD
:10A410009D4201DC00F004FC4346002B23DD524A40
:10A42000524B1000190003F017FA00900191A3E7B6
:10A43000002805D04E4801F0A3FE009001919BE753
:10A44000AC42F7DCA5E75A46414BEB18134300D169
:10A450008EE7444B9D4200DC99E34346009601970A
:10A46000002B00DB88E7002300240093019483E79E
:10A47000002A91D076E73F4B9C423CDC394B9C4212
:10A480008FDD3D4923158C466344142B00DCB2E379
:10A490003421CB1A3100D94008009840904200D0B6
:10A4A0007FE70123194001335B1A049379E74346A0
:10A4B000002B07DA009A019B0020264902F0C2FD1A
:10A4C00000900191029B002B00DB55E7204B9C463E
:10A4D000049B65441D4301D100F00EFC049B012B3D
:10A4E00000D049E7009C019D8021220009066B18DD
:10A4F0000092019340E70223049352E758465146E5
:10A50000434600900191002B00DB35E75A46534645
:10A510000020104902F096FD009001912CE75A4668
:10A5200053465846514603F009FC02000B0002F066
:10A5300089FD009001911FE75A46534658465146FF
:10A5400003F08AF90090019116E7C0460000F07F01
:10A55000000010C00000F03F0000E03F0000E041BC
:10A560000000F043FFFFEF3F9C7500883CE4377E1E
:10A57000B8190100FFFF3F4301FCFFFFE44B00223D
:10A580009D420ADC009801990022E24B03F064F935
:10A5900035220D00009001915242DF492B158C4667
:10A5A000634498462D03DD4CDD4B2D0B90442C432A
:10A5B0009D420ADDDB4B9D4201DC00F001FC0123E2
:10A5C0009C46D94BE0449C466444002200230E92F2
:10A5D0000F931092119300220025D04B06920793FF
:10A5E00000980199069A079B21000890099103F0B1
:10A5F000A5FB069A079B0A900B910898099902F00F
:10A6000005FA02000B000020C44902F01BFD0A00FD
:10A61000010013000C910D9202000A980B9903F0AF
:10A620001BF90A000100130002910392002200921C
:10A630000193802364109B05234380242403A446B4
:10A6400000206344591904000D0002000B0000981B
:10A65000019903F001F902000B000A980B9903F02D
:10A660006DFB069A079B0A900B912000290003F0CE
:10A6700065FB02000B000898099903F05FFB009A44
:10A68000019B03F0E9F802000B000A980B9903F014
:10A6900055FB0C9A0D9B03F0DFF8029C039D08907C
:10A6A000099122002B002000290003F0D5F80400B6
:10A6B0000D009E4A9E4B03F0CFF89E4A9E4B02F03F
:10A6C000A5F922002B0003F0C7F89C4A9C4B02F02E
:10A6D0009DF922002B0003F0BFF89A4A9A4B02F032
:10A6E00095F922002B0003F0B7F8984A984B02F036
:10A6F0008DF922002B0003F0AFF8964A964B02F03A
:10A7000085F92200069007912B002000290003F014
:10A71000A3F802000B000698079903F09DF8009A31
:10A72000019B04000D000298039902F06FF9089A4A
:10A73000099B03F091F822002B0002F067F9009CBE
:10A74000019D0A900B9122002B002000290003F0AC
:10A7500083F80022814B04000D0002F057F90A9A99
:10A760000B9B02F053F900220B0011001A00069116
:10A7700007920A000098019903F06EF800220C90ED
:10A780000D9106980799754B03F0D8FA22002B001B
:10A7900003F0D4FA02000B000A980B9903F0CEFAEA
:10A7A000029A039B03F058F8069A079B04000D00D9
:10A7B0000898099903F050F802000B0020002900C6
:10A7C00002F024F904000D0002000B000C980D9912
:10A7D00002F01CF900221000E022614B12060090EA
:10A7E000019103F039F80C9A0D9B029003910098A7
:10A7F000019903F0A3FA02000B002000290003F0E6
:10A800009DFA584A564B03F027F8574A04000D00AA
:10A8100000980199554B03F01FF802000B0020002F
:10A82000290002F0F3F8109A119B02F0EFF806905D
:10A830000791404603F01CFE069A079B04000D009A
:10A840000298039902F0E2F80E9A0F9B02F0DEF8EC
:10A8500022002B0002F0DAF8002022002B000090EA
:10A86000019103F06BFA0E9A0F9B03F067FA029ABC
:10A87000039B03F063FA02000B000698079903F0AC
:10A880005DFA069007914A46049B013B134300D1B1
:10A8900088E10023214C0293039400223B00300006
:10A8A0003900140003F04AFA009A019B02F0D4FF29
:10A8B00032003B00049005910698079902F0CCFF06
:10A8C00002000B000498059902F0A0F83D00060074
:10A8D0000F000098019922002B000496059702F0C2
:10A8E000BBFF02000B00300039000092019302F020
:10A8F0008DF81F4B04000D008B460200994200DCCE
:10A9000055E11C4BCB18034300D0FBE134E0C046BB
:10A91000FFFF0F000000404301FCFFFF0000F03F7D
:10A920008E98030079B60B000000F0FFEF4E454A09
:10A93000287ECA3F65DBC9934A86CD3F01411DA9E8
:10A940006074D13F4D268F515555D53FFFAB6FDB1E
:10A95000B66DDB3F033333333333E33F000008404E
:10A9600009C7EE3FFD033ADCF5015B14E02F3EBE64
:10A97000FFFF8F40000070BF04980599E84AE94B3B
:10A9800002F044F8009A019B06000F002000290005
:10A9900003F0D4F902000B003000390001F03CFE56
:10A9A000AA46002800D0ADE18024DF4A53469446F1
:10A9B000640322001B1563441A411300DB495B4406
:10A9C0005A001E001B038C461B0B23431424520DFC
:10A9D000D74D62441541A21A134199465B46AE43D6
:10A9E00000203100002B02DA4B465B429946020000
:10A9F0000B000098019903F0A1F94B461B0500904C
:10AA00000191020098460B000498059901F0FEFFA1
:10AA10000D0000240022C74B2000290002F01CFF7B
:10AA2000009A019B069007912000290003F086F907
:10AA300002000B000498059903F080F9BE4ABF4B51
:10AA400002F00AFFBE4A06000F00BE4B200029009C
:10AA500002F002FF02000B003000390001F0D6FFC7
:10AA600004000D0002000B000698079901F0CEFFCC
:10AA7000069A079B06000F0003F060F902000B0026
:10AA80002000290003F05AF93200009001913B00A8
:10AA90003000390002F0E0FE04000D00AA4AAB4B82
:10AAA00002F0DAFEAA4AAB4B03F048F922002B0071
:10AAB00002F0D2FEA84AA94B01F0A8FF22002B0009
:10AAC00002F0CAFEA64AA74B03F038F922002B0079
:10AAD00002F0C2FEA44AA54B01F098FF22002B0011
:10AAE00002F0BAFE02000B003000390003F026F934
:10AAF00004000D0002000B003000390002F0ACFE33
:10AB00008023049005910022DB052000290003F03A
:10AB100015F902000B000498059902F093FA009AC7
:10AB2000019B04000D003000390002F095FE009AF0
:10AB3000019B01F06BFF02000B002000290003F0D5
:10AB4000FDF832003B0003F0F9F802000B00002092
:10AB5000874903F0F3F843465B181A15002A00DC16
:10AB60003FE11900029A039B02F076FE00900191EA
:10AB7000FFF702FC5346002B01DAFFF725FC58468D
:10AB8000514600F04DFB00900191FFF7F5FB434665
:10AB9000002B00DB67E480231B06FB180096019363
:10ABA000FFF7EAFB0023734C0293039475E64B0016
:10ABB0005B089A46704B9A4500DCF9E06F4B5B44AA
:10ABC0001A430AD1009A019B03F0B8F8049A059B36
:10ABD00001F02CFD002800D1E6E602980399684AAE
:10ABE000684B02F039FE664A664B02F035FE009073
:10ABF0000191FFF7C1FB002A01D0FFF7E5FB1432FA
:10AC0000D31A22001A4111009940A14201D0FFF746
:10AC1000CDFB01231A40DB189B1A0493FFF7C6FBF8
:10AC20004346002B01DBFFF71EFCFFF7F8FB564BFA
:10AC30009D42F5DD4E4B9D4201DDFFF7EDFB009897
:10AC4000019900224A4B03F079F8C0224F4BD205FC
:10AC500004000D0002F000FE4D4A029003914D4B9E
:10AC60002000290002F0F8FD0022009001914A4BDB
:10AC70002000290002F0F0FD02000B00474848497F
:10AC800003F05CF822002B0002F0E6FD02000B004E
:10AC90000020444903F052F82200069007912B004F
:10ACA0002000290002F0D8FD02000B000698079949
:10ACB00002F0D2FD1A4A354B02F0CEFD02000B0025
:10ACC0000098019903F03AF802000B0004000D000F
:10ACD0000298039901F09AFE029A039B00200090CB
:10ACE000019103F02BF802000B002000290003F073
:10ACF00025F806900791C6E50098019902000B001F
:10AD0000FFF711FC284A294B0298039902F0A4FD91
:10AD1000254A264B02F0A0FD00900191FFF72CFB85
:10AD2000FE822B654715973C02FCFFFF01FCFFFFED
:10AD3000FFFF0F00432EE63FEF39FAFE422EE63FBB
:10AD4000396CA80C615C20BED0A4BE726937663E27
:10AD5000F16BD2C541BDBB3E2CDE25AF6A56113F1B
:10AD600093BDBE166CC1663F3E5555555555C53F02
:10AD70000000F03F0000F0BFFFCB904000346F3F79
:10AD800059F3F8C21F6EA501FEFFEF3F4715F73FCD
:10AD900044DF5DF80BAE543E0000D03F555555558D
:10ADA0005555D53F0000E03F9C7500883CE4377E58
:10ADB00000220E4B904691469A4500DC29E6F3E5C9
:10ADC00080220B4BD2050E920F930A4A0A4B802524
:10ADD000109211930022094BED0206920793FFF7A0
:10ADE000FFFB4A4601F0D2F9BCE6C0460000E03F56
:10ADF00003B8E23F06D0CF43EBFD4C3E0000F83FE6
:10AE0000F0B54E464546DE465746E0B5E14B4C00B0
:10AE10008FB09046894664089C4200DC87E0DE4B98
:10AE20009C4222DCDD4A002900DC92E0DC4B02F08F
:10AE300085FFDB4B06000F009C4200D17EE1D94A22
:10AE4000D94B02F07BFF02000B00414630000A6044
:10AE50004B60390002F072FFD34BD24A02F06EFF12
:10AE6000434601259860D9606BE0D04B9C4200DCE2
:10AE70008FE0CF4B9C4200DD55E1CE4A2315924630
:10AE80009A4451460905631A19001D00040003F095
:10AE9000B9FA03F0EDFA02000B0020002900089235
:10AEA000099302F04BFF0022C34B02F0D5FC0F00C8
:10AEB000060003F0A7FA03F0DBFA04000D0002001D
:10AEC0000B00300039000A940B9502F037FF002286
:10AED000B94B02F0C1FC002200230C900D9101F04F
:10AEE00081FB002800D192E10023002220002900EC
:10AEF00001F078FB434243410133B04A414601929D
:10AF0000022208A80092524600F07CFB4B46050046
:10AF1000002B16DA802243461206944642465B68AE
:10AF2000454263445360D3686344D36009E00B0037
:10AF3000020041460A604B600022002300258A601F
:10AF4000CB6028000FB03CBC90469946A246AB4669
:10AF5000F0BD934B01F05AFD914B06000F009C424F
:10AF600000D13DE18F4A904B01F050FD02000B00F3
:10AF7000414630000A604B60390002F0DFFE894A2A
:10AF8000894B01F043FD012543466D429860D9602D
:10AF9000D7E701F049F88A4A8A4B06000F0002F011
:10AFA0005BFC0022884B01F031FD03F02BFA050019
:10AFB00003F05EFA794A7A4B0490059102F04CFC5A
:10AFC00002000B003000390002F0B8FE754A06009E
:10AFD0000F0004980599744B02F03EFC0290039117
:10AFE0001F2D00DCC7E0029A039B3000390002F0FD
:10AFF000A5FE83468A4653465B0024155B0DE31A83
:10B00000102B6CDD04980599D322674B520502F092
:10B0100023FC02000B00300039000292039302F07F
:10B020008DFE0A000100130006910792020039000C
:10B03000300002F083FE029A039B02F07FFE0600BE
:10B040000F0004980599614A614B02F005FC32003B
:10B050003B0002F073FE069E079F0B0002003900C2
:10B0600030000292039302F069FE4B005B0D8346B1
:10B070008A46E41A312C32DD04980599B822544BE3
:10B08000920502F0E9FB03000C0002000293039416
:10B090000B000698079902F051FE02000B00060013
:10B0A0000F000698079902F049FE029A039B02F0EE
:10B0B00045FE484A0290039104980599464B02F0D8
:10B0C000CBFB029A039B02F039FE02000B0030001A
:10B0D00039000292039302F031FE83468A465A46B3
:10B0E0005346414630000A604B60390002F026FEAC
:10B0F000029A039B02F022FE44460B000200A2606B
:10B10000E3604B46002B00DB1BE75B46236080239C
:10B110001B065344636080231B069C466144A06069
:10B12000E1606D420DE70B00020002F007FE4346AE
:10B1300000259860D9601860596002E7D3221A4B45
:10B14000520502F0FBFD214A214B0D00040002F0E4
:10B15000F5FD02000B00414620000A604B6029000B
:10B1600002F0ECFD1A4B194A02F0E8FD43460125B6
:10B170009860D960E5E602000B003000390002F06B
:10B18000DDFD6B1E154A9B009B5883468A46A342F1
:10B19000A5D130E7FB21E93F7BD9024000004054B4
:10B1A000FB21F93F3163621A61B4D03DFB21394183
:10B1B000FFFFEF7FEAFBFFFF000070413C1A010038
:10B1C00083C8C96D305FE43F0000E03F7370032E19
:10B1D0008A19A33BC14920259A837B39BC190100F8
:10B1E000D3220C4B520501F011FC0B4A0B4B04000F
:10B1F0000D0001F00BFC02000B00414620000A602C
:10B200004B60290002F09AFD034A044BB9E6032380
:10B2100073E6C04661B4D03D7370032E8A19A33B18
:10B22000F8B54746CE46674B80B50A000F001900B7
:10B2300005003940994200D19BE004000100002F35
:10B2400069DD3F1500D1B4E05F4B12039C468023BB
:10B25000120B5B0313435B00CA0F67449B184A0041
:10B26000F80703D5D20F5B009B188A0079108C4633
:10B27000002180201624894680030D189D4202DC9F
:10B2800029185B1B8144D50F5B00013C5B19520000
:10B290004008002CF1D10020804680202025002786
:10B2A000000609E08B425CD0D40F5B00013DE3183F
:10B2B00052004008002D16D0C4198B42F2DD271829
:10B2C0000E00002C49DB5B1AA242894149425B1AFD
:10B2D000121BD40F5B00013D80443100E318520083
:10B2E0004008002DE8D113434ED143465B0837494F
:10B2F0004A468846494652104244C90702D5802131
:10B3000009060B4361460F05BD18180029000CBC47
:10B3100090469946F8BD7B005B0803433900002B3B
:10B32000F5D0002F3CD1E30A153A6405002BFAD082
:10B330008020400303423FD1002700E00F005B0064
:10B34000791C0342FAD0250020208D40401A2900A4
:10B35000D71B2200C2401A4376E7FE43F60F8E1930
:10B36000B1E79442A0D82718002CF6DB1E0000237A
:10B37000AEE702003B002800390002F06DFA2A0017
:10B380003B0001F043FBC2E74346013303D0434691
:10B3900001335B08ABE7012398460023C144A6E7CD
:10B3A0003B00020002F0CAFC02000B0001F04AFE62
:10B3B000ADE713000022BBE70127210020207F42D8
:10B3C000C6E7C0460000F07F01FCFFFF0000E03F41
:10B3D000F0B54746CE4680B587B000920193754BD5
:10B3E0004F00814688467F089F4263DC03F00AF8DD
:10B3F000002800D1D4E04A4643464846414602F080
:10B400002BFA04000D006C4A6C4B02F025FA6C4AD2
:10B410006C4B01F0FBFA22002B0002F01DFA6A4A85
:10B420006A4B02F08BFC22002B0002F015FA684AEE
:10B43000684B01F0EBFA22002B0002F00DFA664A8D
:10B44000664B02F07BFC22002B0002F005FA644AF6
:10B45000644B01F0DBFA22002B0002F0FDF90290B0
:10B4600003910022604B2000290002F0F5F9029AB6
:10B47000039B06000F002000290002F0EDF9009A5E
:10B48000019B04000D004846414602F0E5F9020028
:10B490000B002000290002F051FC02000B003000DC
:10B4A000390002F04BFC02000B0000204F4902F073
:10B4B00045FC70E002000B0002F0CEF904000D0024
:10B4C0003D4A3E4B02F0C8F93D4A3E4B01F09EFA20
:10B4D00022002B0002F0C0F93B4A3C4B02F02EFC4C
:10B4E00022002B0002F0B8F9394A3A4B01F08EFAEB
:10B4F00022002B0002F0B0F9374A384B02F01EFC54
:10B5000022002B0002F0A8F9354A364B01F07EFAF2
:10B510002B00220002F0A0F9354B029003919F42CC
:10B520009FDD344B00229F423DDC334900207B18D5
:10B530002E4916001F0002F001FC04900591002224
:10B54000294B2000290002F087F932003B0002F06D
:10B55000F5FB029A039B06000F002000290002F071
:10B560007BF9009A019B04000D004846414602F019
:10B5700073F902000B002000290002F0DFFB02003B
:10B580000B003000390002F0D9FB02000B000498D8
:10B59000059902F0D3FB07B00CBC90469946F0BD6C
:10B5A00000201249F7E7154B002604920593144F2B
:10B5B000C5E7C046FFFF3F3ED43888BEE9FAA8BDC4
:10B5C000C4B1B4BD9EEE213EAD529C804F7E923EF2
:10B5D0009015CB19A001FA3E7751C1166CC1563FA8
:10B5E0004C5555555555A53F0000E03F0000F03F34
:10B5F0003233D33F0000E93F0000E0FF0000E73FA7
:10B600000000D23FF0B5DE464E4645465746E0B50F
:10B61000DC4CA5440D9114001900A49A0993DA4B4F
:10B620009200D6584D1E03901821E01E06960295F2
:10B6300000F0CEFEC3430100DB1719404B1C9A00FB
:10B640009B1ADB001B190B9105934C1B771918D41F
:10B65000A59BA5009C463F1922AE6544013707E033
:10B66000286802F005FF013403C60435BC4208D047
:10B67000002CF5DA00200021013403C60435BC4259
:10B68000F6D1069B002B01DA00F0FDFB069B039927
:10B690000133DB009A46099BDA00944600920022AF
:10B6A000914672AA0492B94A6144934688469AAB7D
:10B6B00063449B44029B002B00DABCE15D460026FC
:10B6C0000027039C4D442A686B6803CC02F0C4F841
:10B6D00002000B003000390001F098F9083D060027
:10B6E0000F004445EFD1049B4B441E605F6008236C
:10B6F0009C46E144D145DDD10EA80421844649424F
:10B7000061448C46069A93009C44614684460A91A3
:10B710000399083B63448C460C93009B009263445E
:10B720009B46009A0498D10003008C46634408911C
:10B730001E685F68002A33DD954980468C46624466
:10B74000D300984470AB9A460EAB99460022914BB9
:10B750003000390002F080F802F054FE02F088FE5A
:10B7600000228D4B04000D0002F076F802000B0061
:10B770003000390002F0E2FA02F044FE4B4601C309
:10B780009946434620001A685B68290001F03EF99B
:10B7900008235B429C46E04406000F00D045D5D10B
:10B7A000059B30001A003900984600F0EFFCFF239B
:10B7B00000229B0504000D0002F04EF800F042FC50
:10B7C0000022764B02F048F802000B00200029000E
:10B7D00002F0B4FA0D00040002F014FE814602F0FB
:10B7E00047FE02000B002000290002F0A7FA060025
:10B7F00040460F00002800DCEEE0009B18215A1E96
:10B8000092000EAB9B58091A1D000D41A9448D40B2
:10B810005D1B0EAB9D5017231B1A1D41002D2DDD06
:10B8200001239C46009BE144002B00DC1CE20E9CA3
:10B830000123002C00D0B5E0009A012A09D099001C
:10B840000EAA54580133002C00D0ACE0009A9A4262
:10B85000F5D1059B002B0EDD012B00D1A8E1022BB9
:10B8600009D1009B0EA95A1E92000EAB9B5807935C
:10B870009B029B0A8B50022D00D1C1E000230022C5
:10B880003000390000F0AEFE009B002800D194E2A9
:10B89000069A591E8A4210DC414A0A9894460EAA1A
:10B8A0006344944600229B0063441C68043B22438B
:10B8B0008342FAD1002A00D0C0E0069B0EAA013BC9
:10B8C0009B00D358002B00D0B3E001220C9B043B1B
:10B8D000596801320029FAD0009B9C46624411004D
:10B8E00007921A0001338B4246DC0B986346804670
:10B8F000A59C4344A046099C9B00A1464A44984409
:10B90000D30022AA9146049A99449446089BA59A8A
:10B9100063448446614494469A468B006344009392
:10B920004346586802F0A4FD4B4618605960029BDC
:10B93000002B24DB4D46039C0026002701E02868ED
:10B9400069680CCC01F088FF02000B003000390060
:10B9500001F05CF8083D06000F005C45EFD153464E
:10B960009E60DF6004239C460433E0449C46009BB9
:10B97000E144E2449845D3D1079B0093D1E60026E9
:10B980000027ECE794FDFFFF881B010018FEFFFF76
:10B99000FFFFFF1F0000703E0000704100002040CC
:10B9A000FFFFFF3F002180225204141B0EAA5450B7
:10B9B000009999420EDD0EA884469B000EAA8900CC
:10B9C000D25861446344CF4800E01A68821A04C325
:10B9D0008B42FAD101243CE7059B002B06D1009B4A
:10B9E0000EAA013B9B00D558ED1517E70022C64B68
:10B9F000300000F01BFE002800D024E100253DE7C8
:10BA000032003B000020C14902F098F906000F0007
:10BA1000002C00D132E7059A0020BC4900F0B6FBAB
:10BA200002000B003000390002F088F906000F0018
:10BA300024E7012250E70026002754E64B46059AEA
:10BA4000079388468B000EA9CB58183A08950592A3
:10BA5000002B0DD18C464146AD4B43449B006344C3
:10BA6000043B58680139183A0028F9D088460592F5
:10BA7000059A0020A54900F089FB434604000D000B
:10BA8000002B00DA05E29E000EAB9C464346DB002D
:10BA900066449C46059370AB9946049F67440097A3
:10BAA000306802F0E5FC22002B0001F0D5FE0022F8
:10BAB00038607960974B2000290001F0CDFE083FE7
:10BAC00004000D00043EB945EAD14AAB03939B46FE
:10BAD00000239A46069B424699464346013202920B
:10BAE00004934B46002B00DAAAE080208A4B009D8D
:10BAF0009846C005894900260027002408E008234D
:10BB00009C460835E044544511DC434618685968A2
:10BB10002A686B6801F0A0FE02000B0030003900BB
:10BB200000F074FF013406000F00A145E7DA5B4620
:10BB3000C0C39B4601239C46009BE244083B009304
:10BB4000029B9A45CDD1049B9846A49B022B00DD15
:10BB50008EE0002B37DC1FD1059B00271D00039BC7
:10BB600000249C461E006544083E2A686B68380025
:10BB7000210000F04BFF083D07000C00AE42F4D15D
:10BB8000089B002B03D080231B069C4664443A008C
:10BB900023000D990A604B600720079B18409B23E8
:10BBA0009B009D443CBC90469946A246AB46F0BDE6
:10BBB000009B0EA95A1E92000EAB9B5807935B0286
:10BBC0005B0A8B5057E64346002B00DA70E10020F9
:10BBD0000021DB004AAAD61848AF32687368083ED5
:10BBE00000F014FFB742F8D1089B002B00D025E1EC
:10BBF0000B0002004A984B990D9C2260636002F092
:10BC00009DF8434607000C00002B13DD01254CAEC8
:10BC1000B14638002E0021004C4601360CCC00F015
:10BC2000F5FEA146B045F7DA089B07000C00002B93
:10BC300000D015E13A0023000D998A60CB60ABE794
:10BC40000026002773E701239C46009BE144022560
:10BC5000002B00DDEBE532003B0000202B4902F019
:10BC60006DF806000F0009E60024F2E54AAB0393E5
:10BC7000A49B032B00D08FE74346002B00DC14E18C
:10BC8000039ADB009B46130091465B441E685F6885
:10BC9000234B43440293DB00994448AB9A464B46FE
:10BCA0005C681B681800210032003B000090019185
:10BCB00000F0ACFE04000D0002000B00009801999A
:10BCC00002F03CF83B00320000F0A0FE4B469860CA
:10BCD000D9601C605D6008235B429C46E1442600FD
:10BCE0002F00CA45DBD14346012B00DCE3E0039A79
:10BCF00013005B441E685F68029BDB0099464A4460
:10BD0000904610E0FFFFFF000000E03F0000F03F22
:10BD1000FFFFFF3F0000703E481B0100FB21F93F81
:10BD2000FFFFFF1F984643465C681B681800210010
:10BD300032003B000090019100F068FE04000D000D
:10BD400002000B000098019901F0F8FF32003B005F
:10BD500000F05CFE4346039A9860D9601C605D6009
:10BD6000083B26002F009A42DCD14D46944600261F
:10BD700000244746083565442A686B683000210076
:10BD800000F044FE083D06000C00AF42F4D1039BD6
:10BD90004A9F5D689968D868089B002B65D080220F
:10BDA000120694460D9B6544604464441F605D60C8
:10BDB0009960D8601E615C61EEE69A464B46079337
:10BDC000059B30005A423900089500F0DFF9002247
:10BDD0003A4B06000F0000F029FC002824D0384B15
:10BDE00000223000390001F037FD02F00BFB524613
:10BDF0000400950002F03CFB0022304B01F02CFDCA
:10BE000002000B003000390001F098FF02F0FAFA4E
:10BE10000EAA50510122059B5244183390460593B7
:10BE200093000EAAD45023E65346300039009C00FC
:10BE300002F0E8FA0EAB1851D04619E680230D9AAD
:10BE40001B06CB18106053600B0002004A984B99F8
:10BE500001F074FF434607000C00002B00DDD5E61F
:10BE600080231B069C466444E4E62B003A000D9DAB
:10BE70002A606B600A000300AA60EB6032002300B6
:10BE80002A616B6188E6099BDB00009372AB049327
:10BE900032E4A49B022B00DDE8E6002B00DD92E6F5
:10BEA00000D079E6002700246AE6002600246EE729
:10BEB0000020002198E60026340068E70000704169
:10BEC0000000703EF0B5CE46474680B587B0009280
:10BED0000193474A4B00814688465B08934207DC42
:10BEE0004146484602F08EFA4146031E484666D057
:10BEF0004A4643464846414601F0AEFC04000D0068
:10BF000002000B004846414601F0A6FC394A3A4B74
:10BF100006000F002000290001F09EFC374A384B34
:10BF200001F00CFF22002B0001F096FC354A364B45
:10BF300000F06CFD22002B0001F08EFC334A344BE4
:10BF400001F0FCFE22002B0001F086FC314B324A4E
:10BF500000F05CFD0E9B02900391002B34D0009802
:10BF6000019900222D4B01F077FC029A039B04906B
:10BF700005913000390001F06FFC02000B000498BD
:10BF8000059901F0DBFE22002B0001F065FC009A10
:10BF9000019B01F0D3FE224A04000D00214B30002A
:10BFA000390001F059FC02000B002000290000F0CC
:10BFB0002DFD02000B004846414601F0BFFE07B0D0
:10BFC0000CBC90469946F0BD02000B0020002900F1
:10BFD00001F042FC124A134B01F0B0FE32003B006C
:10BFE00001F03AFC4A46434600F010FDE7E7C04640
:10BFF000FFFF3F3E7CD5CF5A3AD9E53DEB9C2B8ADB
:10C00000E6E55A3E7DFEB157E31DC73ED561C11935
:10C01000A0012A3F1111813FA6F810110000E03F56
:10C02000495555555555C53F49004B0819007047AE
:10C03000034B48009C4640086044C00F7047C04610
:10C0400000001080474AF0B54F4691464B005B0D0B
:10C0500099444646D6464A46C0B505000C000E0037
:10C0600088460700132A27DC002A4BDB3E4B13418E
:10C070009A460B0052461340034318D03B4A3C4BB0
:10C080002800210000F0C2FC0022002300F0C4FAC6
:10C09000002847D0002C04DA80234A465B03134172
:10C0A00098444646534600279E43380031001CBC46
:10C0B00090469946A246F0BD332A08DD8023DB0076
:10C0C0009945F4D102000B0000F0A0FCEFE7294AEB
:10C0D0009446012263445242DA4092460242E6D03C
:10C0E000224A234B2800210000F090FC002200236C
:10C0F00000F092FA002815D0002C1EDB534646466D
:10C100009F430FE0194A1A4B2800210000F07EFCE3
:10C110000022002300F080FA002803D0002C04DB6A
:10C120000027002638003100C1E764006408254379
:10C130000027002DF6D0104EF4E74B46142B0BD001
:10C140003422D21A012393405D19BD4208D2012343
:10C150009C462F00E044D1E7133B9C46E044CDE7EA
:10C160002F00CBE701FCFFFFFFFF0F009C7500884D
:10C170003CE4377EEDFBFFFF0000F0BF002070477E
:10C18000002001497047C0460000F87F4B0070B5A1
:10C190005B0D14000A00002B1AD14B005B0803430F
:10C1A00015D0234B002201F057FB224B9C422DDB84
:10C1B0000A004B005B0D363B1F4DE318AB422ADCF7
:10C1C000002B0DDD1D4C1B0522401A43110070BDD4
:10C1D0001B4DAB42F0D102000B0000F017FCF6E75C
:10C1E0001D00353519DA174B02009C4209DD0B00A2
:10C1F0001548164900F032F8134A144B01F02CFB95
:10C20000E5E70B001248134900F028F8104A114BDB
:10C2100001F022FBDBE70200E9E7084C363322405D
:10C220001B051343190000220B4B01F015FBCEE751
:10C2300000005043B03CFFFFFE070000FFFF0F80EF
:10C24000FF07000050C300009C7500883CE4377E67
:10C2500059F3F8C21F6EA5010000903C30B54A00AA
:10C26000DB0FDB0752081A43110030BD02B47146E0
:10C2700049084900095649008E4402BC7047C0462F
:10C2800002B4714649084900095C49008E4402BC69
:10C290007047C04603B47146490840004900095E32
:10C2A00049008E4403BC704703B4714649084000FE
:10C2B0004900095A49008E4403BC704700224308D4
:10C2C0008B4274D303098B425FD3030A8B4244D35E
:10C2D000030B8B4228D3030C8B420DD3FF220902A0
:10C2E00012BA030C8B4202D31212090265D0030B5F
:10C2F0008B4219D300E0090AC30B8B4201D3CB0355
:10C30000C01A5241830B8B4201D38B03C01A524196
:10C31000430B8B4201D34B03C01A5241030B8B4298
:10C3200001D30B03C01A5241C30A8B4201D3CB0283
:10C33000C01A5241830A8B4201D38B02C01A524168
:10C34000430A8B4201D34B02C01A5241030A8B426B
:10C3500001D30B02C01A5241CDD2C3098B4201D383
:10C36000CB01C01A524183098B4201D38B01C01A01
:10C37000524143098B4201D34B01C01A5241030978
:10C380008B4201D30B01C01A5241C3088B4201D327
:10C39000CB00C01A524183088B4201D38B00C01AD4
:10C3A000524143088B4201D34B00C01A5241411AFB
:10C3B00000D20146524110467047FFE701B5002008
:10C3C00000F0F0F802BDC0460029F7D076E77047CC
:10C3D00003460B437FD4002243088B4274D30309E6
:10C3E0008B425FD3030A8B4244D3030B8B4228D387
:10C3F000030C8B420DD3FF22090212BA030C8B42AD
:10C4000002D31212090265D0030B8B4219D300E04C
:10C41000090AC30B8B4201D3CB03C01A5241830BD1
:10C420008B4201D38B03C01A5241430B8B4201D381
:10C430004B03C01A5241030B8B4201D30B03C01AAA
:10C440005241C30A8B4201D3CB02C01A5241830A24
:10C450008B4201D38B02C01A5241430A8B4201D353
:10C460004B02C01A5241030A8B4201D30B02C01A7D
:10C470005241CDD2C3098B4201D3CB01C01A5241E4
:10C4800083098B4201D38B01C01A524143098B426D
:10C4900001D34B01C01A524103098B4201D30B0156
:10C4A000C01A5241C3088B4201D3CB00C01A52417B
:10C4B00083088B4201D38B00C01A524143088B4240
:10C4C00001D34B00C01A5241411A00D201465241D9
:10C4D000104670475DE0CA0F00D04942031000D3F8
:10C4E0004042534000229C4603098B422DD3030A4D
:10C4F0008B4212D3FC22890112BA030A8B420CD35D
:10C50000890192118B4208D3890192118B4204D385
:10C5100089013AD0921100E08909C3098B4201D305
:10C52000CB01C01A524183098B4201D38B01C01A3F
:10C53000524143098B4201D34B01C01A52410309B6
:10C540008B4201D30B01C01A5241C3088B4201D365
:10C55000CB00C01A524183088B4201D38B00C01A12
:10C560005241D9D243088B4201D34B00C01A5241E9
:10C57000411A00D20146634652415B10104601D376
:10C580004042002B00D54942704763465B1000D300
:10C59000404201B5002000F005F802BD0029F8D0A6
:10C5A00016E770477047C046D0400B1C1141203A37
:10C5B00003D49C46134118436346524293401843A8
:10C5C0007047C0468446101C62468C46191C634660
:10C5D00000E0C0461FB501F0D7F8002801D40021C3
:10C5E000C8421FBD10B501F02FF84042013010BD08
:10C5F00010B501F0C9F8002801DB002010BD0120B2
:10C6000010BDC04610B501F0BFF8002801DD0020C4
:10C6100010BD012010BDC04610B501F051F8002832
:10C6200001DC002010BD012010BDC04610B501F096
:10C6300047F8002801DA002010BD012010BDC046D7
:10C64000002B15D1002A13D1002906DB01DC0028BC
:10C6500006D00020C043410802E0802109060020E6
:10C6600007B4024801A14018029003BD39FFFFFF43
:10C6700003B4684601B5029800F030F8019B9E466D
:10C6800002B00CBC7047C046F0B5CE464746150414
:10C690002D0C2E0080B50704140C3F0C9946030C9A
:10C6A0007E435D43674363437F19340CE4199C4622
:10C6B000A54203D980235B029846C4444B464343BA
:10C6C0005143250C36046544360C2404A4195B1927
:10C6D000591820000CBC90469946F0BDF0B583B0C7
:10C6E00016001F000090019101F06CFF04000D0086
:10C6F00002000B0030003900FFF7C6FF009A019BD3
:10C70000121A8B41089920000A604B60290003B07F
:10C71000F0BDC046F0B54E4657464546DE46E0B54C
:10C7200043025B0A450083B00F1C99462D0EC60FCD
:10C73000002D57D0FF2D24D08020DB00C0041843EB
:10C74000002381469A469B467F3D7C027A00FB0F80
:10C75000640A120E984623D0FF2A4BD0E3008024AF
:10C760000020E4047F3A1C43AD186B1C474601933C
:10C77000534677403A000F2B48D87D499B00CB5851
:10C780009F46002B00D085E008339A46063B9B4627
:10C790007C027A00FB0FFF25640A120E9846DBD15B
:10C7A000002C00D090E0524601231A43924601200B
:10C7B000DBE74C4658461700022824D0032800D156
:10C7C000CFE00022002301284DD15802D205400AB3
:10C7D000FF071043384303B03CBC90469946A2463D
:10C7E000AB46F0BD002B5BD104239A46033B0025EA
:10C7F0009B46AAE7FF35002C60D1524602231A431C
:10C8000092460220B1E7FF220023DEE74B461B0CD5
:10C810009C464B462604360C180461463300220C15
:10C820006446000C43434E435043544380191A0C52
:10C830001218964203D9802149028C4664441B0495
:10C840001B0C1004C01883015E1EB341800E1843F8
:10C85000130C1B199B0103431C00230179D50123F1
:10C8600062081C401443019A7F32002A4DDD6307A1
:10C8700004D00F232340042B00D00434230103D51C
:10C880003C4B019A1C408032FE2ABCDCA3015B0AAF
:10C89000D2B29AE70C239A46093BFF259B4654E700
:10C8A000180001F071FE4A46431F76259A40002386
:10C8B0006D4291462D1A9A469B4646E752460323FF
:10C8C0001A439246032050E7200001F05DFE431F0B
:10C8D0002D1A9C40763D002047E780230027DB038C
:10C8E000FF2272E7424666E74C463200584662E74E
:10C8F00080234A46DB031A4222D01C4220D1234324
:10C900005B025B0A4746FF225FE701239A1A1B2A54
:10C9100021DC23000199D3409E318C401A00230072
:10C920005C1EA34113435A0704D00F221A40042A65
:10C9300000D004335A0111D49B015B0A002244E762
:10C9400080234A46DB0313435B025B0A3700FF2266
:10C950003BE7019587E70022002336E70122002309
:10C9600033E78023DB0323435B025B0AFF222CE7D0
:10C97000981B0100FFFFFFF770B500283DD0C317DB
:10C98000C5185D40C40F280001F0FEFD9E22121A5A
:10C99000962A07DCD2B2082833DD083885406802C1
:10C9A000400A23E0992A0BDD052329001B1AD940F0
:10C9B00003001B339D402B005D1EAB4119430D004E
:10C9C000052801DD431F9D402B000F490B406E07DA
:10C9D00009D00F263540042D05D004335D0102D562
:10C9E0009F220B40121A9B01580AD2B24002D20574
:10C9F000400AE4071043204370BD002400220020B9
:10CA0000F4E76802400AF1E7FFFFFFFBF0B54F468D
:10CA10004646D6460C000903C0B5490A470F5E00DA
:10CA200039431F03DB0F9C4665007B0A570F1F43EA
:10CA30006D0DE40F760DA146C000B846D200AB1BC9
:10CA400064457BD0002B5FDD002E00D0A4E03E00CB
:10CA5000164300D112E15E1E002E00D09EE1871A1F
:10CA60004346B84280410125C91A4042091A0B02C7
:10CA700000D431E149024E0A002E00D16EE13000AF
:10CA800001F082FD0300083B1F2B00DD61E1202245
:10CA90003900D21A9E40D1409F400E439D4200DD96
:10CAA00051E15D1B6B1C1F2B00DD7CE12021C91AAD
:10CAB0003D0030008F408840DD40791E8F413100BD
:10CAC00007222843D940002507433A40002A09D0CD
:10CAD0000F233B40042B05D03B1DBB42BF417F428F
:10CAE000C9191F000B0200D426E26A1CC64B55056B
:10CAF0006D0D9A4200D106E1C44AFF080A4053076F
:10CB000052023B43120B8EE0002B00D0B8E06B1CAE
:10CB10005B055B0D012B00DC30E1871A4346B84210
:10CB2000B641CB1A76429E1B330200D54CE13B0046
:10CB30003343A1D100220024002570E0002B00DC4B
:10CB4000E5E0002E00D183E0AF4EB54260D08026F4
:10CB500036043743B846382B00DC3EE143461343E6
:10CB60001F007A1E97413F188742804140420918B2
:10CB70000B0200D4B0E0A44B01359D4200D1C3E0CC
:10CB8000A24A7B080A4001210F401F435108D307E6
:10CB900007221F433A4099E79B4EB54238D0802682
:10CBA00036043743B846382B00DDDCE01F2B00DCB1
:10CBB00030E11E004746203EF740BC46202B04D003
:10CBC0004026F31A46469E403243170063467A1EBB
:10CBD00097411F43CCE0002B00D104E243461343AE
:10CBE00000D159E14B07C00818438023C9081B0333
:10CBF000194208D04546ED081D4204D14346D008ED
:10CC0000590708432900420FC9007F4D1143C00056
:10CC10004B07CA087C49C00803438D4268D0120301
:10CC20006D05120B6D0D002112031800130B0A0D78
:10CC300012051A43764B2D0513402B435B00E40786
:10CC40005B08234319001CBC90469946A246F0BDE0
:10CC50003E00164312D05E1E002E00D000E1871861
:10CC60008742804141444042091801250B0233D5D7
:10CC7000022585E764463300414610001D00C7E7E2
:10CC8000002D00D0DAE00C000443F3D05C1C00D18E
:10CC90009FE15D4CA64200D12FE1DB43382B00DD44
:10CCA00066E11F2B00DD83E120240500E41A0F005C
:10CCB000DD40D940A0404346A7405B1A441EA04136
:10CCC00098462F433843171ABA429241434652427C
:10CCD000991A64463500CAE607223A40002A00D075
:10CCE000F6E64B07CA084849FF083B438D4296D1F8
:10CCF0001900114300D19EE1802109030A43120368
:10CD0000120B414D8FE71500002200238BE7002B0B
:10CD100000D0C7E06B1C5F057F0D012F00DCF1E048
:10CD2000394DAB4200D1B9E085180A0085428941EE
:10CD30004244494251180722CF076D082F43490842
:10CD40003A401D00C2E607223049ED1A31403A4010
:10CD5000BCE63E002838864000279FE6380001F0F8
:10CD600013FC20308EE6434613431F007A1E974182
:10CD7000C71BB84280414042091A78E60E003B00CA
:10CD800006431343002D61D1002E00D0F4E0002BA8
:10CD900000D11BE164463900100039E71A4FBB424D
:10CDA0007AD03300FFE630001F3DE840202B03D04F
:10CDB0004021CB1A9E4037437B1E9F4107220743E9
:10CDC0003A400021002589E7171A4346BA42B64186
:10CDD000591A76428E1B64464EE61F2B00DDADE0ED
:10CDE00020264746F61AB740B9461700B246DF403C
:10CDF0004E463E4337005646B240561EB241174398
:10CE00004246DA408918AEE6FF070000FFFF7FFFC9
:10CE1000FFFF0F8020264746F61AB740B946170095
:10CE2000B246DF404E463E4337005646B240561E9D
:10CE3000B24117434246DA40891A99E77F4CA6422D
:10CE40005BD0802424045B42214327E7002E0CD1D1
:10CE5000002B00D1CBE0644639001000774DD7E6B7
:10CE6000764FBB4218D0330075E6002B14D04B0729
:10CE7000C00818438023C9081B03194207D0FC08C7
:10CE80001C4204D17907D0080843E14621004C46F2
:10CE9000420FC9001143C000684DB9E61D000022D1
:10CEA0000023C0E6002D5BD10D00054300D1E2E672
:10CEB0005D1C00D1B0E0614DAE421FD0DB43382B8A
:10CEC00071DC1F2B00DD96E020250F00ED1AAF402E
:10CED000B9460700AA46DF404D463D432F00554660
:10CEE000A840D940451EA84188440743BF1897422F
:10CEF00092415142414435003AE66446350041468C
:10CF0000100085E60B000343002D00D063E6002BE4
:10CF1000F5D04346134300D17AE687188742804113
:10CF200007224144404209183A400B0200D4D5E69A
:10CF3000434B01351940C9E5380069E61E004746F4
:10CF4000203EF740BC46202B04D04026F31A46462C
:10CF50009E403243170063467A1E97411F4302E604
:10CF6000364DAE42CAD080252D045B422943A6E748
:10CF70000843411E8841A6E6002B00D148E6871AE7
:10CF80004346B842B641CB1A76429E1B33024BD57C
:10CF9000171A4346BA429241591A5242891A072235
:10CFA00064463A4092E501430F00791E8F419DE7A8
:10CFB0001C000F00203CE740202B03D04024E31A44
:10CFC00099400843411E884138437CE600220024F2
:10CFD00025E6171A4346BA429241591A5242891A13
:10CFE0006446350043E541461000144D10E68022AA
:10CFF0000024120380E61D000F00203DEF40BC46D8
:10D00000202B03D04025EB1A9940084307006346C4
:10D01000781E87411F4369E7871897429B41414427
:10D020005B42C9183500A3E53B003343CED007224D
:10D0300031003A4052E600231A00F4E5FF070000F1
:10D04000FFFF7FFFF0B55746DE464E464546E0B54A
:10D05000834607000E03480085B092461C00360B3D
:10D06000400DCD0F002800D19DE0954B984239D05E
:10D070008023F6001B041E43924A7B0F33439946DC
:10D08000944603006344009300230026FF000293AC
:10D0900023031B0B98466300E40F52465B0D01947B
:10D0A00000D1B3E086498B4200D19EE04246D100D8
:10D0B000802212040A435146490F11438B4681498D
:10D0C00052468C4600996344CB1A0021D20000934B
:10D0D0002B0063409A460F2E00D905E17A4BB6002B
:10D0E0009B599F465B463343994600D0B8E00223E4
:10D0F0000826002700900293CAE7CB463A0002991F
:10D100000195019B9A46022927D0032900D180E28C
:10D11000012944D06D49009B8C4663441C00002CBF
:10D1200038DD530700D013E2D2085B46DB0109D596
:10D130005946674B19408B468021C9008C46009B9D
:10D1400063441C00634B9C4207DC5B4664055F073D
:10D150005B0217431B0B620D02E000230027584AB5
:10D1600000211B031C0B0B0D1B05234314055A4AFE
:10D17000380013401C4353466400DB0764081C431B
:10D18000210005B03CBC90469946A246AB46F0BD96
:10D190000122524201231B1B382B00DCADE100228F
:10D1A00000230027DCE75B46334399465ED0002E20
:10D1B00000D18AE1300001F0E7F903000B3B1C2BA2
:10D1C00000DD7BE11D22D31A5A460100DA400839FE
:10D1D0008E4013005F46334399468F403F4B0026F5
:10D1E0001B1A00930023029352E7414653460B4318
:10D1F0003B499B468C46009B634400935B46002B57
:10D200003BD1022300221E43022161E74346134320
:10D210009B4637D04346002B00D162E1404601F0E7
:10D22000B3F903000B3B1C2B00DD53E10200414628
:10D23000083A914088461D21CB1A5146D9400B002F
:10D2400041460B439B46534693401A00009B254999
:10D250009C46604403008C4663440093002137E7FA
:10D260000323B14600900C26029311E7002300939C
:10D2700001330426002702930AE70323C3461E4313
:10D28000032125E701331E430022012120E700236B
:10D290009A46802300271B03094A61E780234946F9
:10D2A0001B03194200D1E2E05946194200D0DEE0EA
:10D2B0000B431B0317001B0BA246014A50E7C04655
:10D2C000FF07000001FCFFFFD81B0100FF03000067
:10D2D000FFFFFFFEFE070000FFFF0F800DFCFFFFBA
:10D2E00001F8FFFFF3030000D94500D9CBE000D1DE
:10D2F000C6E03C0048460027009B013B00935B468C
:10D30000160E1B021E431302984633041B0C99464B
:10D31000310C0191FFF758F84A4642430B04210CA7
:10D32000050019438A4207D98919013D8E4203D865
:10D330008A4201D9851E8919881A0199FFF744F894
:10D3400009048C464A46210464464243090C030002
:10D3500021438A4204D98919013B8E4200D8F1E069
:10D360002D041D43AB464346891A4246280C12043D
:10D370001D0C5B46140C22001B041B0C5A43039427
:10D380006B434443029568431B19150CEB189C42F0
:10D3900003D980246402A44660441C0C15041B04B9
:10D3A0002D0C20185D19814277D373D00C1AA24A34
:10D3B0007D1BAF42BF419446009B7F426344E01B0C
:10D3C0001C00864200D1DBE00199FEF7FDFF4A46D2
:10D3D00042430B04290C070019438A4207D98919D3
:10D3E000013F8E4203D88A4201D9871E8919881AC3
:10D3F0000199FEF7E9FF09044A46894629044D468A
:10D400004243090C030029438A4207D98919013B89
:10D410008E4203D88A4201D9831E89193F04891A92
:10D420003A00039F1A43380013041B0C58438146EB
:10D430000298150C6F43434345434846000C84460D
:10D44000DB1963449F4203D980204002844665442F
:10D4500048461F0C00041B04000C7D191818A94233
:10D4600000D284E000D17FE001231A4357E68023F5
:10D470004A461B0313431B031B0BAA466F4A6FE666
:10D48000BA4200D935E74B46DC0758087B081C43F5
:10D49000FF0734E70024AF4289D247444745A441FF
:10D4A0005B466442A4196418013BA6421ED2A04206
:10D4B0006DD800D1B6E0241A9B4678E703005A469F
:10D4C000283B9A400027914688E6584601F05CF8D0
:10D4D000203072E603005246283B9A4093460022D1
:10D4E000B4E6504601F050F820309AE6A642E2D168
:10D4F000B845DCD9341A9B4659E71F2B65DC504CE4
:10D500000099A4465C46614408008C4011008240AA
:10D51000D940501E82410C4314435A46DA4013004E
:10D52000620709D00F222240042A05D02200141DD0
:10D530009442894149425B181A0262D501220023B4
:10D5400000270DE68A4200D80AE7831E891907E7FB
:10D550000F231340042B00D1E6E5171D974292419B
:10D5600053429B44FA08E0E5002800D1D7E5711842
:10D57000531EB14227D3A94215D358D01A0073E7DE
:10D58000002B00DC04E6012300229B44CDE50223AE
:10D590004744474589415B429C46494289190C19D9
:10D5A000E344241A03E743465F0047459B41B846DE
:10D5B0005B429E19023A8919A94200D054E74045BE
:10D5C00000D051E7ABE51A00F6E71F215F4649425C
:10D5D0000C1BE740202B07D01A49009B8C46634464
:10D5E00018005B4683401A43501E82413A43072786
:10D5F0000023174009D00F210023114014000429F3
:10D6000095D122005F075B021B0BD2081743002253
:10D61000A6E5802359461B030B431B0317001B0B76
:10D62000064A9DE5BD42B2D89B460024BFE6804530
:10D63000B9D31A00C3E7C046FF030000FF0700008C
:10D640001E0400003E040000F0B54F464646D64694
:10D650008446C0B58046194E18030F034D00000BD9
:10D660005C0082463F0B6D0DC90F9146640DDB0FC8
:10D670000120B5420AD0B44203D0A54201D157459A
:10D680000CD01CBC90469946A246F0BD66463E436F
:10D69000F7D1AC42F5D154461443F2D10120C8452C
:10D6A000EFD1994207D0002DEBD163461F433800DC
:10D6B000471EB841E5E70020E3E7C046FF0700004A
:10D6C000F0B54F464646D6464D00C0B50E03C90FCD
:10D6D0008A462C491F035C008046360B6D0D91462F
:10D6E0003F0B640DDB0F8D421ED08C4216D0002DF7
:10D6F0001ED130438446002C01D13A4323D06246E8
:10D70000002A1AD09A4529D05146022001390840F2
:10D7100001381CBC90469946A246F0BD3900114321
:10D72000E5D002204042F4E73043FAD1AC420FD0BA
:10D73000002C0FD13A43E7D00CE00122013B934388
:10D7400018000130E5E763460020002BE1D0DBE75D
:10D750003A43E6D19A45D7D1A542D5DCA54205DBAF
:10D76000BE42D1D808D00020BE42D2D250460123BA
:10D77000013898430130CCE7C845C5D80020C845DA
:10D78000F4D3C6E7FF070000F0B54F464646D6463D
:10D790004D00C0B50E03C90F8A462E491F035C0019
:10D7A0008046360B6D0D91463F0B640DDB0F8D42AD
:10D7B00018D08C4211D0002D18D130438446002C53
:10D7C0001ED13A431CD163460020002B30D0514675
:10D7D00002200139084001382AE039001143EAD01B
:10D7E000022025E03043FBD1AC4226D0002C26D1CC
:10D7F0003A4324D15146022001390840013817E04C
:10D800006246002A0FD09A45E1D1A54205DBBE420F
:10D81000DDD819D00020BE420AD25046012301387B
:10D820009843013004E00122013B9343180001308A
:10D830001CBC90469946A246F0BD3A43D0D19A45C9
:10D84000C5D1A542C3DCE0E7C845C0D80020C84523
:10D85000E3D3EDE7FF070000F0B55746DE464E463E
:10D860004546E0B5834606000F03480087B0924660
:10D870001D003F0B400DCC0F002800D16FE0DE4BA8
:10D88000984238D08023FF001B041F43730F3B4393
:10D890000193DA4B0027994600239B46F60081440A
:10D8A0002B0369001B0B52469846490DED0F0029CA
:10D8B00000D185E0D04B994200D173E04346DA00B5
:10D8C00080231B0413435246CC48520F8446134313
:10D8D000524600206144D2008944210069400091F1
:10D8E0008C46012149448A460F2F00D990E0C44953
:10D8F000BF00CF59BF465B463B43019300D06AE16E
:10D9000002230827002681469B46C9E73200584675
:10D91000019B61460091022800D175E0032800D1E7
:10D92000FEE1012800D02CE100230027002600257D
:10D930003F032A0D3F0BB34812053A4302401B0533
:10D940001343009A5B00D1075B080B4330001900BA
:10D9500007B03CBC90469946A246AB46F0BD5B463C
:10D960003B43019300D12FE1002F00D1A5E1380006
:10D9700000F00AFE03000B3B1C2B00DD96E11D228C
:10D98000D31A5A460100DA405E4608398F40130028
:10D990008E403B4301939C4B00271B1A9946002362
:10D9A0009B467DE7414653460B4393498C46E144F1
:10D9B000002B00D01AE102220220174300228CE73C
:10D9C000134300D10DE14346002B00D181E14046D5
:10D9D00000F0DAFD02000B3A1C2A00DD72E10100C2
:10D9E000434608398B4098461D239A1A5346D34024
:10D9F0001A004346134352468A404946081A824950
:10DA000089468144002068E77B4B002700268EE78B
:10DA1000140C1204120C1100370C3604350C794327
:10DA200028008C462E006043604483465643210004
:10DA3000300C80465846794340440291844506D9CB
:10DA40008846802149028C46E044414602913604D2
:10DA5000010C360C00048B4681191E0C1B041B0C98
:10DA60000391190079438C46280075436544A84604
:10DA70005843050C45447743A94203D98021490204
:10DA80008C466744290C8C4639000004000C2D0498
:10DA90002D186144AB4405915946049101990F0436
:10DAA0003F0C080C390051434243904602008C461B
:10DAB000090C8B4662437C4344445C44A04503D933
:10DAC0008021490288464244210C88466146090467
:10DAD000090C8C4639005943434370437E430F0C75
:10DAE000F6182404BE19644442448C46B34203D958
:10DAF00080235B0298464044029B61469846049B03
:10DB0000370443449B46AB45AD416B420D04059938
:10DB10002D0C8C467F196744FD18A8465D462D19CB
:10DB2000A542A44193466442A446C344DC448F42C8
:10DB3000BF4198459B4193459241A445A4415B4216
:10DB40007F421F43360C52426442BF192243BF1822
:10DB5000624638184302D20D039913436A020A43FE
:10DB6000501E82416146ED0D2A434E023243D901D7
:10DB700000D4B3E00126500832400243DE073243AE
:10DB80005B08224C5444002C62DD510709D00F2061
:10DB90001040042805D0101D9042924152429B181B
:10DBA0000200D90104D580241948E40003405444FC
:10DBB0001848844200DD27E75E075B02D2081F0B8E
:10DBC000630516435B0DB2E6002399460133042733
:10DBD00000269B4664E60323019781460C279B465B
:10DBE0005EE6012201201743002276E6032303208C
:10DBF0001F43434671E6C046FF07000001FCFFFFDC
:10DC0000181C0100FFFF0F800DFCFFFFFF03000049
:10DC1000FFFFFFFEFE0700000023802700933F0365
:10DC20000026434B83E6019B3200A446584670E62B
:10DC3000AC466EE6802701993F0339422DD03B4226
:10DC40002BD11F433F033F0B00951600384B6EE668
:10DC500001252D1B382D00DD66E61F2D40DC3548E3
:10DC60001C005044160082408440EE40501E824109
:10DC700034431443EB40620709D00F222240042AA8
:10DC800005D02200141D9442804140421B181A0204
:10DC90003ED501230027002649E68027019B3F034C
:10DCA0001F433F033F0B0094214B40E603005A46BD
:10DCB000283B9A40002601926DE6584600F064FC2D
:10DCC000203057E603005246283B9A4013000022BA
:10DCD00093E6504600F058FC20307BE6CA4650E7F9
:10DCE0001F201E004042041BE640202D03D0124C92
:10DCF0005444A3401A43501E824132430726002752
:10DD0000164009D00F200023104014000428B9D178
:10DD100022005E075B021F0BD2081643002306E6B3
:10DD200080273F031F433F033F0B1600004BFEE5D8
:10DD3000FF0700001E0400003E040000F8B557462F
:10DD40004E464546DE460C000903E0B5490A460F3B
:10DD50005F0031431E03DB0F760A9B46530F3343AC
:10DD6000C84E6500C000E40FD2006D0DA24681468A
:10DD70007F0D9C469046B74200D1B9E05B46012634
:10DD800073409B46EE1BA34500D183E0002E63DD6C
:10DD9000002F00D0B1E06346134300D123E1731E8E
:10DDA000002B00D0BAE1861A6346B04280410125BB
:10DDB000C91A4042091A0B0200D447E149024B0A32
:10DDC00098464346002B00D189E1404600F0DCFB39
:10DDD0000300083B1F2B00DD7CE120223000D21A1B
:10DDE0004146D040994002009E400A439D4200DDDA
:10DDF0006AE15D1B6B1C1F2B00DD94E120211000EC
:10DE00003500C91A8E40DA408840DD40711E8E41CF
:10DE1000110007222843002506433240002A09D07A
:10DE20000F233340042B05D0331DB342B641764255
:10DE300089191E000B0200D43DE26A1C914B550566
:10DE40006D0D9A4200D119E18F4AF6080A40570732
:10DE500052023743120B9BE0002E00D0C5E06E1C2F
:10DE60007605760D012E00DC48E16746861ACB1B4D
:10DE7000B042BF417F42B8461F004346FF1A3B00F5
:10DE8000B8461B0200D55FE137439AD10022002437
:10DE9000002579E0002E00DCFAE0002F00D18DE0B3
:10DEA000784B9D4267D0802367461B041F43BC46C6
:10DEB000382E00DC52E1634613435A1E93411E186C
:10DEC00086428041404209180B0200D4BEE06D4BEF
:10DED00001359D4200D1D2E06B4A73080A4001210E
:10DEE0000E401E435108D30707221E43324095E7D8
:10DEF0001E00164300D045E740E7624B9D423AD0F2
:10DF0000802367461B041F43BC46382E00DDEBE030
:10DF10001F2E00DC3AE133006746203BDF403B0028
:10DF2000202E05D04027BF1B6646BE403243904698
:10DF30004646721E96413343DAE0002B00D114E2CC
:10DF40006346134300D168E180234E07C008C90827
:10DF50001B030643194208D06046C008184204D18A
:10DF600063460100D2085E071643F3009946C900D4
:10DF7000720F444D11434B46DE08424B4F07374367
:10DF8000CA089D4200D16EE012036D05120B6D0DA3
:10DF900000211203130B0A0D12051A433B4B2D05EA
:10DFA00013402B435B00E4075B0823433800190050
:10DFB0003CBC90469946A246AB46F8BD6346134327
:10DFC00011D0731E002B00D007E1861886428041D5
:10DFD00061444042091801250B0237D502257BE731
:10DFE0003E00614691463500C5E75C46002D00D0F5
:10DFF000E1E00B000343F3D0731C00D1ACE1214BF3
:10E000009F4200D13AE1F343382B00DD6FE11F2B33
:10E0100000DD8CE120250E00ED1AAE40B046060072
:10E02000AA46DE40454635432E005546D940A84015
:10E030006346451EA8415B1A9C463043161AB242FD
:10E04000924163465242991A3D00B4E6072232409B
:10E05000002A00D0E4E60B4BF6084F073743CA0806
:10E060009D4200D090E73B00134300D1A6E18023FE
:10E070001B031A431203120B024D89E715000022FD
:10E08000002785E7FF070000FFFF7FFFFFFF0F80EE
:10E09000002E00D0C7E06B1C5E05760D012E00DC63
:10E0A000F0E0C84DAB4200D1B9E085180A008542C6
:10E0B00089416244494251180722CE076D082E4318
:10E0C000490832401D00A9E6BF49ED1A1140072258
:10E0D0003240A3E6320028388240002686E630002F
:10E0E00000F052FA203073E6634613435A1E934100
:10E0F000C61AB04280414042091A5CE60E006746EB
:10E1000006431743002D5ED1002E00D0F3E0002F10
:10E1100000D11EE15C46614691462CE7A94FBE4204
:10E120007BD01E00F1E610001F3DE840202B03D0FD
:10E130004021CB1A9A401643731E9E410722064384
:10E1400032400021002583E7161A6346B24280411F
:10E15000591A40420B1A98465C4632E61F2E00DDE3
:10E16000ABE02027BB1B9A4663465746BB40994607
:10E1700013004F46F3401F433B005746BA40571E1B
:10E18000BA4113436246F240891898E62027BB1B28
:10E190009A4663465746BB40994613004F46F340A4
:10E1A0001F433B005746BA40571EBA4113436246CD
:10E1B000F240891A9CE7834B9F425FD080252D0453
:10E1C0007342294320E7002E0CD1002F00D1D0E06C
:10E1D0005C46614691467B4DCDE67A4FBE421CD0EF
:10E1E0001E0065E6002F18D0C0084E0706438020A9
:10E1F000C9080003014208D06346DC08044204D188
:10E200002100DA46D2085E071643F300994601243E
:10E210005346C900720F11431C406A4DABE61D0006
:10E2200000220027B4E6002D59D10B00034300D192
:10E23000D6E6731C00D1B2E0624B9F421ED0F3437E
:10E24000382B6FDC1F2B00DD97E020250E00ED1A28
:10E25000AE40B0460600AA46DE40454635432E0095
:10E260005546A840D940451EA8418C440643B618DF
:10E2700096429241514261443D0025E63D0061468F
:10E28000914678E60B000343002D00D055E6002BA5
:10E29000F5D06346134300D16DE68618864280416F
:10E2A00061444042091800220B0200D4D0E6464BDC
:10E2B00001351940B2E5B1465DE633006746203BC3
:10E2C000DF403B00202E05D04027BF1B6646BE40E6
:10E2D000324390464646721E96413343EFE5394B32
:10E2E0009F42CBD080252D0473422943A8E70843E1
:10E2F000411E8841A2E6002F00D13CE66346861A03
:10E30000CF1AB0429B415B42FB1A98461B024ED586
:10E31000161A6346B2429241591A5242891A5C4611
:10E3200000227BE501430E00711E8E419FE71D0018
:10E330000E00203DEE40B046202B04D04025EB1AC5
:10E3400099400843814648464346411E8841184348
:10E3500074E60022002417E6161A6346B242924180
:10E36000591A5242891A3D0025E561469146154DDC
:10E3700001E680220024120379E61D000E00203DF4
:10E38000EE40B046202B04D04025EB1A99400843BC
:10E3900081464E464346711E8E411E4367E78618EE
:10E3A00096429B4161445B42C9183D008CE547465B
:10E3B0003743CED007224146324049E600273A0093
:10E3C000E6E5C046FF070000FFFF7FFF70B50C4E7B
:10E3D0000D031C0349005B002D0B490D240B5B0D45
:10E3E000B14208D0064900208B4203D114432000DB
:10E3F000441EA04170BD05430120002DFAD1F1E774
:10E40000FF07000030B5144D0A034B00120B5B0DE3
:10E41000C90F0024AB4211DD104CA34210DC802454
:10E42000640322430E4CE41A1F2C0CDD0D48C31A62
:10E43000DA4013005C42002900D11C00200030BDEE
:10E44000094BCC18FAE7094DE040AC4663449A40CA
:10E4500013000343EEE7C046FE0300001D04000066
:10E460003304000013040000FFFFFF7FEDFBFFFFFC
:10E4700070B500282DD0C317C5185D40C40F280003
:10E4800000F082F8154B1B1A5B055B0D0A2815DDA1
:10E490000B38854000222D032D0B002110002D0389
:10E4A0000A0D2D0B12052A430D4D1B052A4013435F
:10E4B0005B00E4075B082343190070BD02002900DC
:10E4C000153291400A000B21081AC5402D032D0B6F
:10E4D000E3E70024002300250022DEE71E040000FD
:10E4E000FFFF0F804100090E4B1C70B5DBB24602E6
:10E4F000750AC40F012B14DDE0239B006D07360B5A
:10E50000CB1800210A0D280012051C4D32435B0573
:10E510002A405B0813435B00E4075B0823431900B0
:10E5200070BD002914D1002D1ED0280000F02CF859
:10E530000A281CDC0B232A001B1ADA4003001533BF
:10E540009D400F4B12031B1A5B05160B5B0DD8E7A2
:10E55000002D06D0320B802636036D071643094B7B
:10E56000CFE7084B0026CCE700230026C9E70300CD
:10E570002A000B3B9A400025E3E7C046FFFF0F80CF
:10E5800089030000FF0700001C2101231B0498429F
:10E5900001D3000C10391B0A984201D3000A083934
:10E5A0001B09984201D30009043902A2105C4018EB
:10E5B0007047C0460403020201010101000000008F
:10E5C00000000000F0B54E465746DE464546E0B531
:10E5D0000F00002183B006008946002F06DA3900BB
:10E5E000002746428F41012149428946002B07DA24
:10E5F0004946C943100089461900002342428B4115
:10E6000034003D0092469846BB4269D866D04146E8
:10E61000504600F0AFF883463900300000F0AAF809
:10E620005B461B1A9C46203B9B4600D575E0514635
:10E63000584681400B005146604681400A00BB426B
:10E6400061D85ED034003D005946A41A9D4100298E
:10E6500000DA7AE00021002001260090019159465D
:10E660008E400196614601268E4061460096002943
:10E6700050D0D90756085F080E4363460EE0AF42FC
:10E6800001D1A6420CD8A41BBD41012124196D4122
:10E690000022013B64185541002B06D0AF42EED951
:10E6A000013B24196D41002BF8D1009801995B467C
:10E6B00000196941002B3DDB2E00DE4063462C0033
:10E6C000DC405B46002B4BDB34005D46AC40230056
:10E6D0006446A6403200801A994103E0B24296D9BE
:10E6E000002000214B46002B04D003000C00002129
:10E6F0005842A14103B03CBC90469946A246AB4665
:10E70000F0BDB1429ED900210020009001916146E8
:10E710000029AED100980199E4E7202362465146D2
:10E720009B1AD940404600916146884003000099F9
:10E730000B4380E7624620239B1A2A009A4026005A
:10E7400013006246D6401E43B8E7614620260127E3
:10E75000761A00200021F74000900191019781E78F
:10E760006746202362463500BC409B1ADD402300EB
:10E770002B43ADE710B5002903D1FFF705FF20308B
:10E7800002E0081CFFF700FF10BDC04630B51C00BA
:10E79000094B05001B6885B0D868084B002A01D1D9
:10E7A000074B1A000292019300912B0022000549A9
:10E7B00000F026F800F0A6FDA0000020581C010083
:10E7C000CF050100651C0100014B18687047C04669
:10E7D000A0000020084B10B50400002B02D000213F
:10E7E00000E000BF054B1868836A002B00D09847F3
:10E7F000200001F05DFBC04600000000941C0100F9
:10E800000EB403B5010003AB044804CB00680193C8
:10E8100000F076F802B008BC03B01847A000002052
:10E8200070B500260C4D0D4C641BA410A64209D1F6
:10E83000002601F03FFB0A4D0A4C641BA410A642BF
:10E8400005D170BDB300EB5898470136EEE7B30031
:10E85000EB5898470136F2E7700200207002002062
:10E860007002002080020020002310B59A4200D1DF
:10E8700010BDCC5CC4540133F8E710B5884202D90E
:10E880008B18984203D3002307E08B5C8354013A32
:10E89000FBD210BDCC5CC45401339A42FAD1F8E7E4
:10E8A00003001218934200D1704719700133F9E741
:10E8B000936810B5013B9360002B04DA9469A3427E
:10E8C00007DB0A2905D01368581C1060197008006E
:10E8D00010BD00F04BFC0100F9E7F8B506000F0091
:10E8E0001400D518AC4201D1002007E021783A008D
:10E8F0003000FFF7DDFF0134431CF3D1F8BD000009
:10E90000F0B59FB002900F0016000593002805D0C7
:10E9100083690493002B01D100F0F4FD7B4B9F42EF
:10E920005BD1029B5F68BB891B0762D53B69002BEB
:10E930005FD0002306AC6361203363761033A37687
:10E9400035002B78002B01D0252B5CD1AB1B049319
:10E950000CD0320039000298FFF7BFFF431C00D1F2
:10E96000C4E06269049B9446634463612B78002B86
:10E9700000D1BBE0012200235242626002A954325E
:10E9800052186E1C2360E360A3601370A365317896
:10E9900005225F4800F0D4FE751C002835D122689E
:10E9A000D30604D5532302A95B182021197013073D
:10E9B00004D5532302A95B182B21197033782A2B15
:10E9C0002CD0350000210A20E3682A786E1C303AEA
:10E9D000092A64D900292ED026E04E4B9F4202D14D
:10E9E000029B9F689FE74C4B9F429CD1029BDF6834
:10E9F00099E73900029800F00FFC002899D0012017
:10EA000040421FB0F0BD01359BE7414B2268C01A60
:10EA100001238340134323602E00B8E7059B191D93
:10EA20001B680591002B01DB099304E05B42E36066
:10EA30000223134323602B782E2B0AD16B782A2BC9
:10EA400035D1059B02351A1D1B680592002B2BDB67
:10EA50000793324E29780322300000F071FE00281F
:10EA600006D04023801B8340226801351343236076
:10EA7000297806222A486E1C217600F061FE0028C3
:10EA80003AD0284B002B25D10722059B073393430F
:10EA9000083305936369039A9B18636150E7434306
:10EAA00001219B18350090E701235B42D0E700234A
:10EAB0000A201A000135636029786E1C3039092953
:10EAC00003D9002BC5D00792C3E742430123521854
:10EAD0003500F1E705AB00933A00134B2100029893
:10EAE00000E000BF0390039B0133D3D1BB895B06D9
:10EAF00000D584E70B9884E705AB00933A000A4BF6
:10EB00002100029800F080F8ECE7C046EC1C010000
:10EB1000981C01000C1D0100CC1C01009E1C010072
:10EB2000A21C010000000000DBE80000F7B51500A2
:10EB300001938A680B6900900C00934200DA13007D
:10EB400022002B6043321278002A01D001332B605F
:10EB500023689B0602D52B6802332B6006272368A7
:10EB60001F4027D0230043331B785A1E934122684D
:10EB7000920630D42200019943320098089EB04793
:10EB8000431C25D0062320682A68E168034000253D
:10EB9000042B03D18D1AEB43DB171D40A3682269B8
:10EBA000934201DD9B1AED180027BD4220D10020C1
:10EBB00010E00137E3682A689B1ABB42D2DD2200CD
:10EBC0000123193201990098089EB047431CF0D1E7
:10EBD00001204042FEBD3020E11843310870210081
:10EBE0005A1C45310978A218433202331170C1E72B
:10EBF000220001231A3201990098089EB047431C55
:10EC0000E6D00137D1E70000F0B589B004920A00E0
:10EC100043320593039002920A7E0C000E9B6E2AEB
:10EC200000D186E01FD8632A33D008D8002A00D14B
:10EC30008CE0582A4DD0250042352A7030E0642AF5
:10EC400001D0692AF7D1196825680A1D280629D537
:10EC500008681A60002803DA2D23029A40421370D4
:10EC60006B4E0A274FE0732A74D008D86F2A1FD042
:10EC7000702AE0D1202209680A43226003E0752A45
:10EC800016D0782AD7D12200782145321170614EF2
:10EC900022E025001A684235111D196013682B7097
:10ECA000012365E008681A606906D3D500B2D1E790
:10ECB00019682568081D186008682E0605D5544E89
:10ECC00008276F2A1BD00A2719E06D06F7D580B2F6
:10ECD000F5E745314E4E0A7018682268011D00683C
:10ECE0001960150621D5D30702D520231A432260C7
:10ECF0001027002803D1202322689A432260230092
:10ED0000002243331A706368A360002B58DB04228F
:10ED1000216891432160002854D1029D002B5AD0D4
:10ED20002500337842352B7055E05506DBD580B28F
:10ED3000D9E71A680D68101D4969186013682E0616
:10ED400001D5196002E06D06FBD519800023029DF4
:10ED500023614FE01A68111D19601568002162686F
:10ED6000280000F0EDFC002801D0401B60606368C3
:10ED700023610023029A13703CE023692A0004995E
:10ED80000398059DA847431C3ED023689B0715D4D4
:10ED9000079BE068984239DA180037E02200012327
:10EDA000193204990398059EB047431C2CD00135B5
:10EDB000E368079A9B1AAB42F0DCE9E70025F7E726
:10EDC0000028ADD0029D3900FDF7FEFA735C013DCD
:10EDD0002B700028F7D1082F09D12368DB0706D54F
:10EDE00063682269934202DC3023013D2B70029B51
:10EDF0005B1B2361059B07AA00932100049B0398DA
:10EE0000FFF794FE431CB8D10120404209B0F0BD89
:10EE1000A91C0100BA1C01000D4B70B51C6805004F
:10EE2000A36B002B0FD1182000F06EFC094BA063E0
:10EE30000360094B01224360084B83600B238381ED
:10EE40000023026143610022A36B1D615A6170BD02
:10EE5000A00000200E33CDAB34126DE6ECDE0500D1
:10EE6000124B10B51C68A36B002B0FD1182000F0BB
:10EE70004BFC0F4BA06303600E4B012243600E4B13
:10EE800083600B238381002302614361A46B0B4ADF
:10EE9000206961690A4BFDF7F7FB01220023801806
:10EEA0005941206161614800400810BDA000002068
:10EEB0000E33CDAB34126DE6ECDE05002D7F954CA4
:10EEC0002DF451580CB430B5164B9DB00C1E1D6876
:10EED00008DA8B2301202B6040421DB030BC08BCF7
:10EEE00002B01847822302A99B008B810023029065
:10EEF00008619C4200D0631E8B604B6101235B4222
:10EF0000CB81209A21AB2800019300F055FD431CD2
:10EF100001DA8B232B60002CDFD00023029A1370C0
:10EF2000DBE7C046A00000200EB400B50B499CB042
:10EF30001DAB02900690079104910948094904CB42
:10EF40000591006802A9019300F036FD0023029AA2
:10EF500013701CB008BC03B01847C046FFFFFF7F0A
:10EF6000A00000200802FFFF020010B51378541C17
:10EF7000002B05D1CC5CD4540133002CFAD110BD48
:10EF80002200F3E7C9B20378002B04D08B4200D1F2
:10EF900070470130F7E74B42594149420840F7E7D3
:10EFA00002780B78002A03D0013001319A42F7D061
:10EFB000D01A70470023C25C0133002AFBD1581ECF
:10EFC0007047002330B59A420AD0013AC45CCD5C48
:10EFD000AC4204D1934202D00133002CF6D1631B22
:10EFE000180030BD30B50500002A00D130BD0C78C6
:10EFF000013A6B1C2C700131002C05D19A189A42F1
:10F00000F4D01C700133FAE71D00EDE710B503786A
:10F01000002B0FD10B785A4253415B42184010BD70
:10F020000023CA5C002AFAD0C45C944201D10133A7
:10F03000F7E701300378002BF2D11800EFE700006A
:10F04000F0B51F000E0087B00590019102920C9858
:10F05000347800F0EAFA082200194378751C13404E
:10F0600036D12D2C36D1B51C74780126002F62D0F4
:10F07000102F09D1302C07D120222B789343582B05
:10F0800054D110276C7802352D4B3900F318180035
:10F090000393FDF799F904910121002349420200ED
:10F0A0008C4618002100303909291AD80C00A742D3
:10F0B00023DD591C09D06346824206D302D104994C
:10F0C000A14202DB0123784320182C780135E9E7BF
:10F0D0002E00BCE72B2C01D01E00C7E7B51C7478AE
:10F0E000FAE721004139192901D8373CDFE721002F
:10F0F0006139192901D8573CD9E75A1C08D1059A1A
:10F1000023331360029B0398002B09D107B0F0BD95
:10F11000002E00D04042029A002AF7D0002B01D0E6
:10F120006B1E0193029B019A1A60EFE73024002FB7
:10F13000AAD10827A8E7302C9ED00A27A4E7C0460A
:10F14000FFFFFF7F37B51300064A05001068046A09
:10F15000002C00D1044C0A0000942900FFF770FF36
:10F160003EBDC046A000002004010020F8B5050007
:10F170000E001400002804D08369002B01D100F098
:10F18000C1F9224B9C422DD16C68A369A360A3896D
:10F190001B0731D52369002B2ED023682269F7B2D3
:10F1A000981A6369F6B2834205DC2100280000F05A
:10F1B0003BF9002826D1A3680130013BA3602368F6
:10F1C0005A1C22601F706369834204D0A389DB0745
:10F1D0001AD50A2E18D12100280000F025F90028A0
:10F1E00012D00FE00A4B9C4201D1AC68CDE7094B2D
:10F1F0009C42CAD1EC68C8E72100280000F00CF856
:10F200000028CAD0012676423000F8BDEC1C01006F
:10F210000C1D0100CC1C0100364B70B51D680600AA
:10F220000C00002D05D0AB69002B02D1280000F0A6
:10F2300069F9314B9C420FD16C680C23E25E93B2AA
:10F2400019072DD4D90611D409230120336037338F
:10F250001343A381404270BD284B9C4201D1AC684E
:10F26000EBE7274B9C42E8D1EC68E6E75B0713D558
:10F27000616B002908D023004433994202D030004A
:10F2800000F06AFA002363632422A3899343A381D5
:10F2900000236360236923600823A2891343A381A9
:10F2A0002369002B0BD1A0218022A3898900920021
:10F2B0000B40934203D02100300000F0E1F901231C
:10F2C000A289134011D00023A36063695B42A3614C
:10F2D000002023698342BED10C23E25E1306BAD517
:10F2E00040231343A3810138B5E7920700D4636933
:10F2F000A360EDE7A0000020EC1C01000C1D010044
:10F30000CC1C010010B5062000F090FC012000F09C
:10F31000CFFD0000F7B58A8905000C00130760D403
:10F320004B68002B04DC0B6C002B01DC0020FEBDC5
:10F33000E76A002FFAD000232E682B6080235B0140
:10F34000216A1A4034D0606DA3895B0706D56368D3
:10F35000C01A636B002B01D0236CC01A0200216A13
:10F3600000232800E76AB847A189431C06D12B680F
:10F370001D2B30D82B4ADA40D3072CD500236360ED
:10F3800023692360CB0405D5431C02D12B68002BD5
:10F3900000D16065616B2E600029C7D02300443323
:10F3A000994202D0280000F0D7F900206063BEE740
:10F3B00001232800B847431CC6D12B68002BC3D0BB
:10F3C0001D2B01D0162B01D12E60AFE74023A2895F
:10F3D0001343A381ABE740230B430120A3814042A9
:10F3E000A5E70F69002FA1D00B680F60DB1B01930D
:10F3F0000023920700D14B69A360019B002B00DC26
:10F4000094E7019B3A00216A2800A66AB0470028C9
:10F4100003DC4023A2891343DFE7019B3F181B1A3B
:10F420000193EAE7010040200B6970B505000C006C
:10F43000002B01D1002070BD002804D08369002B6F
:10F4400001D100F05FF80B4B9C4209D16C680C2293
:10F45000A35E002BEED021002800FFF75BFFEAE758
:10F46000054B9C4201D1AC68F1E7044B9C42EED1C4
:10F47000EC68ECE7EC1C01000C1D0100CC1C010049
:10F48000002310B5040003604360836081814366FC
:10F49000C281036143618361190008225C30FFF778
:10F4A000FFF9054B24626362044BA362044BE362E1
:10F4B000044B236310BDC0466DFC000095FC0000AA
:10F4C000CDFC0000F9FC000010B5024900F08CF8FA
:10F4D00010BDC04629F4000070B568254A1E55438A
:10F4E0000E002900743100F081F9041E08D00021BB
:10F4F0002A00016046600C30A0606832FFF7D0F946
:10F50000200070BD836913B50400002B28D18364EB
:10F51000C3640365134B144A1B68826201939842CB
:10F5200001D101238361200000F020F860602000F9
:10F5300000F01CF8A060200000F018F80022E06045
:10F5400004216068FFF79CFF01220921A068FFF7F2
:10F5500097FF02221221E068FFF792FF0123A361C7
:10F5600013BDC046941C0100C9F40000F8B51C4B43
:10F5700007001E68B369002B02D13000FFF7C2FFFD
:10F580004836B4687368013B04D53368002B07D054
:10F590003668F6E70C22A55E002D0DD06834F2E740
:10F5A00004213800FFF798FF30600028F0D10C23C9
:10F5B00004003B602000F8BD20000A4B6566256012
:10F5C0006560A560E36025616561A5610822290089
:10F5D0005C30FFF765F96563A563A564E564E9E759
:10F5E000941C01000100FFFFF7B50400070000268E
:10F5F00001914834002C01D13000FEBD6368A5683C
:10F600000093009B013B009301D52468F2E7AB898E
:10F61000012B08D90E22AB5E013304D0290038003B
:10F62000019B984706436835EBE7EC30006870476C
:10F6300070B50E001D000E23C95E96B0140000299F
:10F6400007DA00232B60B3891B0611D48023DB006B
:10F650000FE06A4600F088FB0028F2DBF022019BF5
:10F6600012021340054A9B185A4253412B60EDE7A2
:10F6700040230020236016B070BDC04600E0FFFFAD
:10F68000F7B502268B8905000C00334206D0230013
:10F6900047332360236101236361F7BD01AB6A46F1
:10F6A000FFF7C6FF00990700280000F09FF8002828
:10F6B00008D10C22A35E9A05EFD4032293431E4384
:10F6C000A681E4E70F4BAB628023A289206013433D
:10F6D000A381009B20616361019B002B0DD00E2351
:10F6E000E15E280000F052FB002806D00322A38927
:10F6F00093431A0001231343A381A0893843A081B7
:10F70000CBE7C046C9F4000010B5034B01001868F0
:10F7100000F06CF810BDC046A000002082B00029A7
:10F7200000D101A9101E06D0002B06D013780B6063
:10F730001078431E984102B0704702204042FAE719
:10F74000C9B28218904201D10020704703788B42E1
:10F75000FBD00130F6E7000070B50500002910D09D
:10F760000C1F2368002B00DAE418280000F034FB9B
:10F770001D4A1368002B05D163601460280000F057
:10F780002CFB70BDA34209D9216860188342F3D1D4
:10F7900018685B6841182160EEE713005A68002A78
:10F7A00001D0A242F9D919685818A0420BD120689B
:10F7B0000918581819608242E0D11068526841183F
:10F7C00019605A60DAE7A04202D90C232B60D5E712
:10F7D00021686018824203D1106852684118216084
:10F7E00062605C60CAE7C046081C0020032370B555
:10F7F000CD1C9D43083506000C2D1ED20C25A942B8
:10F800001DD8300000F0E8FA254A146821000029CC
:10F8100019D1244C2368002B03D1300000F0CAF921
:10F8200020602900300000F0C5F9431C2BD10C23C7
:10F830003000336000F0D1FA03E0002DDFDA0C2352
:10F840003360002070BD0B685B1B19D40B2B03D9F0
:10F850000B60CC18256003E04B688C420DD113601F
:10F86000300000F0BAFA200007220B30231D90432D
:10F87000C31AE7D05A42E250E4E763600C00EFE7B6
:10F880000C004968C3E70323C41C9C43A042E1D099
:10F89000211A300000F08EF9431CDBD1C7E7C046C7
:10F8A000081C00200C1C0020F8B507000D001600F5
:10F8B000002905D11100FFF799FF04002000F8BDD1
:10F8C000002A03D1FFF748FF3400F7E700F086FA7B
:10F8D0002C00B042F2D231003800FFF787FF041E3F
:10F8E000ECD029003200FEF7BFFF29003800FFF7F7
:10F8F00033FFE3E7F0B58E6885B007000C00039294
:10F9000001939E423CD890238A89DB001A4234D06E
:10F910000325096923685B1A0293636902985D43B2
:10F92000EB0F5D19019B6D1001331B18AB4200D921
:10F930001D00530532D529003800FFF757FF061E7A
:10F9400009D10C233B6040230120A289404213438C
:10F95000A38105B0F0BD029A2169FEF785FFA38956
:10F96000144A1A4080231343A381029B2661F61890
:10F9700026606561019EED1AA560019B9E4200D93B
:10F98000019E320003992068FEF777FFA3680020EC
:10F990009B1BA36023689E192660DAE72A003800C3
:10F9A000FFF782FF061EE0D121693800FFF7D4FE81
:10F9B000C7E7C0467FFBFFFFF0B59FB002900593FD
:10F9C0008B890F0016001B0611D50B69002B0ED179
:10F9D0004021FFF70BFF38603861002805D10C2368
:10F9E000029A013813601FB0F0BD40237B610023F1
:10F9F00006AC6361203363761033A37635002B7831
:10FA0000002B01D0252B46D1AB1B04930CD0320028
:10FA100039000298FFF76EFF431C00D1AEE0626927
:10FA2000049B9446634463612B78002B00D1A5E0CE
:10FA3000012200235242626002A9543252186E1C05
:10FA40002360E360A3601370A365317805225448F6
:10FA5000FFF776FE751C00281FD12268D30604D557
:10FA6000532302A95B1820211970130704D55323CF
:10FA700002A95B182B21197033782A2B16D0350078
:10FA800000210A20E3682A786E1C303A092A4ED9F0
:10FA9000002918D010E00135B1E7414B2268C01AA7
:10FAA00001238340134323602E00CEE7059B191DDD
:10FAB0001B680591002B01DB099304E05B42E360C6
:10FAC0000223134323602B782E2B0AD16B782A2B29
:10FAD00035D1059B02351A1D1B680592002B2BDBC7
:10FAE0000793304E297803223000FFF729FE0028C3
:10FAF00006D04023801B83402268013513432360D6
:10FB00002978062228486E1C2176FFF719FE002866
:10FB10003CD0264B002B25D10722059B073393436E
:10FB2000083305936369039A9B18636166E743434F
:10FB300001219B183500A6E701235B42D0E7002393
:10FB40000A201A000135636029786E1C30390929B2
:10FB500003D9002BC5D00792C3E7424301235218B3
:10FB60003500F1E705AB00933A00114B21000298F4
:10FB700000E000BF0390039B0133D3D1BB890B98F6
:10FB80005B0600D42FE7012040422CE705AB009331
:10FB90003A00074B21000298FFF736F8EAE7C04623
:10FBA000981C01009E1C0100A21C01000000000026
:10FBB000F5F80000002370B5064C0500080023602E
:10FBC00000F060F9431C03D12368002B00D02B60A8
:10FBD00070BDC046C02F002070B504000D001F2965
:10FBE00004D9162303600120404270BD436C002BF2
:10FBF00004D08A009B181A68002A08D1200000F05F
:10FC000031F82A000100200000F01AF8EDE700208A
:10FC1000012AEAD0511C03D1162301302360E4E706
:10FC2000002428001C6090472000DEE710B5034B3D
:10FC300001001868FFF7D0FF10BDC046A0000020EB
:10FC4000002370B5064C050008001100236000F089
:10FC500001F9431C03D12368002B00D02B6070BD39
:10FC6000C02F002010B500F0E5F810BD70B50C00F5
:10FC70000E25495F00F0BAF8002803DB636D1B18FE
:10FC8000636570BDA389024A1340A381F9E7C046AA
:10FC9000FFEFFFFFF8B51F008B8905000C00160071
:10FCA000DB0505D50E23C95E0022022300F080F893
:10FCB000A389054A28001340A38132000E23E15E88
:10FCC0003B0000F02BF8F8BDFFEFFFFF70B50C0014
:10FCD0000E25495F00F06CF8A389421C03D1054A48
:10FCE0001340A38170BD802252011343A38160653C
:10FCF000F8E7C046FFEFFFFF10B50E23C95E00F026
:10FD000021F810BD0B1E04D0FF2A04D98A230360FA
:10FD10008B3B180070470A700123FAE770B50500A5
:10FD2000080011000022064C22601A0000F0B8F80A
:10FD3000431C03D12368002B00D02B6070BDC0464C
:10FD4000C02F0020002370B5064C0500080023607A
:10FD500000F060F8431C03D12368002B00D02B6017
:10FD600070BDC046C02F0020002370B5064C0500B2
:10FD700008001100236000F055F8431C03D12368EC
:10FD8000002B00D02B6070BDC02F0020002370B569
:10FD9000064C05000800236000F054F8431C03D112
:10FDA0002368002B00D02B6070BDC046C02F002000
:10FDB00070B50500080011000022064C22601A00F0
:10FDC00000F050F8431C03D12368002B00D02B60B7
:10FDD00070BDC046C02F0020704770470B1F1B68C6
:10FDE000181F002B01DA0B58C018704770B50500BA
:10FDF000080011000022064C22601A0000F03AF8B8
:10FE0000431C03D12368002B00D02B6070BDC0467B
:10FE1000C02F002058220120014B40421A60704739
:10FE2000C02F002058220120014B40421A60704729
:10FE3000C02F002058220120014B40421A60704719
:10FE4000C02F00205822024B00201A607047C04685
:10FE5000C02F002058220120014B40421A607047F9
:10FE6000C02F002058220120014B40421A607047E9
:10FE7000C02F002058220120014B40421A607047D9
:10FE8000C02F0020044A1368002B00D1034B181820
:10FE9000106018007047C046101C0020C82F0020BA
:10FEA00058220120014B40421A607047C02F0020A9
:10FEB000FEE7C046F8B5C046F8BC08BC9E46704791
:10FEC000F8B5C046F8BC08BC9E467047F3FE00007B
:10FED00081010000FDFE00008D01000007FF000011
:10FEE000850100000FFF00008901000063616D655E
:10FEF00072610068617343616D6572610074616B6A
:10FF00006550686F746F0073657453697A65007328
:10FF10006574456E636F64696E6700646174610047
:10FF2000D9FF000081020000E2FF00007D0B00000D
:10FF3000E8FF000011030000F0FF0000310C00009A
:10FF4000F7FF00006D0D0000FCFF00003905000008
:10FF500002000100250700000D00010081030000E0
:10FF600012000100C50F00001E000100B1020000D8
:10FF700028000100A90A000036000100C5060000A3
:10FF800043000100B10800004F0001008506000099
:10FF90005A0001005511000072616E646F6D0062BD
:10FFA0006F6F6C65616E006E756D62657200737463
:10FFB00072696E67006C69737400627974652061A0
:10FFC0007272617900616C6C006C61737400310055
:10FFD000252E3135732E2E2E006D616B654C6973A5
:10FFE000740072616E6765006164644C61737400D3
:10FFF00064656C657465006A6F696E0073706C6926
:020000021000EC
:100000007400636F707946726F6D546F0066696E2D
:1000100064006A6F696E537472696E677300756EFF
:1000200069636F6465417400756E69636F646553DD
:100030007472696E67006E65774279746541727299
:100040006179006173427974654172726179006609
:100050007265654D656D6F727900636F6E7665725E
:100060007454797065000000E5000100C5180000B7
:10007000EA000100E3180000F0FF0000E7180000AC
:10008000F0000100C9180000FA000100EB180000A0
:1000900003010100EF1800000D010100F31800003A
:1000A00016010100CD18000023010100F71800001F
:1000B00033010100FB1800003E010100FF180000A1
:1000C0004A0101000319000053010100DB18000080
:1000D0005D010100D118000068010100DF18000077
:1000E00066696C65006F70656E00636C6F736500A8
:1000F000656E644F6646696C6500726561644C6943
:100100006E65007265616442797465730072656141
:1001100064496E746F0072656164506F73697469CD
:100120006F6E0073657452656164506F73697469B2
:100130006F6E00617070656E644C696E6500617011
:1001400070656E6442797465730066696C655369A5
:100150007A650073746172744C697374006E6578AB
:1001600074496E4C6973740073797374656D496E6C
:10017000666F0000B801010023190000C2010100F0
:100180002F190000CD01010033190000DA01010030
:1001900037190000E60101003B190000EF010100E2
:1001A0003F190000F70101002719000002020100B9
:1001B0002B190000686964006D6F7573654D6F766B
:1001C00065006D6F7573655072657373006D6F7543
:1001D000736552656C65617365006D6F757365530A
:1001E00063726F6C6C0070726573734B6579006835
:1001F0006F6C644B65790072656C656173654B6506
:10020000790072656C656173654B657973000000F8
:10021000941D0000A41D0000C81D00002A1E00003F
:100220006A1E0000A41E0000E21E0000121F000053
:10023000601F0000AC1F00000620000068200000C6
:10024000D42000001221000042210000842100007F
:10025000D82100000822000040220000782200007F
:100260003C3D00004E2300003A240000C42400005E
:100270002025000078250000A4250000D2250000DC
:1002800050270000A0270000222800005A28000064
:1002900096280000D228000044290000B62900005A
:1002A0001C2A0000842A0000122B00008E2B000064
:1002B000F42B0000582C0000982C0000E82C0000C3
:1002C000382D0000882D0000E62D00005C2E000077
:1002D000A42E0000382F0000782F0000C82F000047
:1002E0001830000068300000AC300000FC30000026
:1002F0004C310000F2320000402200008421000056
:10030000BE310000941D0000FE3100003C320000B0
:100310007C320000B2320000941D0000941D0000E9
:10032000941D0000941D000076330000C0330000CF
:100330000E340000683400009E34000022350000B6
:100340007C350000B435000018360000941D000014
:1003500092360000CC360000063700004637000019
:100360007A370000BA370000EE370000203800006E
:10037000523800008C380000C6380000FA380000FF
:100380002E390000683900009C390000941D0000DF
:10039000941D0000941D0000941D0000941D000099
:1003A000E43900001A3A0000503A0000863A000092
:1003B000BC3A0000FC3A00003C3B00007C3B0000E3
:1003C000BC3B0000F23B0000283C0000683C000001
:1003D000941D0000941D0000941D0000941D000059
:1003E000941D0000941D0000941D0000941D000049
:1003F000941D0000941D0000941D0000941D000039
:100400009E3C00009E3C0000003E0000363E000086
:1004100066616C73650074727565005B25642069A4
:1004200074656D206C6973745D00282564206279A1
:100430007465732900286F626A656374207479702B
:10044000653A2025642900537461636B20756E64DE
:100450006572666C6F770000070000000300000003
:10046000F10401005D3F0000F90401000D400000AF
:10047000020501009D4400000B050100613F0000E2
:1004800014050100A14400001C050100C941000041
:10049000250501008542000033050100F9400000F8
:1004A0003E0501005146000049050100DD41000004
:1004B00054050100A945000060050100A5400000A9
:1004C0006C050100214600001C0000000100000036
:1004D000020000000400000005000000060000000B
:1004E000100000001100000043616C6C696F7065C2
:1004F00000686173546F6E6500706C6179546F6E43
:100500006500686173536572766F00736574536537
:1005100072766F00646163496E6974006461635749
:100520007269746500736F66745772697465427995
:1005300074650073717561726557617665007365E6
:1005400074557365724C454400616E616C6F6752FF
:1005500065616400616E616C6F67577269746500F4
:100560006469676974616C52656164006469676994
:1005700074616C577269746500474320746F6F6BC8
:100580002025642075736563733B20667265652062
:10059000256420776F726473003C496E74656765EB
:1005A000723E003C4C6973743E003C4F626A656366
:1005B000743E003C4279746541727261793E000D6F
:1005C0000A564D2050616E69633A2025730D0A006A
:1005D000FFFFFF7FFFFFFF7FFFFFFF7FFFFFFF7F2B
:1005E000FFFFFF7FEA51B87EFFFFFF7F21DBF97E2F
:1005F000FFFFFF7FFFFFFF7FC776BE7FF4285C7F92
:10060000FFFFFF7FEA51B87EFFFFFF7FFFFFFF7F05
:10061000000024F40000127A0000093D0080841ECE
:10062000FF583E0F548C93070090D0031038EC0114
:100630009062F40000127A0000093D0080841E00E0
:1006400040420F0020A1070090D0030048E80100BD
:100650006D69736300000000BD060100C550000015
:10066000C6060100BD510000CE0601008151000008
:10067000D206010055510000D7060100E1520000EA
:10068000EA06010015520000FE060100B550000008
:100690000D070100B51C00001C07010009500000F7
:1006A00024070100AF4F00002E070100454F000056
:1006B0003A070100474E00006E756C6C0068657863
:1006C000546F496E740072657363616C6500736981
:1006D0006E00737172740070726573737572655415
:1006E0006F416C74697475646500626D653638308D
:1006F000476173526573697374616E636500636FFC
:100700006E6E6563746564546F4944450062726F30
:10071000616463617374546F494445006A736F6E1A
:10072000476574006A736F6E436F756E74006A7309
:100730006F6E56616C75654174006A736F6E4B65C0
:1007400079417400400801006D5300004808010021
:1007500071530000520801008F5300005B08010034
:100760009953000066080100A353000072080100BD
:10077000AD53000080080100B75300008808010055
:10078000C15300008E080100CB530000A3080100F4
:10079000D5530000B8080100DF530000C408010071
:1007A000E9530000D4080100F3530000E008010001
:1007B000FD530000ED08010007540000F608010099
:1007C00011540000FE0801001B5400000C09010038
:1007D000255400001D0901002F54000030090100BC
:1007E000395400003E090100435400004D09010046
:1007F0004D540000600901005754000076090100C3
:100800006B54000082090100755400009209010038
:100810007F540000A109010089540000AF090100C4
:1008200093540000B709010061540000C30901009E
:100830007B530000CB090100855300006E657400F6
:1008400068617357694669007374617274576946C9
:10085000690073746F7057694669007769666953F8
:100860007461747573006D79495041646472657385
:1008700073007374617274535349447363616E00FF
:1008800067657453534944006D794D414300687462
:1008900074705365727665724765745265717565DB
:1008A000737400726573706F6E64546F4874747003
:1008B000526571756573740068747470436F6E6E01
:1008C00065637400687474704973436F6E6E65631A
:1008D0007465640068747470526571756573740032
:1008E00068747470526573706F6E736500756470B0
:1008F00053746172740075647053746F7000756422
:100900007053656E645061636B65740075647052FA
:100910006563656976655061636B657400756470C5
:1009200052656D6F746549504164647265737300FC
:1009300075647052656D6F7465506F727400776581
:1009400062536F636B657453746172740077656290
:10095000536F636B65744C6173744576656E740098
:10096000776562536F636B657453656E64546F4350
:100970006C69656E74004D515454436F6E6E6563BF
:1009800074004D5154544973436F6E6E65637465C2
:1009900064004D515454446973636F6E6E656374A3
:1009A000004D5154544C6173744576656E74004D1E
:1009B000515454507562004D5154545365745769E5
:1009C0006C6C004D515454537562004D5154545544
:1009D0006E73756200000000260A0100B554000025
:1009E0002B0A0100C9540000350A0100CD54000053
:1009F0003E0A0100D1540000450A0100D554000010
:100A00004F0A0100C1540000590A0100B954000006
:100A1000620A0100BD540000670A0100C5540000CD
:100A2000317769726500696E6974007363616E5332
:100A300074617274007363616E4E657874007365DF
:100A40006C6563740073656C656374416C6C0077EE
:100A50007269746542797465007265616442797483
:100A6000650063726338006372633136000D0E0FE8
:100A700004050C0B0A06070809000000000008081E
:100A80000800080A4A4000000A5FEA5FEA0ED92E11
:100A9000D36E19324489330C924C924D08080000F1
:100AA0000004880808040804848488000A448A40F2
:100AB00000048EC480000000048800000EC0000006
:100AC0000000080001224488100C9252524C048C01
:100AD00084848E1C824C901E1EC244924C06CA52C4
:100AE0005FE21FF01EC13E02448ED12E1FE24488F9
:100AF000100ED12ED12E0ED12EC488000800080071
:100B000000048004880244880482000EC00EC008DD
:100B1000048244880ED126C0040ED135B36C0C92E9
:100B20005ED2521C925C925C0ED010100E1C92523F
:100B3000525C1ED01C901E1ED01C90100ED0137143
:100B40002E12525ED2521C8808081C1FE242524CE0
:100B50001254981492101010101E113B75B13111DF
:100B60003935B3710C9252524C1C925C90100C921D
:100B7000524C861C925C92510ED00C825C1FE48415
:100B80008484125252524C1131312A44113135BBF6
:100B90007112524C9252112A4484841EC488101E31
:100BA0000EC808080E10080482410EC242424E04CC
:100BB0008A400000000000001F0804800000000EB2
:100BC000D2524F10101C925C000ED0100E02424EFA
:100BD000D24E0C925C900E06C81C88080ED24EC2F3
:100BE0004C10101C92520800080808024002424CA7
:100BF00010149814920808080806001B75B13100FB
:100C00001C925252000C92524C001C925C90000EAE
:100C1000D24EC2000ED010100006C8049808080E6C
:100C2000C807001252524F0011312A4400113135C9
:100C3000BB00124C8C9200112A4498001EC4881EDE
:100C400006C48C8486080808080818080C88180050
:100C5000000C8360000000000100000002000000A2
:100C60000300000004000000050000000600000072
:100C70000700000008000000090000000A00000052
:100C80000B0000000C0000000D0000000E00000032
:100C90000F0000001000000012000000140000000F
:100CA00016000000180000001A0000001C000000E0
:100CB0001E000000200000002300000026000000AD
:100CC000290000002C0000002F000000320000006E
:100CD000360000003A0000003E0000004200000024
:100CE000460000004B0000005000000055000000CE
:100CF0005A00000061000000680000006F00000062
:100D0000760000007D000000840000008B000000E1
:100D10009200000099000000A0000000A700000061
:100D2000AE000000B5000000BC000000C3000000E1
:100D3000CA000000D1000000D8000000DF00000061
:100D4000E6000000ED000000F4000000FB000000E1
:100D5000FF000000B40D0100F1540000BF0D0100C0
:100D6000D1560000CA0D0100E55A0000D40D010063
:100D7000F1560000E10D010055580000E80D01009A
:100D8000A5580000F10D0100F5580000FD0D01000F
:100D9000ED5700000E0E01007D5700001E0E0100F1
:100DA000E55900002B0E010049570000646973707B
:100DB0006C6179006C696768744C6576656C006D70
:100DC00062536574436F6C6F72006D624469737037
:100DD0006C6179006D62446973706C61794F66660D
:100DE000006D62506C6F74006D62556E706C6F7444
:100DF000006D62447261775368617065006D625383
:100E000068617065466F724C6574746572006D62DE
:100E1000456E61626C65446973706C6179006E65E2
:100E20006F506978656C53656E64006E656F5069CC
:100E300078656C53657450696E004E6F7420656EF2
:100E40006F75676820726F6F6D206576656E2061C3
:100E50006674657220636F6D70616374696F6E0094
:100E6000436F6D70616374656420466C61736820C4
:100E7000636F64652073746F72650A2564206279FC
:100E800074657320757365642028256425252920E1
:100E90006F6620256400426164207265636F72642E
:100EA00020666F756E6420647572696E6720696E66
:100EB000697469616C697A6174696F6E0025642078
:100EC00025642025642028256420776F72647329A7
:100ED000002564207265636F7264732C2025642082
:100EE000776F7264732C206D617849442025642CDF
:100EF00020636F6D70616374696F6E206379636CDA
:100F0000657320256400526573746F7265642025D3
:100F100064207363726970747300537461727465D2
:100F20006400726164696F00BD0F01000965000013
:100F3000CA0F010005680000DA0F01008567000094
:100F4000E80F010099690000F30F0100216500001E
:100F5000031001009D650000171001008565000069
:100F600026100100496B000032100100C76A000022
:100F70003B1001006B6A000046100100E5690000AB
:100F800051100100216A00005A100100556A00004A
:100F900063100100316500007210010065650000FA
:100FA0007B1001004165000025303878006E6F6EBF
:100FB00065006F74686572007061697200646973BE
:100FC00061626C65526164696F006D65737361671E
:100FD000655265636569766564007061636B65740D
:100FE00052656365697665007061636B657453650E
:100FF0006E64007265636569766564496E746567E1
:1010000065720072656365697665644D65737361C9
:1010100067655479706500726563656976656453C8
:101020007472696E670073656E64496E7465676596
:10103000720073656E64506169720073656E64530B
:101040007472696E67007365744368616E6E656C77
:101050000073657447726F757000736574506F77B5
:101060006572007369676E616C537472656E677444
:1010700068006465766963654944006C6173744D0A
:10108000657373616765494400556E6B6E6F776E6B
:10109000207072696D6974697665205B25733A25E5
:1010A000735D000000000000963007772C610EEEA3
:1010B000BA51099919C46D078FF46A7035A563E9AF
:1010C000A395649E3288DB0EA4B8DC791EE9D5E0D6
:1010D00088D9D2972B4CB609BD7CB17E072DB8E7D5
:1010E000911DBF906410B71DF220B06A4871B9F32A
:1010F000DE41BE847DD4DA1AEBE4DD6D51B5D4F463
:10110000C785D38356986C13C0A86B647AF962FDC7
:10111000ECC9658A4F5C0114D96C0663633D0FFA14
:10112000F50D088DC8206E3B5E10694CE44160D51A
:10113000727167A2D1E4033C47D4044BFD850DD204
:101140006BB50AA5FAA8B5356C98B242D6C9BBDB17
:1011500040F9BCACE36CD832755CDF45CF0DD6DC12
:10116000593DD1ABAC30D9263A00DE518051D7C8B9
:101170001661D0BFB5F4B42123C4B3569995BACF44
:101180000FA5BDB89EB802280888055FB2D90CC665
:1011900024E90BB1877C6F2F114C6858AB1D61C1DE
:1011A0003D2D66B69041DC760671DB01BC20D298FD
:1011B0002A10D5EF8985B1711FB5B606A5E4BF9F8A
:1011C00033D4B8E8A2C9077834F9000F8EA809967D
:1011D00018980EE1BB0D6A7F2D3D6D08976C6491E8
:1011E000015C63E6F4516B6B62616C1CD830658501
:1011F0004E0062F2ED95066C7BA5011BC1F40882DE
:1012000057C40FF5C6D9B06550E9B712EAB8BE8B1E
:101210007C88B9FCDF1DDD62492DDA15F37CD38CA7
:10122000654CD4FB5861B24DCE51B53A7400BCA3A5
:10123000E230BBD441A5DF4AD795D83D6DC4D1A4D7
:10124000FBF4D6D36AE96943FCD96E34468867ADAE
:10125000D0B860DA732D0444E51D03335F4C0AAA4D
:10126000C97C0DDD3C710550AA41022710100BBE50
:1012700086200CC925B56857B3856F2009D466B997
:101280009FE461CE0EF9DE5E98C9D9292298D0B0CC
:10129000B4A8D7C7173DB359810DB42E3B5CBDB779
:1012A000AD6CBAC02083B8EDB6B3BF9A0CE2B603FA
:1012B0009AD2B1743947D5EAAF77D29D1526DB04AF
:1012C0008316DC73120B63E3843B64943E6A6D0DFA
:1012D000A85A6A7A0BCF0EE49DFF099327AE000A45
:1012E000B19E077D44930FF0D2A3088768F2011ED8
:1012F000FEC206695D5762F7CB67658071366C196F
:10130000E7066B6E761BD4FEE02BD3895A7ADA108F
:10131000CC4ADD676FDFB9F9F9EFBE8E43BEB71770
:10132000D58EB060E8A3D6D67E93D1A1C4C2D838FA
:1013300052F2DF4FF167BBD16757BCA6DD06B53F60
:101340004B36B248DA2B0DD84C1B0AAFF64A03369F
:10135000607A0441C3EF60DF55DF67A8EF8E6E311E
:1013600079BE69468CB361CB1A8366BCA0D26F2567
:1013700036E2685295770CCC03470BBBB9160222B4
:101380002F260555BE3BBAC5280BBDB2925AB42BC9
:10139000046AB35CA7FFD7C231CFD0B58B9ED92CDE
:1013A0001DAEDE5BB0C2649B26F263EC9CA36A7543
:1013B0000A936D02A906099C3F360EEB85670772FA
:1013C00013570005824ABF95147AB8E2AE2BB17B61
:1013D000381BB60C9B8ED2920DBED5E5B7EFDC7CE8
:1013E00021DFDB0BD4D2D38642E2D4F1F8B3DD683F
:1013F0006E83DA1FCD16BE815B26B9F6E177B06F3A
:101400007747B718E65A0888706A0FFFCA3B066626
:101410005C0B0111FF9E658F69AE62F8D3FF6B61B3
:1014200045CF6C1678E20AA0EED20DD75483044E55
:10143000C2B30339612667A7F71660D04D476949E3
:10144000DB776E3E4A6AD1AEDC5AD6D9660BDF40F6
:10145000F03BD83753AEBCA9C59EBBDE7FCFB247A9
:10146000E9FFB5301CF2BDBD8AC2BACA3093B3538E
:10147000A6A3B4240536D0BA9306D7CD2957DE5497
:10148000BF67D9232E7A66B3B84A61C4021B685D70
:10149000942B6F2A37BE0BB4A18E0CC31BDF055AE9
:1014A0008DEF022D416C6C207461736B732073742B
:1014B0006F7070656400763231300020257320250E
:1014C00073004D656D6F727920636C656172656440
:1014D000004E6F2066726565207461736B20656EC7
:1014E0007472696573004C53420000006C15010072
:1014F000D1860000791501003584000085150100B2
:10150000058400008B150100158400009115010071
:10151000258400009715010065810000AD150100CC
:10152000AD850000BB1501007D7D0000C5150100E3
:1015300039860000CD150100A5810000D6150100F7
:10154000657E0000E7150100C97F0000F31501006A
:101550009D7E0000FC1501001D7F000004160100A7
:10156000B580000073656E736F72730061636365AD
:101570006C65726174696F6E0074656D706572611F
:10158000747572650074696C74580074696C745970
:101590000074696C745A00736574416363656C65AB
:1015A000726F6D6574657252616E6765006D61671B
:1015B0006E657469634669656C6400746F75636811
:1015C0005265616400693263526561640069326327
:1015D000577269746500693263536574436C6F6355
:1015E0006B53706565640073706945786368616EFC
:1015F0006765007370695365747570007265616426
:10160000444854006D6963726F70686F6E650000C6
:10161000E5000100E1870000EA0001008D8700007D
:1016200057160100E58800000D010100A9870000A0
:101630005C160100FD88000062160100258800008C
:101640006D1601008987000076160100E188000010
:1016500073657269616C00726561640077726974A8
:10166000650077726974654279746573006D6964A9
:101670006953656E64006D69646952656376000044
:1016800014170100B189000021170100B58900007D
:101690002A170100C189000034170100C589000024
:1016A0003D170100C989000042170100CD890000E3
:1016B00047170100D189000053170100D5890000A8
:1016C0005A170100D989000063170100DD89000065
:1016D00068170100E189000075170100E589000025
:1016E00083170100E98900008F170100ED890000D0
:1016F0009A170100F1890000A5170100F589000083
:10170000AF170100B9890000B9170100BD890000B9
:10171000746674007365744261636B6C69676874A6
:101720000067657457696474680067657448656923
:1017300067687400736574506978656C006C696ED5
:1017400065007265637400726F756E6465645265DE
:10175000637400636972636C6500747269616E67BB
:101760006C650074657874006465666572557064B4
:101770006174657300726573756D6555706461742D
:101780006573006D657267654269746D61700064B0
:1017900072617742756666657200746674546F751F
:1017A0006368656400746674546F75636858007488
:1017B0006674546F7563685900746674546F75630A
:1017C000685072657373757265007661727300009C
:1017D000F0170100858E0000FA170100658E0000E9
:1017E00003180100418E00000F180100CF8D00008A
:1017F000766172457869737473007661724E616DBB
:101800006564007365745661724E616D656400763F
:1018100061724E616D65466F72496E6465780057FE
:10182000656C636F6D6520746F204D6963726F42E4
:101830006C6F636B732100705F73706920213D20B2
:101840004E554C4C002F686F6D652F6769742F2EB5
:10185000706C6174666F726D696F2F7061636B611C
:101860006765732F6672616D65776F726B2D61723C
:101870006475696E6F6E6F726469636E7266352F20
:101880006C69627261726965732F5350492F5350AE
:10189000492E63707000535049436C6173733A3A38
:1018A000535049436C617373284E52465F535049FD
:1018B0005F547970652A2C2075696E74385F742CBA
:1018C0002075696E74385F742C2075696E74385F8A
:1018D0007429000000000000000000005990000082
:1018E000159000003B900000459000004F900000D4
:1018F000399000000000000001000000020000001C
:1019000016000000040000000500000006000000B2
:101910000700000008000000090000000A000000A5
:101920000B0000000C0000000D0000000E00000085
:101930000F0000001A0000001B000000140000004F
:10194000130000001100000017000000100000004C
:101950001C0000001D0000001E000000120000001E
:10196000150000000300000018000000190000002E
:10197000000000000000000045940000799C000079
:10198000C5940000D9940000CF9400004194000059
:1019900035940000E594000061940000319400004B
:1019A000000000000000304300000000000030C3D1
:1019B000706F77007371727400000000FB21F93FB3
:1019C000FB2109407CD91240FB2119407A6A1F4053
:1019D0007CD92240BBFD2540FB2129403A462C40C2
:1019E0007A6A2F405C4731407CD932409C6B34404E
:1019F000BBFD3540DB8F3740FB2139401BB43A40FB
:101A00003A463C405AD83D407A6A3F404C7E40407E
:101A10005C4741406C1042407CD942408CA243401C
:101A20009C6B4440AC344540BBFD4540CBC6464072
:101A3000DB8F4740EB584840FB21494083F9A20027
:101A4000444E6E00FC291500D1572700DD34F50007
:101A500062DBC0003C999500419043006351FE0059
:101A6000BBDEAB00B761C5003A6E2400D24D420028
:101A70004906E00009EA2E001C92D100EB1DFE0091
:101A800029B11C00E83EA700F535820044BB2E00BA
:101A90009CE98400B4267000417E5F00D691390035
:101AA000538339009CF439008B5F840028F9BD0012
:101AB000F81F3B00DEFF97000F980500112FEF0085
:101AC0000A5A8B006D1F6D00CF7E360009CB2700B0
:101AD000464FB7009E663F002DEA5F00BA277500AB
:101AE000E5EBC7003D7BF100F739070092528A0011
:101AF000FB6BEA001FB15F00085D8D0030035600EC
:101B00007BFC4600F0AB6B0020BCCF0036F49A00A3
:101B1000E3A91D005E619100081BE6008599650040
:101B2000A0145F008D40680080D8FF0027734D002F
:101B300006063100CA561500C9A873007BE2600092
:101B40006B8CC0000000000000000040FB21F93F4A
:101B5000000000002D44743E000000809846F83CD0
:101B60000000006051CC783B00000080831BF039FE
:101B70000000004020257A38000000802282E336F1
:101B8000000000001DF369350200000003000000A2
:101B900004000000060000000CC80000B6C70000EA
:101BA000B6C70000E4C80000B2C70000B2C700001A
:101BB000DAC80000E4C80000B2C70000DAC80000BC
:101BC000B2C70000E4C80000E8C80000E8C8000090
:101BD000E8C80000F0C80000E8D200005AD10000B8
:101BE0009ED1000002D100009ED100008ED20000E4
:101BF0009ED1000002D100005AD100005AD100004D
:101C00008ED2000002D10000FAD00000FAD000000D
